:020000040800F2
:1000000000200010B1EF020819270208B1ED000826
:1000100015270208112702080D270208000000001A
:100020000000000000000000000000000927020896
:1000300005270208000000000127020875B000082B
:1000400019F0020819F0020819F0020819F0020864
:1000500019F0020819F0020861BC00088DBD000803
:1000600051BD000815BD0008D9BC00089133000837
:1000700081330008713300086133000851330008F0
:100080003D3300082933000819F0020819F002086E
:10009000992A020819F0020819F002089DBC00080C
:1000A0007DF70008DDF700086DF7000805F8000887
:1000B000CDF70008BDF70008ADF7000819F00208F9
:1000C00019F0020819F0020819F0020819F00208E4
:1000D00019F00208A1B1000825B10008A9B0000874
:1000E00025BC000819F00208F126020819F00208E0
:1000F0008DF7000819F002089DF7000819F00208B2
:1001000000000000000000000000000019F00208DC
:1001100019F0020819F0020819F0020819F0020893
:100120001533000801330008ED320008D932000809
:10013000C532000819F002080000000000000000AD
:1001400019F0020819F0020819F002080000000076
:10015000000000000000000000000000000000009F
:10016000000000000000000019F0020819F0020869
:1001700019F002080000000000000000000000006C
:080180000000000019F0020864
:10018800002870B51EDB0928044620DD012303EB97
:1001980083035B00B0FBF3F2092AF8D87BB10E4E5B
:1001A800B4FBF3F00928CCBF57223022A6FB03E5A5
:1001B800024403FB1044EB0801F8012BF0D10023A3
:1001C8000B7070BD2D230B7040420131DBE73030DE
:1001D80001F8010BF3E700BFCDCCCCCC884230B49A
:1001E8004FF001042ED301FB04F4B0FBF4F58D426B
:1001F800F9D284B1AAB901E0B0FBF4F5092DCCBF5E
:10020800572230222A4404FB150003F8012BB4FBC3
:10021800F1F4002CF0D100221A7030BC7047B0FB0A
:10022800F4F5092DCCBF372230222A4404FB1500EF
:1002380003F8012BB4FBF1F4002CF0D100221A7062
:1002480030BC70470546002AEBD1D7E703685A1C33
:1002580002601970704700BF2DE9F047089C2578A7
:10026800002B804689460CBF4FF0200A4FF0300A19
:10027800661C35B3002A29DD334601E0024698B1F1
:1002880013F8011B501E0029F8D1971E60B13D4696
:10029800013D51464046C8476B1C002BF8DC2578C9
:1002A80027EAE770013055B1041B29464046C84784
:1002B800301916F8015B002DF7D1BDE8F087BDE8CD
:1002C800F087002A04DC2846BDE8F0870020EBE729
:1002D800571EDCE70A44914251D030B441F2210460
:1002E80011F8013B80EA0320430010F4004F84EA30
:1002F80003059BB2ADB208BF1D466B0015F4004F55
:1003080084EA03009BB280B208BF1846430010F489
:10031800004F84EA03059BB2ADB208BF1D466B00CF
:1003280015F4004F84EA03009BB280B208BF184658
:10033800430010F4004F84EA03059BB2ADB208BF36
:100348001D466B0015F4004F84EA03009BB280B28F
:1003580008BF1846430010F4004F84EA03059BB217
:10036800ADB208BF1D466B0084EA030015F4004FC8
:1003780085B298B218BF28468A42B1D130BC7047BE
:1003880083684268D0ED037A00EB8301013393421E
:1003980081ED040A836004BF0023836000EB8303BC
:1003A80093ED047A036870EE277A9A42C0ED037AD7
:1003B80077EEC77AC0ED037A0CDA013307EE103A0C
:1003C800F8EEC76AB7EE007A87EEA60A036030EE49
:1003D800070A704707EE102AB8EEC77A87EE870A31
:1003E800704700BF90ED097A90ED004AD0ED0A6A97
:1003F800D0ED014AD0ED047A90ED035AD0ED025ABF
:10040800A4EE007AB0EE406AB0EE470AB0EE667A23
:10041800A6EE247A67EEC07AA0EE457AE6EE257A53
:1004280080ED097AC0ED0A7A704700BFD0ED057AF1
:1004380090ED013AD0ED003AD0ED064A90ED024A2F
:1004480090ED077A90ED035A90ED086AD0ED045AC2
:10045800C0ED067AF0EE406A27EE830AC0ED056A21
:10046800A3EEA60A80ED087AA4EE240AA5EE470AB0
:10047800A5EEC60A80ED070A704700BFD0ED007AE6
:1004880090ED017A30EE670AE7EE007AB0EE670A7F
:10049800C0ED007A704700BF704700BFF0B540F666
:1004A800280340F62C0240F6360440F6210140F6B7
:1004B8004D1740F66A1640F6E1050380428040F683
:1004C800781340F681124481818140F6611440F628
:1004D800D901C781068240F6330740F6F8064582FF
:1004E800838240F6A71540F6C713C282048340F6FC
:1004F800E71240F64114418340F659118783C683B9
:1005080040F6491740F60C060584438440F6011569
:1005180040F621138284C48440F6010240F6120496
:10052800018540F62F114785868540F62E1740F63F
:100538000A168586C38640F6881540F6C8030286E3
:10054800C485012240F68B04C18740F6381187879D
:10055800A0F8446005878380C380038140F6181C97
:10056800428640F6A10E40F6C1074FF00136448797
:100578004FF0011580F85C204FF00124A0F84010DE
:1005880014220A490A4BA0F842C0A0F846E0A0F895
:100598004870C0F84A60C0F84E50C0F85240C0F8E1
:1005A8005E1080F856208365F0BD00BF000A010A7E
:1005B800980864004FF480530382704750F8043C55
:1005C800012280F83520143803B11847704700BF5E
:1005D80090F8493013B1002280F849201846704736
:1005E80070B5044682B00830256A6B4606223B2166
:1005F800A847A8B19DF804009DF800609DF8011077
:100608009DF802509DF803209DF8053041EA062127
:1006180043EA002342EA05226182A282E3820120A2
:1006280002B070BD30B490E81200057B4369022225
:10063800AA404A602268586A996A4FF6FE752A40AD
:100648008842226004D1012283F8442030BC7047DC
:100658009C695A6B0C44D4600DD818690024411A5F
:1006680051609C621168002041F0010183F8440048
:1006780030BC11607047411A51609862F2E700BFC0
:1006880070B40468037B2268022101FA03F31A425A
:1006980013D042690A49582000FB02124FF6FE7631
:1006A80050685289C5680068296831402960C16866
:1006B800D24392B20A40C260636070BC704700BF08
:1006C8001C56002030B4094B1C7864B1084B002537
:1006D80003EBC4041A6899885562D068083301434B
:1006E800A342D160F6D130BC704700BF3C5A00200D
:1006F800405A002010B40268047B11680223A3400A
:10070800194209D00649406800240C7001684FF668
:10071800FE742140016053605DF8044B704700BFD0
:10072800215E00202DE9F0410446164D0846164684
:100738000F462DF05BFF2A68023011689072D47260
:100748003B4610464F6922460221B84728680E4B9F
:100758000268C47215218172576914212246B8476C
:1007680030462DF043FF296816300D688872CC7228
:1007780022466C6933460846A4461621BDE8F04176
:10078800604700BF04220020B8400308014B1868E6
:100798000AF07CBD689A0020F0B5044690F84D0038
:1007A80083B0002840F0A780694E3779002F43D0E6
:1007B80004F11805A0692CF0FBFB94F846201A21D7
:1007C80028460AF099F801200AF058FBA0692CF095
:1007D800DDFB284694F85C10256D6B460622A84779
:1007E800D0B19DF802609DF803309DF800509DF847
:1007F80001109DF804009DF8052043EA06231BB26A
:10080800E3845BB241EA052142EA00220133A18474
:10081800228506D003B0F0BDB4F926305BB20133AF
:10082800F8D194F924300133F4D1062025F03CFAAC
:10083800484B494ADA60EDE7254655F8180F2CF081
:10084800B7FB80226B2128460AF056F896200AF05A
:100858006FFB0322682128460AF04EF896200AF01A
:1008680067FB03226B2128460AF046F80F200AF09E
:1008780005FB10226A2128460AF03EF80F200AF0EC
:10088800FDFA3A466C2128460AF036F80F200AF09D
:10089800F5FA94F84820192128460AF02DF80F2077
:1008A8000AF0ECFA18221B2128460AF025F80F2036
:1008B8000AF0E4FA10221C2128460AF01DF80F203D
:1008C8000AF0DCFA1022372128460AF015F80F2022
:1008D8000AF0D4FA0122382128460AF00DF80F2030
:1008E8000AF0CCFAA0692CF051FB01200AF0C6FAF4
:1008F800012333715EE70AF0DBFC0546D8B12023FB
:1009080000218371C1710AF069FF2146134B41F838
:10091800143F28462BF078FCAB88B3FA83F3C3F175
:100928001F035A1C3FF440AF01229A400C490B6840
:1009380013430B6038E701460AF050FF2146074B86
:1009480041F8143F28462BF05FFC0122EEE700BF78
:100958000422002000ED00E00400FA05C5050008A7
:100968000004014070B582B00446694618302BF087
:10097800ABFCA8B19DF805009DF801609DF8021038
:100988009DF803509DF804209DF8063041EA0621A1
:1009980043EA002342EA0522A184E2842385012058
:1009A80002B070BDF0B5064683B00D46002401279D
:1009B80014E003290CBF03220122C3F3011E694678
:1009C800C3F3810330468DF805208DF806E08DF8D5
:1009D80007301BF0D1FC0134102C0FD02B8807FAFC
:1009E80004F21342F7D0AB78E9780092022903F0B9
:1009F80003028DF80420DCD10A46DEE703B0F0BD1F
:100A0800F8B51A4D2B789F2B2ED16B78BE2B2BD196
:100A180005221749A81C30F04BFF28BB072229469E
:100A28004FF6FF70FFF756FC124FEC1D22884AB1B3
:100A3800A618BE4218D2052A16D92146FFF74AFC45
:100A48003446F3E721460222FFF744FC0222A118AC
:100A5800FFF740FC0634084B641B1C8041F60F531B
:100A6800C31A58425841F8BD0020F8BD00F00308E9
:100A7800B040030800000408B02900202DE9F04F19
:100A8800DFF86091504F8DB00326A7EB09071822B5
:100A98000DEB0200002130F0C0FE4C4BCDF8189051
:100AA80007971A69120604D5494A5A6002F1883232
:100AB8005A6001228DF82C203422DA60454B464CCE
:100AC80018689A8804909B79ADF8142004A9072225
:100AD80006A88DF816300BF0ABFB072204A94FF6D9
:100AE800FF70FFF7F7FBDFF800B180464FF0000A10
:100AF8005C4536D30CAC002524F82C5D0222214637
:100B080006A80BF095FB022221464046FFF7E2FBC0
:100B180040BAC043ADF80800022202A906A80BF0AB
:100B280087FB099860B108ABC0F104022946184454
:100B380030F073FE089906A80BF020FB09950A907F
:100B48009DF82C300A9A23B120490B6943F08003A1
:100B58000B61013E2DD0002A99D1FFF751FF50B308
:100B68002FE065888DF80DA0C5F30B05AA1DADF81B
:100B780008202288C2F30B01120BADF80A108DF879
:100B88000C2002A9062206A80BF052FB062202A995
:100B98004046FFF79FFB616880462A4606A80BF08F
:100BA80047FB616840462A46FFF794FB14348046A9
:100BB8009EE7002AD1D0052025F076F8074B084A91
:100BC800DA600DB0BDE8F08F000004080020024094
:100BD800230167458C190308A078030800ED00E09D
:100BE8000400FA0500F00308B07C03080378202B02
:100BF800024600F10100F9D0092BF7D02D2B2CD09B
:100C08002B2B03BF5378B7EE000A0246B7EE000A53
:100C1800A3F13001C8B209289FED467A10D8F2EE48
:100C2800046A07EE901AF8EEE77A12F8013FE7EE49
:100C3800267AA3F13001C8B20928B0EE677AF0D954
:100C48002E2B4CD003F0DF03452B0BD0F7EE007AA8
:100C580067EE276A20EE260A70475378BFEE000A2F
:100C68000246D5E710B451782D2959D02B290ABF4F
:100C78009178501C901C0024A1F13003092B53D803
:100C8800002303EB830301EB430310F8011FA1F1D9
:100C98003002092AA3F13003F3D9B3F59A7F28BFAC
:100CA8004FF49A73072B42D9DFED236A1A46F7EE01
:100CB800007A083A072A67EEA67AFAD803F00703FB
:100CC8002BB1F2EE046A013B67EEA67AFBD124B39E
:100CD800C7EE276A5DF8044B20EE260A7047537862
:100CE800A3F13001C8B2092802F10102AAD8F2EE34
:100CF800046AF0EE665A07EE901AF8EEE77A12F8F0
:100D0800013F87EEA66AA3F13001C8B2092866EE52
:100D1800A56A37EE067AEED994E767EE276AD9E72F
:100D2800901C91780124A7E7F7EE007ACFE7F7EE59
:100D3800007AC5E70000000020BCBE4CB5EEC00A32
:100D4800DFED317AF1EE10FACCBF30EE270A30EE43
:100D5800670ADFED2E7A20EE270A30B5FDEEC07A5D
:100D680087B017EE904A054684EAE470002303A989
:100D7800A0EBE47001930093029325F0E1F8002CB6
:100D8800ACBF20232D2303A88DF800302DF02EFCB6
:100D9800012803A924D002282DD0032805BF302319
:100DA800684668468DF8013030F05DFD68462DF0E4
:100DB8001DFC0338C4B222466946284630F0B1FD0E
:100DC80000232B5528462DF011FC2E22431C2A54B3
:100DD8000DEB0401E81830F063FD284607B030BD7C
:100DE800302368468DF801308DF802308DF80330D5
:100DF80030F039FDDAE7302368468DF801308DF898
:100E0800023030F030FDD1E76F12033A00007A4427
:100E18002DE9F041064615460846B6FBF2F43CB902
:100E280005FB1464124B1B5D00F8013BBDE8F08123
:100E3800B4FBF2F767B90E4B05FB174705FB1464C3
:100E4800DA5D00F8012B1B5D00F8013BBDE8F0817D
:100E5800B7FBF2F8B8F1000F02D04046FFF7D8FF11
:100E680005FB1878024B13F8082000F8012BE3E77C
:100E7800BC40030830B402681146531C036011F8E3
:100E8800024B0160D31C517803609378151D0560EF
:100E98001B0443EA0123D078234343EA006030BCB3
:100EA800704700BF0368591C1A46016012F8021BFC
:100EB8000260587841EA0020704700BF38B5044600
:100EC800006815462EF092F922682A44226038BD3F
:100ED800036810B40A0A5C1C04601A7003685A1C80
:100EE800026019705DF8044B704700BF03685A1C14
:100EF800026010B4197003680A0A5C1C04601A7056
:100F080003680A0C5C1C04601A700368090E5A1CFA
:100F1800026019705DF8044B704700BF03685A1CE3
:100F2800026019700368090A5A1C02601970704738
:100F38002DE9F047002488B080460F461E46A1469A
:100F480005AD531C0393117839B3252933D1931C6C
:100F5800CDF810900393507830284ED04FF0000A07
:100F6800A0F13003DBB2092B42D96C2819D06428D0
:100F780000F0938024D825281CD063D9582876D02F
:100F880063281BD131784046B847039A531C039312
:100F98001178043601340029D7D1204608B0BDE8BD
:100FA800F087039B5A1C03921B78642B7CD02AD8A9
:100FB800252B54D1252140460134B847039AC0E770
:100FC800732833D044D975284FD106F1040E306800
:100FD8002B4600220A217646FFF700F9049A00956D
:100FE800534639464046FFF737F9039A0444A8E7C1
:100FF80004AA03A924F080FFB7E7D31C03939078D1
:101008004FF0010AACE7732B10D05BD9752B3AD09F
:10101800782B96D1A3F15802B2FA82F230685209BD
:101028002B4610210436FFF7D9F8D7E73368049A1E
:101038000093394600234046FFF70EF9043604446E
:10104800039A7EE70028B9D1204608B0BDE8F087AA
:101058006E28B3D1039A336804361C6071E72AD925
:10106800582BD7D0632B8DD06BE77828A6D1A0F169
:101078005802B2FA82F2306852092B461021FFF763
:10108800ADF80436AAE706F1040E30682B460022B4
:101098000A217646FFF7A2F8A0E7331D30682946F3
:1010A8001E46FFF76DF899E7331D306829461E463E
:1010B800FFF766F892E7002B7FF443AF204608B0AD
:1010C800BDE8F0876E2BC6D03BE700BF0EB400B575
:1010D80084B005AB019053F8042B0649039301A88B
:1010E800FFF726FF019B00221A7004B05DF804EB9D
:1010F80003B07047550200080FB430B583B006AB93
:101108000B490C4853F8042B096800680193FFF752
:101118000FFF094C0546206803685B69984700285B
:10112800F9D0284603B0BDE8304004B0704700BF8E
:10113800B04C0020B44C0020689A0020DFED2B7AD8
:10114800B4EEE70AF1EE10FA4ADDDFED296A9FED09
:10115800297A01E0B0EE670AB4EEC70AF1EE10FA98
:1011680070EE667AF6DC9FED247AF4EEC77AF1EE3B
:1011780010FA38D5DFED1E6A9FED207A01E0F0EE17
:10118800407AF4EEC77AF1EE10FA37EEA60AF6D4F2
:10119800DFED1B7AB4EEE70AF1EE10FA14DDDFEDAD
:1011A800137A37EEC00A60EE006A9FED166A9FED6B
:1011B800167ADFED167AA6EE867A20EE266AE6EE35
:1011C800877AA6EE270A7047DFED117AB4EEE70AB0
:1011D800F1EE10FA44BFDFED087A37EEC00AE2E715
:1011E800F0EE407ABFE7B0EE670AD1E7DB0F49407F
:1011F800DB0FC940E4CB1641DB0F49C0E4CB16C175
:10120800DB0FC93F92E741B99730083C15A82ABEC1
:10121800DB0FC9BF41404A0011F0800F82F0D503AF
:10122800D2B2DBB208BF1346590013F0800F81F029
:10123800D502C9B2D2B208BF0A46510012F0800FD7
:1012480081F0D503C9B2DBB208BF0B46590013F0D1
:10125800800F81F0D502C9B2D2B208BF0A46510048
:1012680012F0800F81F0D503C9B2DBB208BF0B467C
:10127800590013F0800F81F0D502C9B2D2B208BF6D
:101288000A46510012F0800F81F0D503C9B2DBB2D3
:1012980008BF0B465A0082F0D50013F0800FD2B277
:1012A800C0B208BF1046704709B909E0194690FB5B
:1012B800F1F301FB13030846002BF7D108467047EA
:1012C8000146FBE710B507EE901A2DED028BB8EE3C
:1012D800678ADFED227A28EE008A044628EE278AFC
:1012E800B0EE480A2EF0D8F9F0EE408AB0EE480A7F
:1012F8002EF034F9F7EE007A9FED197AF0EE675A7E
:10130800E8EE875A0023A361B0EE676AC7EEA56AC4
:1013180063612362E361A3626362A8EEC76ABDECFE
:10132800028B77EEC07AB6EE007AF8EE005A27EE16
:10133800877A20EE250A27EE267A26EE266A67EEB9
:10134800A67A20EE260A84ED046AC4ED017A84EDBB
:10135800007A84ED027A84ED030A10BD27D4D236D0
:10136800F304353F10B44C09012250F8243001F041
:101378001F0102FA01F10B4340F824305DF8044BD9
:10138800704700BF4B0901F01F0150F823200123CB
:1013980003FA01F1114214BF18460020704700BF3C
:1013A800BB4B33F81020110566D52DE9F043B94938
:1013B8000446400904F01F0551F820000121A94006
:1013C80001428DB005D0B449097811B10DB0BDE81E
:1013D800F08302F01F07C2F34415242CF6D801A2AB
:1013E80052F824F0BF140008EB1400086115000837
:1013F80085150008D5160008331C0008331C0008A2
:10140800B11B0008F51B00085D170008EB1C00085D
:10141800B31C0008511D0008D5130008D513000897
:10142800A5170008C9170008E9170008FB170008E6
:101438000D180008351800084F1800088318000810
:10144800D5130008D5130008EB1800084B1B00083B
:101458004B1B0008891A0008971B0008D5130008C1
:10146800D513000811190008751900088B19000810
:10147800E7190008831400087047DFF84C82D8F891
:1014880020200AB1B2F90820844904AE3046FFF79B
:101498001DFE30462DF0AAF8D8F800403844A07256
:1014A8002068E5722A463346456939462046A847EA
:1014B8000DB0BDE8F0837A4B78491B88DFF80882C5
:1014C800642202FB03F29212632A4FF00103A8BFC1
:1014D80063220DF111008DF8103004AEFFF7F6FD10
:1014E800D7E7704B704A1B781088022B00F0A8844D
:1014F8006E4B6F4C5A781978247802EB82025200AE
:1015080000EB800301EB81015B0093FBF4F39B1A72
:10151800C3EBC303C2EB410293FBF2F3062BA8BF54
:10152800062323EAE373C3F19603DBB2614A8DF81D
:101538001030A2FB0032D20802EB8203A0EB430377
:101548005D4906209BB200900DF11100FFF7BEFD2A
:1015580004AEDFF874819CE7DFF86C81D8F80000EE
:1015680003681B6998470CAEB0F5F07F534B46F8FB
:10157800203D0CBF072506250D278AE7504BDFF8CD
:101588004881B3F90070D8F80000B3F90250026836
:101598004C491369B7F5C87FA8BF4FF4C877C82D61
:1015A800A8BFC8256FF0C7028F42B8BF0F46954243
:1015B800B8BF15469847B0F5F07F18BF0224002D34
:1015C800B8BF0735ED10BB0048BF3F33A5F129066A
:1015D800C6EBA313512B40F26A8507EB4705002D94
:1015E8002B46B8BF05F13F03C6EBA313512B40F2BE
:1015F8004185ED1B002D2B46B8BF05F13F03C6EB17
:10160800A313512B40F21985ED1B002D2B46B8BFB3
:1016180005F13F03C6EBA313512B40F2F184ED1BF8
:10162800002D2B46B8BF05F13F03C6EBA313512B82
:1016380040F2C984ED1B002D2B46B8BF05F13F03CE
:10164800C6EBA313512B40F2A184ED1B002D2B46B2
:10165800B8BF05F13F03C6EBA313512B40F27984C1
:10166800ED1B002D2B46B8BF05F13F03C6EBA313B6
:10167800512B40F25184ED1B48BF3F35C6EBA516F0
:10168800512E40F20B840420FFF78AFE9EE600BF2D
:1016980004340020145E00200000002004410308E8
:1016A800C85B0020CB5B002018410020D05B0020E5
:1016B8004F410020CDCCCCCC08410308267E270022
:1016C800983D002070FEFFFF04220020DFF8AC8365
:1016D800D8F8000003681B699847B0F5F07F0CBF85
:1016E8000727062707F1040614BF03240424082546
:1016F800D8F800000368C4728572D3F8189022469F
:1017080013230721C847D8F8000016220368C472BB
:10171800827222460134D3F8189015211323E4B2BB
:10172800C847A642E4D1D8F8000009220368C77266
:1017380082729C693A4603230821A047D8F8000022
:1017480015220368C77282729C693A4602231421E3
:10175800A0473BE6AB4BAC4AB3F90630AB49DFF8E0
:101768001C83B3F5FA6FA8BF4FF4FA63B3F57A7F19
:10177800B8BF4FF47A73A3F57A7382FB0302DB17C1
:10178800C3EBA202042405230DF112008DF81040CA
:101798008DF8113004AEFFF799FC7AE693F85C30C7
:1017A8009B49DFF8D882002B0CBF0F220C2204AE15
:1017B80000230192304600932022FFF787FC68E659
:1017C800944B954A18689549847803780194407831
:1017D800009004AE3046FFF779FCDFF8A08258E6A7
:1017E8008C4B8F4A18688D494479C37801940079E5
:1017F800EEE7884B8B4A18688849047A8379019404
:10180800C079E5E7884A894B10881B68884A894966
:10181800DFF8688203FB00F382FB030204AEDB17E8
:10182800C3EBA2123046FFF751FC32E6824A8349E5
:1018380053781278DFF8448204AE0133013230461F
:10184800FFF744FC25E600217D48FFF79BFD20B10A
:101858007C4B1B88002B40F05A847B4B1B78012B58
:1018680000F05183022B40F0408304AE30467749A4
:10187800DFF80882FFF72AFC0BE66B4B724A1B88DD
:101888001278734903EB8303022A09784FEA43036A
:1018980093FBF1F300F0D2826E4A5178127801EB93
:1018A8008101490002EB82005A1AC2EBC202C1EB65
:1018B800400192FBF1F2062AA8BF062222EAE27250
:1018C800C2F19602D2B264488DF8102080FB032042
:1018D800DA17C2EB601264246049062004FB123355
:1018E80031E65F485F49B0F90230B0F90020B0F93D
:1018F8000640B0F90400009004AE01943046FFF7AA
:10190800E5FBDFF87881C4E5574B3F4AB3F904306B
:1019180056485749DFF8648182FB0342DB17C3EB63
:10192800A2031BB203F5B47480FB04621619E21714
:10193800C2EB26224FF4B47606FB1242520080FB1B
:1019480002401044D217C2EB6012D2B2C2F11802A0
:10195800504200F00F0002F00F0258BF42426032BE
:1019680004AED2B23046FFF7B1FB92E504AE0023D5
:101978003046009368223F49DFF80081FFF7A6FB55
:1019880087E5394B204AB3F9043038483A49DFF83B
:10199800EC8082FB0342DB17C3EBA2031BB203F507
:1019A800B47280FB02439C18D317C3EB24234FF473
:1019B800B47404FB13235B0080FB03021A44DB1797
:1019C800C3EB621351FA83F304AE186859681C7AA2
:1019D800334603C300221C708DF8192059E5DFF83F
:1019E8009C80D8F820300E228DF81020002B00F0B3
:1019F8008C8393F9012005490DF11100FFF766FB6F
:101A080004AE46E5445E0020676666660441030846
:101A18001C410308C83400205C41030860410308E6
:101A28007041030874410308184100201C4100203C
:101A3800D34D621078410308003600207C4103082A
:101A480068300020005C0020CB5B00209441030834
:101A58004F410020D05B00201F85EB51AC410308AB
:101A680084400020B8410308983D0020B7600BB6B9
:101A7800E4410308EC4103089419030804220020F8
:101A8800BA4BBB4ADB889268BA499A1A9A42A8BFED
:101A98001A4622EAE27207EE902AA1FB0313DB083A
:101AA800B8EEE77A07EE903AF8EEE77AC7EE276ADB
:101AB80016EE900A2CF006FF41EC100B2DF074FC8A
:101AC80051EC100B2DF0ECF98A23C0B28DF81030D0
:101AD800002840F0A9818D238DF811308D238DF8D1
:101AE8001230022800F276818D238DF813308D2371
:101AF8008DF814308D238DF815308D238DF8163020
:101B08008D238DF817308D238DF818308D238DF89F
:101B180019308D238DF81A308D238DF81B30431E14
:101B28008F22092B8DF81C2004D80CAB18448E2367
:101B380000F81F3C00238DF81D3004AEDFF85C82EE
:101B4800A7E48D4B8D488E49DFF850821A2C0CBFC4
:101B5800B3F90220B3F9002080FB0230D317C3EB9E
:101B6800A00404EB8400A2EB400383EAE370002A9C
:101B7800A0EBE37004AE84EAE4730090ACBF2022CB
:101B88002D22A3EBE4733046FFF7A0FA81E47D4BE6
:101B98001B78DB073FF51AAC04AE30467A49DFF80C
:101BA800FC81FFF793FA74E4784B1B68DE0040F180
:101BB8004A81774B0322774909884C0500F1D38085
:101BC800C80700F18C8201F00201734800291CBF8C
:101BD80003220346714908683A4404688272C57250
:101BE80039462A466469A047FFF7F0BB6C4B1A795F
:101BF800002A00F06C811C1D03F114080DF10F0977
:101C080026782DF0D3FA30440134437803F00303E7
:101C1800022B14F8013C08BF203E09F8016F002B85
:101C28003FF496ACA045EBD192E403EB4403B3F840
:101C3800543013F00F0200F01A81022A8CBF2021C1
:101C48009C21012AC3F303148DF8101000F04A8276
:101C5800C0F01281022A40F04F82DFF840815149DA
:101C6800D8F81800504AA1FB0031890C82FB0132D8
:101C78000A445211C2EB0213A1EB8303012C40F07A
:101C8800EE804A4E4A4C4B49A6FB0060400BA4FB31
:101C980000646409642606FB140000900DF111002D
:101CA800FFF714FA04AEFFF7F4BB314B40481B684A
:101CB8004149DFF8E88083EAE374A4EBE37480FB2E
:101CC8000430E217C2EB6012642000FB12439A242E
:101CD8000DF111008DF8104004AEFFF7F7F9FFF78A
:101CE800D8BB364E316800248DF80D408DF80E4073
:101CF800002900F033820A68D269002A00F00282C3
:101D08000DF10E010DF10D00904731688DF80F406F
:101D180039B10B68196A21B10DF10F0088479DF898
:101D28000F109DF80E4026489DF80D20254B825C2B
:101D3800009104AE53F824302349DFF86080304620
:101D4800FFF7C4F9FFF7A5BB094B20499A68DFF8EC
:101D58004C8007230DF111008DF8103004AEFFF709
:101D6800B5F9FFF796BB0422194B33E7D05B002087
:101D78001C410020A38B2EBA983D0020676666663A
:101D8800CC410308173C0020D841030868300020E4
:101D9800EC4003086C5E0020004103080422002088
:101DA8000036002083DE1B43898888885917B7D1FD
:101DB8001F85EB513441030814410308BC6200201D
:101DC800582203086022030850410308044103080D
:101DD800F04003088B2303288DF813307FF687AE75
:101DE80004288DF814307FF685AE05288DF8153057
:101DF8007FF683AE06288DF816307FF681AE072869
:101E08008DF817307FF67FAE08288DF818307FF6EA
:101E18007DAE09288DF819307FF67BAE0A288DF83B
:101E28001A303FF67AAE77E68B2301288DF8113009
:101E380018BF8DF812307FF454AE4FE6972242E572
:101E48009723FFF773BBCB4ACB491268CB4B02F4FD
:101E58008002002A16BF0B4604220322ABE6C849BB
:101E68000DF11100FFF732F904AEFFF712BB9B2208
:101E7800C3F303148DF8102008F0B4FFC14BC24A15
:101E8800DFF82483A3FB00139B0C82FB03121A4484
:101E98005211C2EB0211A3EB8103EFE6BB4AD8F85B
:101EA800000082FB0632F317C3EB6203E21803EB70
:101EB800C3031324D2B2F61A0168C272A6F18003D2
:101EC80084728C69DBB21221A047FFF7DCBBB04BF0
:101ED800DFF8D48293E8070004AE334603C323F83F
:101EE800022B120C1A70FFF7D4BADFF8BC8298F8EC
:101EF8001C30002B3FF46AAA04AE3046A549FFF710
:101F0800E5F8FFF7C6BA04AE3046A349DFF8988271
:101F1800FFF7DCF8FFF7BDBA9C49D8F8000081FB51
:101F28000321DA17C2EB610204EB020E02EBC201D5
:101F38005B1A5FFA8EF20168C2724FF0120E80F8D7
:101F48000AE0803BD1F81890DBB21121C847FFF7AF
:101F580092BB8E49D8F8000081FB0321DA17C2EB47
:101F6800610204EB020E02EBC2015B1A5FFA8EF209
:101F78000168C2724FF0110E80F80AE0803BD1F878
:101F88001890DBB21021C847FFF76ABB7F49D8F821
:101F9800000081FB0321DA17C2EB610204EB020E99
:101FA80002EBC2015B1A5FFA8EF20168C2724FF04F
:101FB800100E80F80AE0803BD1F81890DBB20F21B0
:101FC800C847FFF742BB7149D8F8000081FB0321DD
:101FD800DA17C2EB610204EB020E02EBC2015B1AD4
:101FE8005FFA8EF20168C2724FF00F0E80F80AE0B5
:101FF800803BD1F81890DBB20E21C847FFF71ABB17
:102008006249D8F8000081FB0321DA17C2EB6102AC
:1020180004EB020E02EBC2015B1A5FFA8EF2016852
:10202800C2724FF00E0E80F80AE0803BD1F818908B
:10203800DBB20D21C847FFF7F2BA5449D8F80000BF
:1020480081FB0321DA17C2EB610204EB020E02EBFB
:10205800C2015B1A5FFA8EF20168C2724FF00D0E70
:1020680080F80AE0803BD1F81890DBB20C21C84711
:10207800FFF7CABA4549D8F8000081FB0321DA17EF
:10208800C2EB610204EB020E02EBC2015B1A5FFABB
:102098008EF20168C2724FF00C0E80F80AE0803BA5
:1020A800D1F81890DBB20B21C847FFF7A2BA37491D
:1020B800D8F8000081FB0321DA17C2EB6102A518EA
:1020C80002EBC2015B1AEAB20168C2720B25803BBF
:1020D80085728D69DBB20A21A847FFF77EBA2F4BBC
:1020E800042277E5DFF8C080264BD8F80800264A96
:1020F800A3FB0013990CB9E50023DFF8AC801A465E
:102108001846BBE58DF80F2003E61A4673E4DE0790
:1021180027D4C3F34002A2B95C074FD418074BD4A5
:10212800D90647D49A0643D45E063FD41C061ED46B
:10213800D8051AD4990516D45A0548BF0A227FF53E
:1021480007AA174B1749DFF8608003EB820204AE39
:10215800126A3046FEF7BAFFFFF79BB98DF80F10E9
:10216800DFE50022EDE70922EBE70822E9E707228D
:10217800E7E700BFE8790020EC400308E4400308E3
:102188002841030883DE1B4389888888398EE33811
:1021980044410308A041030888410308F8400308A4
:1021A8008C19030884410308042200200622C8E78A
:1021B8000522C6E70422C4E70322C2E70222C0E7D9
:1021C8002DE9F04FBA4BBB4C1B788DB005460BB1CF
:1021D80001232377626AB84BA3FB02139B0803EB26
:1021E8008303511CD31A616240F0AB80B34F94F85B
:1021F800280097F8008008F00108404500F0518158
:10220800B8F1000F00F0AD80266863613068A36103
:102218004FF0FA714FF4C6028368E16030462261DC
:1022280098472068DFF8D492DFF8D4A2FF237373AD
:10223800012203683273112107228172C272D3F816
:1022480014809F4B9F4E0C21C04705F5F42101F5E2
:1022580090713160387800F0010084F82800B4F9F2
:102268000C30994AB4F910E01788002BB8BF002346
:102278004FF0640202FB07F2B8BFA381B4F90E70F5
:10228800B9F800309F42C8BFE381904FDAF80030B8
:1022980087FB03C7DB17C3EB67131BB29E45B8BFA9
:1022A8002382B4F91230C2F387229342B4F914306E
:1022B800C8BF6282002BB8BF002384F82920B8BFAA
:1022C800A38238B1E36AA068A269EB1A18441344E0
:1022D800A060A361E56271B1691A0029C0F2768134
:1022E80027683B6838469B6898470121FF220023EE
:1022F80039737A733360764F76493B68764AAD090D
:10230800A1FB0515C5F380151801157000F145826C
:102318002368002B00F06D8193F90E20002A40F30A
:102328006881002222779BB193F90E30002B0FDDD4
:102338006A4A138843F400739BB213800DB0BDE85A
:10234800F08F20680368DB6898472368002BEBD17F
:10235800624A138823F400739BB213800DB0BDE862
:10236800F08FD4F800905E4ED9F8003048469B684C
:1023780098472068FF2389F80D300122036889F8FF
:102388000C20112102228172C272D3F81490554B8D
:102398001146C84796F85230002B40F0FB820A23BA
:1023A8000793092305930823049306234FF007098D
:1023B80003934FF0050B4FF0040A4FF0030896F80B
:1023C8005330002B40F0978296F84A3023B1464BA1
:1023D8001B789B0700F15A8396F85430C3B196F8DE
:1023E8005C30B4F91620002B00F025830C233F49FC
:1023F80009A8FEF76BFE404609AA3D49FEF792F987
:10240800D046DA46DDF80CB0CDF80C90DDF8109027
:1024180096F84B30002B40F0198296F85130DFF8CF
:10242800DC90002B40F04A8296F84C30002B40F0AC
:102438002F82304B5B79002B40F0B481DFF8C0A0CD
:1024480096F84F30002B00F0898096F85C30B4F98C
:102458001400002B58D100EB800300EBC3001B4A8B
:10246800C00082FB0031C317D3EB611100F159831F
:1024780082FB012ECA17C2EB6E124FF0640BDFF815
:1024880078C0DFF880E00BFB12128CFB02C18EFBD8
:1024980000E0D217C2EBA101C3EB203320220F20AA
:1024A8004DE0084EDFF854903168DFF854A0D6E6C6
:1024B800025C002004220020CDCCCCCC173C0020AC
:1024C800F84103081C5E0020C85B00201F85EB5103
:1024D800E8790020632D3E0500000020005C002004
:1024E8000434002000420308703000201C42030816
:1024F80024420308D05B0020676666661841002006
:102508001C410020AD8BDB68BB4BBC4983FB00231F
:10251800C217C2EB6313642202FB130281FB021E83
:10252800D1170028C1EBAE01ACBF20222D22002913
:10253800B8BF4942002B4FF00C00B8BF5B42019076
:10254800009109A8AE49FEF7C1FD08F10103404614
:1025580009AAAC495FFA83F8FEF7E4F896F8503018
:10256800DBB1A94B9B7853B3032B28D0022B00F087
:10257800F5820022114609ABB2FBF1F2184692B27D
:10258800A2490693FEF7A2FD08F101034046069A08
:102598009F495FFA83F8FEF7C5F896F8553073B18E
:1025A800994B9B785BB1032B09D09A4B09A9186901
:1025B80023F0C6FC09AA40469749FEF7B3F89749A5
:1025C800974E294400233160A36143E6954AB2F946
:1025D800061040F2D663994203DCB2F902209A420F
:1025E80001DD00233360206803681B6A984723686D
:1025F80097E68D4E94F8293096F856209A4240F284
:10260800F6808A4D2B6843F00103894A1278002A24
:1026180040F0E88023F4C00323F00203854A1278CF
:10262800910700F1DC8043F48043B6F85E802B60AC
:1026380008F00F02012A00F02782C0F02182022A46
:1026480000F006820020754A4FEA182802FB08F2BB
:10265800002A00F00782824200F2048243F020033D
:10266800B6F860802B6008F00F02012A00F00082A3
:10267800C0F00282022A40F0FD81A069674A4FEA51
:10268800182802FB08F2002A00F0E981824200F2D1
:10269800E68143F04003DAF80820B6F85810914272
:1026A800B6F85A20D4BF43F0102323F01023002A91
:1026B80000F0DB8123F4004326682B603368304642
:1026C8009B6898470122FF233273737313215A487A
:1026D800FEF758FE002886D1584B1B689A0700F170
:1026E8000D820120FEF75CFE0020FEF759FE022055
:1026F800FEF756FE0520FEF753FE0620FEF750FEB5
:102708000720FEF74DFE0920FEF74AFE0A20FEF7D5
:1027180047FE0B20FEF744FE0C20FEF741FE082082
:10272800FEF73EFE0F20FEF73BFE1020FEF738FEB8
:102738001120FEF735FE1220FEF732FE1320FEF7B9
:102748002FFE1420FEF72CFE1520FEF729FE16207A
:10275800FEF726FE1920FEF723FE1A20FEF720FEBC
:102768001B20FEF71DFE1C20FEF71AFE1D20FEF79B
:1027780017FE2020FEF714FE2120FEF711FE22206E
:10278800FEF70EFE3B681B017FF52DAF2320FEF7F9
:1027980007FE2420FEF704FE25E7FF201BF0A2FD1C
:1027A8002062B5E596F84D30002B40F0848196F80C
:1027B8004E30DFF894A0002B3FF442AEDAF8082040
:1027C8001F4909A80723FEF781FC08F101034046C9
:1027D80009AA1C495FFA83F8FDF7A4FF30E623F441
:1027E800804322E743F4C00343F0020316E70F4D8A
:1027F8002B6823F0010308E71F85EB5167666666BF
:102808001C41030878420308414D0020A0420308F8
:1028180088420308284D0020944203080087930348
:102828001C5E0020445E002004340020145E00205A
:10283800CB5B002070300020683000203C4E002028
:102848001C4203086C4203081C410020B4F90E30F6
:10285800C84AC94982FB0302D817C0EBA20202EB9F
:1028680082004FF0060EA3EB40031BB212B2CDF864
:1028780000E009A8FEF72AFC404609AABF49FDF76F
:1028880051FFD046DA46DDF80CB0CDF80C90C4E51F
:1028980009AA1146B4F91200039223F051FB039AD6
:1028A80010462BF0A3FEB64B039A1B881352B5496A
:1028B8004046FDF737FFD046DA46BAE5B9F80030AA
:1028C800B14AAD49A2FB0302D20802EB82004FF0E5
:1028D800060EA3EB40039BB2CDF800E009A8FEF773
:1028E800F5FB404609AAA949FDF71CFFD046DA4680
:1028F800DDF80CB098E5B6F8603003F00F02012A55
:10290800C3F30313069300F0A580C0F00681022AE2
:1029180040F0FF80D4F818E09D4B9E4AA3FB0E13AD
:102928009B0C82FB03121A445211C2EB0211A3EB57
:1029380081030699012940F0DA80DFF880C29648C1
:102948009649ACFB0ECE4FEA5E3EA0FB0EC0400996
:102958004FF0640C0CFB10EECDF800E009A80690CF
:10296800FEF7B4FBB6F860308D49069A03F00F0302
:10297800404651F82310FDF7D5FE059BD046DA46B0
:10298800DDF80CB0CDF80C90DDF810900493079B9F
:10299800059319E5B6F85E3003F00F02012AC3F378
:1029A80003195AD0C0F0B280022A40F0AB80A06967
:1029B800774B784AA3FB00139B0C82FB03121A4443
:1029C8005211C2EB0218A3EB8803B9F1010F40F0D2
:1029D8008780DFF8E8C1DFF8C0E17049ACFB00C0D0
:1029E800400BAEFB00CE4FEA5E1E4FF0640C0CFBB2
:1029F8001E0ECDF800E009A80690FEF767FBB6F8B2
:102A08005E306749069A03F00F03032051F823103C
:102A1800FDF788FE0B2307930A23059309230493E4
:102A280007234FF0080903934FF0060B4FF0050AF0
:102A38004FF00408C3E402EB820302EBC3025649D9
:102A4800D30081FB0321DA17C2EB61120F23CEE416
:102A5800A069F8E5D4F808E05EE7A068A8E723F0E5
:102A6800400318E623F02003FAE543F4004323E685
:102A7800A06803E6002001E608F0B4F92B68FDE53C
:102A880008F0B0F92B68DEE5A068DCE509A9B4F91F
:102A98000C0023F055FA404609AA4249FDF742FEC8
:102AA800059BD046DA46DDF80CB0CDF80C90DDF881
:102AB8001090049390E40DF1240B5946B4F91000DA
:102AC80023F03EFA58462BF091FD374B37491B88C7
:102AD8002BF800305A464046FDF724FED04666E6FD
:102AE80009A9069108463249FEF7F0FA87E709A9CD
:102AF800069108462E49FEF7E9FA33E70320FEF768
:102B08004FFCEEE54346424640465EE708F06AF968
:102B18004EE700231A469E460BE708F063F98646FF
:102B2800FAE682FB01E24FEAE17CDFF894E0CCEBC5
:102B380062124FF0640C0CFB12128EFB00E00D4980
:102B4800C3EB203381FB021E002B4FEAE271A1EB9D
:102B5800AE01B8BF5B420F202D22F0E4154B186878
:102B680009F052F870B309AB184613490693FEF7FB
:102B7800ADFA09E56766666608410308344203084A
:102B88004C42030850420308CDCCCCCC4042030849
:102B980083DE1B43898888881F85EB5134410308ED
:102BA800F8250308104203085C4203086042030842
:102BB800284103086C440020A84203085917B7D1DC
:102BC800AD8BDB680C4B93F82420002ACBD00B4A42
:102BD80051780329C7D141F27810D96B084B1258A4
:102BE800A3FB0101C909A3FB0232A1EB1242642332
:102BF80003FB02F2BFE400BFE096002054820020ED
:102C0800D34D62102DE9F043314A324E13683060DB
:102C1800042B89B004D0304C591C44F823001160AF
:102C28002E4B2F4A1B78002103F0010311605160DD
:102C380086F82830012709F00BF9A0230424FDB2F7
:102C480003E00134E4B21C2C13D0FF2BF9DC30680C
:102C580002688472C572611E0134D2F8188003F1CB
:102C68000109C9B2DBB22A46E4B2C0471C2C4B4664
:102C7800EBD10137052FE1D168461A4A1A49FEF708
:102C880025FA6B4606221421306809F0BDF8174B67
:102C980030680822072109F0B7F8154B3068092277
:102CA8000B2109F0B1F80A220B21124B306809F008
:102CB800ABF8306803685B6A984708F093F80E4BE6
:102CC80000F5741000F51060186009B0BDE8F083D5
:102CD800BC4D002004220020C04D0020173C0020DD
:102CE800145E0020B0420308B8420308BC4203083F
:102CF800CC420308D84203081C5E00202DE9F84F97
:102D0800DFF8B490DFF8B480DFF8B4A0274E0123D1
:102D1800082089F800302AF05FF9D8F8000008F098
:102D280019FF05202AF008F900202AF005F90620E5
:102D38002AF002F900202AF0FFF89AF8004004204F
:102D480044F001042AF0F8F820462AF0F5F8338810
:102D58008BB1174D174F002415F804B007202AF03F
:102D6800EBF858462AF0E8F82A5D33883A550134DA
:102D7800A4B2A342F0D807202AF0DEF8FF202AF0F8
:102D8800DBF89AF8004004202AF0D6F820462AF00A
:102D9800D3F8D8F8000008F0E3FE02202AF01CF966
:102DA800002389F80030BDE8F88F00BFF41F002029
:102DB8000C5C0020845E00206F5E002038640020D8
:102DC800755E00202DE9F0414A4E08202AF004F9EA
:102DD800306808F0BFFE484B1B78012B7BD062D3CC
:102DE800022B0AD1DFF83081082388F800300D253E
:102DF8004FF4C373414F3B8010E0DFF81C813F4F15
:102E080098F8003003F04003002B14BF4FF4F07320
:102E18004FF4C3733B8014BF10250D25002404F123
:102E28001000C0B22AF088F8013401202AF084F892
:102E3800A3B2AB42F3D398F80040314D00202AF0FA
:102E48007BF820462AF078F82E4B1C7802202AF0CE
:102E580073F820462AF070F82B4B1C7803202AF0D0
:102E68006BF820462AF068F8284B1C7804200443A5
:102E78002AF062F820462AF05FF8306808F070FE01
:102E880002202AF0A9F83A88214800212EF0C5FC32
:102E98006B7833B11F4B1B7833B300236B70BDE8DD
:102EA800F081BDE8F081A0202AF046F800202AF041
:102EB80043F800F00603022BDFF85C8007D000F02F
:102EC8000500012803D1482388F8003008E00823CA
:102ED80088F800308BE7DFF84080482388F8003016
:102EE80010254FF4F07385E7FFF708FF00236B7098
:102EF800BDE8F081386400203C640020F41F002005
:102F0800000000204364002044640020755E002017
:102F1800845E00206F5E0020F71F0020F0B5574B3D
:102F2800574A97B01968914200AF00F09C80554904
:102F3800554A00234FF47000C1F888003B607B605D
:102F4800136843F48033136003E03B68B3F5A04F84
:102F580009D0136803F400337B603B6801333B609E
:102F68007B68002BF1D0484B1B6813F4003318BF63
:102F780001237B607B68012B4BD0424D424B434A77
:102F8800EA60434A596A11605A6A424E42F08072B6
:102F98005A625A6907F1580442F4FC0241F6FF717B
:102FA8005A6124F8501D032321464FF09040BB720C
:102FB800FDF7F8FC4FF6FF73214637483B81FDF7D4
:102FC800F1FC21463548FDF7EDFC21463448FDF774
:102FD800E9FC21463348FDF7E5FC21463248FDF778
:102FE800E1FC204618F0D4FFBB683049304AA1FB09
:102FF800031330499B0CF02400204FF0070E5C3778
:103008000B60566085F823409060C2F800E0BD462A
:10301800F0BD294A1C4B122111605A685A605A683F
:103028005A605A6842F480625A605A6822F47C12E4
:103038005A605A6842F4E8125A601A6842F080727C
:103048001A601A689201FCD559680F4A21F00301E9
:103058005960596841F002015960536803F00C0344
:10306800082BFAD189E700221A6062B6134B1B6855
:1030780083F30888124B1B689847FEE7FC9F0020E3
:10308800EFBEADDE00ED00E0001002400005FA05DD
:10309800E47900203F1901000004004800080048B6
:1030A800000C0048001000480014004883DE1B4351
:1030B80010E000E0049A00200020024000D8FF1F22
:1030C80004D8FF1F064A00235168814202F11C02FE
:1030D80004D001330C2BF7D100207047D8B27047C9
:1030E8002400002070B50F4C0F4DC0EBC00004EB5E
:1030F8008004686926693043686182B09209667BFA
:10310800A1600025012101A863618DF804608DF894
:1031180005208DF806508DF8071029F0B3FD02B090
:1031280070BD00BF2400002000100240074BC0EB18
:10313800C00030B403EB8000054C056963692B437C
:1031480063610176427630BC704700BF24000020DE
:10315800001002402DE9F04F554C54F8204083B040
:10316800002C60D0656D1F469046524B6A682265F8
:10317800A160236004F15A014FF4807304F5AD7225
:103188006161A261E36023610646287E29F0EAFBBB
:10319800E86858B1FFF796FF721CD2B20C21FFF70E
:1031A800C5FF236DEA6822632433E364A86890B1FD
:1031B800FFF788FF721C8146D2B20B21FFF7B6FFDA
:1031C8002346EA7E3C494846FFF78CFF236DAA68F0
:1031D80062632833A36494F8590008F069F88146BB
:1031E80094F8580008F064F83A07824695F819B040
:1031F8001DD5B9F1000F1AD017F0110F4FF00B03BE
:1032080006F1010614BF4E213E2189F8063089F8DF
:1032180007605A46484608F00FF9FB0743D5236B69
:103228006BB3636B5BB3204603B0BDE8F08F17F058
:10323800010F0CBF2E274E2718F0020F0DD0B9F141
:10324800000F0AD00B22731C89F8062089F8073072
:1032580048465A46394608F0EFF818F0010FDED014
:10326800BAF1000FDBD001360C238AF807605A4602
:1032780039468AF80630504608F0DEF8CFE72B7F4B
:10328800AA7E8DF804209B090021012201A88DF84F
:1032980005308DF806108DF8072029F0F3FC20463C
:1032A80003B0BDE8F08F484608F054FCB7E700BF0C
:1032B800BC4C0020D81903082D0600080348D0F894
:1032C8003C3113B100F59A7018477047240000206C
:1032D8000348D0F8203113B100F58C7018477047B7
:1032E800240000200348D0F804310BB1FC30184703
:1032F800704700BF240000200348D0F8E8300BB125
:10330800E0301847704700BF240000200348D0F879
:10331800CC300BB1C4301847704700BF24000020E0
:103328000348D0F8B0300BB1A8301847704700BF39
:10333800240000200348D0F894300BB18C30184793
:10334800704700BF240000200248836F0BB1703023
:1033580018477047240000200248C36D0BB1543051
:1033680018477047240000200248036C0BB138301E
:1033780018477047240000200248436A0BB11C30EC
:1033880018477047240000200248836803B1184793
:10339800704700BF240000201749184B184A1948E5
:1033A80010B4D1F8884044F47004C1F888401C680F
:1033B80044F001041C605C6822405A601A6822F0DC
:1033C800847222F480321A601A6822F480221A6009
:1033D8005A6822F4FE025A60DA6A22F00F02DA62B0
:1033E8001A6B002410404FF0006218639C608A60DA
:1033F8005DF8044B704700BF00ED00E0001002408C
:103408000CC07FF8CCFC00FF2DE9F04F05462DEDF0
:10341800048BB0F9080008815FFA80F897B040463D
:103428000C4691460BF002F940B101231A461846A2
:10343800628117B0BDEC048BBDE8F08FA8F10A03D8
:10344800E72B00F2EA80DFE813F03106E800E80035
:10345800E800E800E800E800E800E800E800E80024
:10346800E800E800E800E800E800E800E800E80014
:10347800E800E800E800E800E8004306E800E800A3
:10348800E8007306E800E800E8002F05E8003305C7
:10349800E800A305E800BC05E800C805E800CD057C
:1034A800E800F305E800E800E8009A01A101E80057
:1034B800A901E800E800B701E800E800E800E80032
:1034C800E8008D01E800E800E800E800BF01E80036
:1034D800DA01E800FB012102E800E800E800E80062
:1034E800E800E800E8005902E8009C02E800C6028B
:1034F800E800E604E800B104E800E800E800E800B5
:10350800C1043B046E0477049F04E800E8005203FA
:103518006A03E8007503AE03E800E800E800E80085
:10352800CA03E800E800D503E800E800E800110451
:103538002204F4020403E800E800E8004203E8007B
:10354800E800E800E800E800E800E800E800E80033
:10355800E800E800E800E800E800E800E800E80023
:10356800E800C104E800E800E800E800E800E80036
:10357800E800E800E800E800E800E800E800E80003
:10358800E800E800E800E800E800E800E800E800F3
:10359800E800E800E800E800E800E800E800E800E3
:1035A800E800E800E800E800E800E800E800E800D3
:1035B800E800E800E800E800E800E800E800E800C3
:1035C800E800E800E800E800E800E800E800E800B3
:1035D800E800E800E800E800E800E800E800E800A3
:1035E800E800E800E800E800E800E800E800E80093
:1035F800E800E800E800E800E800E800E800E80083
:10360800E800E800E800E800E800E800E800E80072
:10361800E800E800E80084060606B8F1740F38D020
:10362800B8F1770F0DD12B686A689A421EBF5A1CF1
:103638002A601978A14A08BF002120460BF046FBF2
:10364800F3E6B8F1F50F32D0B8F1390F2A6800F077
:10365800FC8500F28E85B8F1210F01F0D385B8F111
:10366800290F40F0EB86531C2B6013780A2B01F0CE
:103678007D86502B40F0FB852846FDF713FC904EC5
:1036880030802846FDF70EFC4FF0FF3370801A4655
:10369800CDE62B686A689A421EBF5A1C2A601978C0
:1036A800884A08BF002120460BF010FBBDE62B68B6
:1036B8006A689A4241F02A86834BFF221A724FF0B9
:1036C8000008824D14F020FA41463022804885F8DF
:1036D80000802EF0A2F88DF818809DF818300B2B7A
:1036E80001F2A4867B4F7A4E42469DF8183003EBD0
:1036F800430307EBC3035B7CE3B19DF8183003EB8E
:10370800430307EBC3035B69A3B19DF8183003EBD0
:10371800430307EBC3032021586946F8220008F049
:103728005DF82B7856F8230008F01AFA2A78013247
:10373800D2B22A709DF818300133DBB28DF81830F8
:103748009DF818300B2BD0D92368591C21601A70AA
:10375800B9F1000F3FF469AE5F4BC9F8003001239F
:103768001A4664E6236800255A1C2260294620462A
:103778001D70FDF7BBFB29462046FDF7B7FB00216E
:103788002046FDF7B3FB01231A4650E621680120C5
:103798000A18226003460246087048E622684F4B22
:1037A800501C997820601170216858784A1C0123B0
:1037B80022601A4608703AE6082249492046FDF771
:1037C8007DFB01231A4632E62368464D591C2A78A8
:1037D80021601A7023686A78591C21601A706988F8
:1037E8002046FDF79BFB23682A79591C21601A7033
:1037F800E9882046FDF792FB2168287AD6E73A4EF9
:103808003378002B3FF411AE384D0027A8462368C3
:1038180015F81720591C21601A7098F8011001EB4F
:10382800810101EB810101F2EE2189B22046FDF709
:1038380075FB337801379F4208F10208E7DBF4E5AE
:1038480023682B4D01269A1922601E701BF050FF29
:10385800002841F04A85274B2268511C21601070CE
:10386800226841F2B410511C185C216041F27811B1
:10387800107059582046890AFDF738FBE96B204635
:103888004908FDF733FB01231A46D0E521681A4A97
:103898000123481C20600B7021689078CD182560A2
:1038A800087021681078CD18256008702168507854
:1038B800CA1822601A460870B9E500BF9DE40008DE
:1038C800B84400204DE500085C220020333C00206D
:1038D800882D0020C8520020F9C60108047900206C
:1038E800F05A00203C730020742C00206C2E00201D
:1038F800E096002054820020414D002022F0B8F9C3
:10390800FF28064601F0FA8416A9002501F84A5D49
:103918000DF10D008DF80D5022F0ACF816A800F846
:10392800495D22F09BF816A800F8485D22F08AF855
:1039380016A820F8405D22F079F823685A1C226006
:103948001E7023689DF80D20591C21601A70236889
:103958009DF80E20591C21601A7023689DF80F20CD
:10396800591C21601A7023689DF81020591C216089
:103978001A70BDF818102046FDF7D0FA01231A4630
:1039880055E5AD4EF378002B01F05D8423680822DD
:10399800591C21601A7023680122991821601A7035
:1039A8002368A64D591C2A7921601A702368AA78C1
:1039B800591C21601A7029882046FDF7AFFA698AD8
:1039C8002046FDF7ABFA2368F279591C21601A707A
:1039D8002168E878EAE6984D23686A79984E591C78
:1039E80021601A7033682046198CFDF797FA3368FE
:1039F8002046598CFDF792FA69892046FDF78EFA20
:103A0800A9892046FDF78AFA33682046998CFDF784
:103A180085FA33682046D98CFDF780FAE989204673
:103A2800FDF77CFA298A2046FDF778FA01231A4621
:103A3800FDE42368804A83491078834A5D1C256029
:103A4800187023688978581C20601970216890784C
:103A5800ACE6DFF814E20027FEB2714600232268C4
:103A6800501C206016702268501C20601370226859
:103A780011F8010F0133551C062B25601070EED18B
:103A88000137062F0EF1060EE6D170490023226891
:103A9800501C206017702268501C20601370226828
:103AA80011F8010F0133551C0B2B25601070EED156
:103AB8002368674A581C0721206019702368002171
:103AC800581C20601970216892F8F0006EE65B4D72
:103AD8002046A98AFDF722FAE98A2046FDF71EFA50
:103AE800298B2046FDF71AFA01231A469FE4594DFF
:103AF80020462988FDF712FA69882046FDF70EFA54
:103B0800B5F904305449DA1781FB0313C2EBA30358
:103B180099B22046FDF702FA01231A4687E40021EC
:103B28002046FDF7E3F900212046FDF7F7F90123C8
:103B38001A467CE4494D23682A68591C127821608A
:103B48001A702B6822689978531C2360002311701F
:103B58002A6821681A4401335279481C032B2060D3
:103B68000A70F5D123682A68591C127A21601A70E4
:103B780023682A68591CD27821601A7023682A6839
:103B8800591C127921601A702B6820465989FDF753
:103B9800C5F923682A68591C527A21601A702B6863
:103BA8002168587802E6264E00232268306803EB25
:103BB8004301551C405C25601070326820680A4437
:103BC800451C527825600270326820680A44013327
:103BD8009278411C0A2B21600270E6D125E4204925
:103BE80052232268501C2060137011F8013F002BEB
:103BF800F7D11AE41B4D05F16006A9882046FDF7A8
:103C08008DF9E9882046FDF789F929892046FDF7CD
:103C180085F92368AA7A591C21601A702368EA7A00
:103C2800591C21601A7055F80C1B2046FDF75EF9E7
:103C3800B542E2D1FFF7F9BB80640020F0550020BF
:103C4800C8340020E0780020F878002043430020A2
:103C580060420020983D002067666666E09A002072
:103C6800001A0308A03D00201F430020B04D204645
:103C78002988FDF753F969882046FDF74FF9A98887
:103C88002046FDF74BF901231A46FFF7D0BB2268FF
:103C9800A84BA7491878551C2560107022685878D9
:103CA800551C2560107022689B78501C206013708A
:103CB800C9882046FDF732F901231A46FFF7B7BB3A
:103CC8009D4E338AB3F5007F06F1340594BF012772
:103CD8000427403655F8041B91FBF7F1204689B2BA
:103CE800FDF71CF9AE42F5D1944D954F05F10C0640
:103CF800B5EC010AD7ED087A80EE270A2BF080FC94
:103D080081B22046FDF70AF9B542F1D18D4D05F192
:103D18000C0655F8041B204689B2FDF7FFF8AE42A1
:103D2800F7D1FFF782BB102287492046FDF7C6F876
:103D380001231A46FFF77BBB844D854EDFF844828A
:103D4800DFF84492DFED838ADFED839A9FED839A53
:103D580005F1200708E020460435FDF7DFF8AF42FB
:103D680006F118063FF461AB717C0029F3D095ED9C
:103D7800008AB0EE480A2BF043FC98F80030002B7C
:103D880041F06E8281B2E6E7754E3378002B3FF43E
:103D98004CAB744F002537F8021F2046FDF7BEF8DC
:103DA800337801359D42F6DBFFF73FBB23686E4A47
:103DB8006E49D0786E4A5D1C2560187023680978B2
:103DC800581C206019702168D078EFE40DF11809AB
:103DD80000250695DFF8B4A1664B04950595C9F84A
:103DE800045001214FF6FF7B05E001350B2D00F053
:103DF80082821AF9011F4E1CF7D04BFA05F2D00740
:103E0800F3D51A882A41D207EFD548460193FDF722
:103E1800A9FA019BE9E700212046FDF77FF8002178
:103E28002046FDF77BF800212046FDF777F8226849
:103E3800514D0023511C2160137022682968501CC1
:103E480091F82F102060117022682968501C91F891
:103E58003A102060117022682968501C91F83B10B4
:103E6800206011702268511C216013702268511C57
:103E7800216013702268511C216013702B68204642
:103E8800D98FFDF74BF82B682046998FFDF746F838
:103E980023682A68591C92F8312021601A702B680F
:103EA800216893F8320081E4344B216818787DE466
:103EB800334D23682A7A591C21601A70A98B204631
:103EC800FDF72CF8298B2046FDF728F8698B20464A
:103ED800FDF724F82368EA7C591C21601A70E98CE4
:103EE8002046FDF71BF8298D2046FDF717F82368B3
:103EF800AA7F591C21601A70236895F82020591C44
:103F080021601A70A98C2046FDF708F82368EA7A20
:103F1800591C21601A70E9682046FCF7E7FF2368FE
:103F28002A7C591C21601A70216895F821003DE40B
:103F380014790020D878002084780020BC6C0020F8
:103F4800946400205473002098300020A83000208A
:103F5800C8520020000040420040744400E08244FF
:103F6800742C0020425E0020E0780020F0780020C9
:103F7800F87800206C5E0020C8340020343300201C
:103F8800F05A002018560020E8790020301A03085B
:103F9800B94D05F14006B5F880102046FCF7BEFF84
:103FA800236895F88220591C21601A70236895F8B7
:103FB80083200435591CAE4221601A70EBD1FFF7FB
:103FC80034BAAE4D05F1800655F8041F2046FCF7BB
:103FD8008DFFB542F8D1FFF728BAA94B2168587D63
:103FE800FFF7E4BBA74B03F15A0522685979501C27
:103FF8002060117022681978501C206011702268A6
:104008005978501C2060117022689978501C2060E3
:1040180011702268D978501C2060117022681979B3
:104028000633501C9D4220601170DED1FFF7FDB9A8
:10403800954D964E05F1300795F902100023F2567A
:104048008A4200F03B810C33482BF8D10835BD4239
:10405800F2D1FFF7EAB98E4B03F17005226819789F
:10406800501C2060117022685978501C2060117013
:1040780022689978501C206011702268D978501CE9
:104088002060117022681979501C20601170226814
:104098005979501C20601170226899790733501C97
:1040A8009D4220601170D9D1FFF7BFB979482AF035
:1040B8009DFA00287FF7B9A9764B1D18226813F8D6
:1040C800011B501C9D4220601170F7D1FFF7ADB95C
:1040D800714D724F05F1500600212878704A0B4641
:1040E80006E00133242B02F10C023FD012F80C1C1D
:1040F8008842F6D103EB4303226807EB8303511C84
:1041080093F844302160137023686A78591C216041
:104118001A702368AA78591C21601A702368EA78F3
:104128000435591CB54221601A70D5D1FFF77DB905
:104138005C4D20462988FCF7F1FEA9882046FCF74B
:10414800EDFE29892046FCF7E9FE01231A46FFF710
:104158006EB9554D2046A989FCF7E0FE69892046CD
:10416800FCF7DCFE01231A46FFF761B900231B7A2E
:10417800FFDEB8F1550F01F02280B8F1570F40F07B
:104188005D81531C2B6012F8377B0DF11701013349
:104198002B6013F8010C01F8010F9A42F7D1DFF8F0
:1041A800149199F80050002DFDD1DFF80CA10126DB
:1041B800082089F8006028F00FFFDAF8000007F0FF
:1041C800C9FC3A4B28461E7028F0B6FE284628F04F
:1041D800B3FE092028F0B0FE384628F0ADFE06AF41
:1041E8003D460DF14E08EE1BF6B20A2028F0A4FE5B
:1041F800304628F0A1FE15F8016B0B2028F09CFE34
:10420800304628F099FE002007F044F8A845EAD186
:10421800082028F091FEA02028F08EFEA02028F08B
:104228008BFE002028F088FE10F02005F6D1DAF881
:10423800000007F095FC022028F0CEFE4FF0FF3377
:1042480089F800501A46FFF7F2B8531C2B60137810
:104258000A2B0CD1931C2B60154B51781970D11C6B
:10426800296091785970111D2960D2789A704FF0A1
:10427800FF331A46FFF7DBB8604200205C4200209B
:10428800F05A0020C82A00204C640020845A0020DC
:10429800943E00200436002038330020001A03081A
:1042A800481A0308DC4C0020E0780020765E0020E5
:1042B800BF3400206F5E00203864002023685A1C39
:1042C8002260197029882046FCF728FE2368EA78BE
:1042D800591C21601A7023682A79591C21601A70A8
:1042E8002368AA79591C21601A7023686A79591CB5
:1042F80021601A70AAE6DFF840B100254FF0080ADD
:104308000135242D1AD0C5F120020AFA02F22BFA3F
:1043180005F6A5F1200316432AFA03F31E4306F017
:10432800010200231343EBD0E8B229F01BFE00285A
:10433800E6D029464846FDF715F8E1E7384B1B78E3
:10434800DF0701F10D800025364E2F4602E00135CA
:10435800242D0DD029463046FDF714F80028F6D054
:1043680029464846FDF70EF8002854D10137EEE7F4
:104378002D4B2E4DB3F850102046FCF7CFFD0021F1
:104388002046FCF7CBFD2A4B1A68530103F02001A5
:10439800C2F340030B43C2F3800143EA4103C2F373
:1043A800C00143EA8103C2F3401143EAC10102F0AC
:1043B800100211432046FCF7B1FD04A9042220464F
:1043C800FCF77CFD236829781A4A581C206019706C
:1043D80011886429A8BF64212046FCF79FFDB8F125
:1043E800960F00F0C98700212046FCF797FD216849
:1043F800B7F1190348BFA7F11203A3F3C4034A1C7A
:10440800226020461A460B7005A9FCF757FD0123C8
:104418001A46FFF70CB8394604A8FCF7A3FFA5E72E
:10442800173C00205C220020A40800200036002051
:104438003C4E0020B229002090E33FF46F68A8F1B9
:104448000B00BF1AEF283FF612AF01A353F820F074
:10445800C1500008774200087742000877420008F8
:104468007742000877420008774200087742000840
:104478007742000877420008774200087742000830
:104488007742000877420008774200087742000820
:104498007742000877420008774200087742000810
:1044A8007742000877420008774200087742000800
:1044B8000F51000877420008F550000877420008BD
:1044C800A5510008774200087742000877420008A3
:1044D8009D4C0008774200082D4E000877420008DE
:1044E800BF4D000877420008994D00087742000840
:1044F800874D000877420008334D000877420008CE
:10450800E54C000877420008774200087742000827
:10451800774200083334000877420008C94C000885
:104528007742000877420008AF4C0008774200083D
:10453800774200087742000877420008774200086F
:10454800774200087742000877420008774200085F
:10455800774200081150000877420008C74F00084A
:104568007742000877420008994F00087742000810
:10457800774200087742000877420008774200082F
:104588007742000877420008CD4E000877420008BD
:104598005150000877420008554C0008774200083F
:1045A800F74B000877420008CF4B00087742000815
:1045B80077420008774200087742000877420008EF
:1045C80077420008774200087742000877420008DF
:1045D80077420008774200087742000877420008CF
:1045E80077420008774200087742000877420008BF
:1045F80077420008774200087742000877420008AF
:10460800774200087742000877420008774200089E
:10461800774200087742000877420008774200088E
:10462800774200087742000877420008774200087E
:10463800774200087742000877420008774200086E
:10464800774200087742000877420008774200085E
:10465800774200087742000877420008774200084E
:10466800774200087742000877420008774200083E
:10467800774200087742000877420008774200082E
:10468800774200087742000877420008774200081E
:10469800774200087742000877420008774200080E
:1046A80077420008774200087742000877420008FE
:1046B80077420008774200087742000877420008EE
:1046C80077420008774200087742000877420008DE
:1046D80077420008774200087742000877420008CE
:1046E80077420008774200087742000877420008BE
:1046F80077420008774200087742000877420008AE
:10470800774200087742000877420008774200089D
:10471800774200087742000877420008774200088D
:10472800774200087742000877420008774200087D
:10473800774200087742000877420008774200086D
:1047480077420008754B0008774200083D4B000887
:1047580077420008794A00085F4A0008434A00087F
:1047680077420008294A000877420008014A0008F1
:1047780077420008A34900087742000875490008F5
:104788007742000877420008534900082549000885
:1047980011490008E9480008C9480008A748000866
:1047A80077420008774200087742000877420008FD
:1047B80077420008774200087742000877420008ED
:1047C80077420008774200087742000877420008DD
:1047D80077420008774200087742000877420008CD
:1047E8008D480008774200087742000833480008DF
:1047F80077420008774200087742000877420008AD
:1048080077420008774200087742000819480008F4
:10481800B84B1B78DB073FF52AAD0AF0FBFA0AF024
:1048280095FB01231A46FEF702BE531C2B60137832
:104838000F2B3FF61CAD911C2960C3EBC303AE4997
:104848005078C854D01C28600B4491785970111DB9
:104858002960D1789970511D29601179D970911DFD
:10486800296051791971D11D29609179597102F125
:1048780008012960D2799A7118F052FE01231A466C
:10488800FEF7D5BD2846FCF70DFB9C4EB0812846A7
:10489800FCF708FB012370811A46FEF7C8BD2846BD
:1048A800FCF700FB964EB0822846FCF7FBFAF08234
:1048B8002846FCF7F7FA012330831A46FEF7B7BDFE
:1048C8001346511C296013F8020B2B60D31C517836
:1048D8002B6092781AF08EFA00287EF4A6ADC6E412
:1048E8001346511C2960874913F8020B08702B6086
:1048F800824953788B70D31C2B60834B92789A70C3
:1049080001231A46FEF793BD804B814918684A2255
:104918002AF06CFC01231A46FEF789BD1146531C88
:104928002B607C4B11F8020B187029605178597074
:10493800D11C296092789A702846FCF7B3FA764A17
:104948000123D0801A46FEF772BD2846FCF7AAFA62
:10495800714E30802846FCF7A5FA70802846FCF78F
:10496800A1FA0123B0801A46FEF761BDDFF8B881CD
:1049780098F80030002B3EF458AD684F00262846C2
:10498800FCF790FA23F074F898F80030A7EC010AC5
:1049980001369E42F3DBFEF748BD0F2F7FF467AC6C
:1049A800531C2B601678072E3FF661ACDFF87C812C
:1049B80028460C27FCF776FA07FB06F708EB0706EC
:1049C800B0802846FCF76EFAF0802846FCF76AFAB1
:1049D8002B6830811A46591C296012F8021BB172E3
:1049E8002A605B78F3722846FCF744FA012348F8FA
:1049F80007001A46FEF71BBD531C2B6010780606ED
:104A080000F1B8853B4B1B78DD073EF50EAD03285A
:104A180028BF00200AF0E2F901231A46FEF707BD75
:104A2800344B1B78D8073EF500AD0AF067FC0AF056
:104A38008DFA01231A46FEF7FABC2E4B1B78DA07CB
:104A48003EF5F3AC36490A78012342F004020A70B5
:104A58001A46FEF7ECBC274B1B78D9073EF5E5ACA8
:104A6800304A4FF4C871012311801A46FEF7DFBCA3
:104A7800092F7FF6FCABDFF8B8801346511CD8F835
:104A88000060296013F8021B31702B605378B370F3
:104A9800D31C2B609378642B02F10401A8BF642314
:104AA80073712960D378642B02F10501A8BF6423D0
:104AB800B37129601379F371931D2B605379642BBB
:104AC80028BF6423D11D337229609379F37002F1F2
:104AD80008032B60D37933712846FCF7E3F90A2FD2
:104AE800708140F0528529F0B5FA01231A46FEF785
:104AF8009EBC00BF173C0020943E0020E0780020B8
:104B0800F055002080640020F8780020C834002088
:104B180034290308D8780020147900201C79002053
:104B280070300020FC9A002071400020A03D002039
:104B3800E09A0020AC4B1868D31C014621329E1E17
:104B48002E6013F8036C0E705E1E2E6013F8026C54
:104B58004E702B6013F8016C8E700333934201F191
:104B68000301ECD118F0B6FEFEF75FBCC7F34707A8
:104B7800122F3FF67CABB7B116AB0DF1160803EB5D
:104B88004706C146423E2846FCF78CF929F8020F31
:104B98004E45F8D1954B38F8022F23F8022FC1451E
:104BA800F9D1112F09D8924A7B00023B1344002106
:104BB800223223F8021F9A42FBD18E490122134662
:104BC8000A70FEF734BC1346511C29608A4913F851
:104BD800020BC8702B60894953780B70D31C2B606B
:104BE800874B9278DA7001231A46FEF720BC2846D4
:104BF800FCF758F92846FCF755F92846FCF752F90E
:104C08002B68794E9A1CD6F800802A605A7888F862
:104C18002F20DA1C2A609A7888F83A201A1D2A6010
:104C2800DA7888F83B2007332B602846FCF73AF9F6
:104C3800A8F83E002846D6F80080FCF733F9112F73
:104C4800A8F83C0000F27F8430688BE7531C2B6087
:104C5800654EDFF8CC811378D6F8009088F80530D7
:104C68002846FCF71FF9A9F820002846D6F8009036
:104C7800FCF718F9052FA9F8220000F20F840AF0B2
:104C8800D3F821F053FF306822F02AFD01231A4699
:104C9800FEF7CDBB531C2B605A4B12781A700123B8
:104CA8001A46FEF7C4BB584B02F1080101322A60CC
:104CB80012F8010C03F8010F9142F7D1FEF7B5BBCA
:104CC8001346511C2960514913F8020B88702B6058
:104CD80053784B7001231A46FEF7A9BB0723B7FB8D
:104CE800F3F3C3EBC301791A7FF4C1AADBB203F172
:104CF800FF385FFA88F8002B3EF497ABDFF8109185
:104D080008F101088A46531C2B6092F90010404BA9
:104D1800002693F902208A4200F055830136062EB8
:104D280003F10803F5D1FFF7A2BA531C2B601378DF
:104D38000E2B3FF69CAA911C29605678032E3FF64D
:104D480096AA3448062101FB03F14318D71C5E716B
:104D58002F6096784654111D2960D1785970511DDD
:104D6800296011799970911D29605179D970D11DE7
:104D7800296092791A7101231A46FEF758BB531C11
:104D88002B60254B12785A7501231A46FEF74FBB44
:104D9800531C2B6016781F2E3FF669AA052F7FF447
:104DA80066AA2846FCF766F81C4B43F8260020F054
:104DB800B3FDFEF73ABB194E06F140072846FCF74B
:104DC80071F82B68A6F88000591C1A46296012F859
:104DD800021B86F882102A605B7886F883300436D6
:104DE800BE42EBD1FEF721BBC8340020822C002044
:104DF800842C0020A82C0020E0780020F0780020E7
:104E0800F878002034330020EF5A0020047900207D
:104E18004C640020C82A0020F05A0020604200207C
:104E280080640020531CBE4E2B60137833722846D2
:104E3800FCF738F8B0832846FCF734F83083284666
:104E4800FCF730F82B6870835A1C2A601B78F374BF
:104E5800082F7EF6EAAA2846FCF724F8F0842846AC
:104E6800FCF720F80C2F30857EF6DFAA2B681A464F
:104E7800591C296012F8021BB1772A605B7886F802
:104E880020302846FCF70EF8102FB0847EF6CDAA05
:104E98002B685A1C2A601B78F3722846FBF7EAFF36
:104EA8002B68F0605A1C2A601A783274162F7EF626
:104EB800BCAA9A1C2A605B7886F8213001231A461E
:104EC800FEF7B5BA2846FBF7EDFF064620F0D0FE00
:104ED800FF283EF4AAAAB6F57A7F80F0AA820DF1DF
:104EE8005809002309F8403DF708494604A88DF8F9
:104EF8001030013720F0BEFD9DF81030FFB206F0EB
:104F08000706BB4206F1010603D19DF81830B342EB
:104F180003D03146384620F097FE2B686A68D21ACB
:104F2800012A7EF782AA5A1C16A82A6000221E7837
:104F380000F8482D20F092FD9DF81030B3420AD0B9
:104F4800784B1B683BB19A79B24204D31B681B6942
:104F58000BB1304698472B685A1C2A6048460022F5
:104F68001D788DF8182020F06DFD9DF81830AB42A3
:104F78003EF45BAA6B4B1B68002B3EF456AA1B68D9
:104F88005B69002B3EF451AA28469847FEF74DBAB4
:104F9800654B1B78012B3EF648AA1146531C2B6023
:104FA800624B11F8020B9870296051781970D11C66
:104FB800296092785A7001231A46FEF738BA531CB2
:104FC8002B601778112F3FF652A9931C2B60584E6F
:104FD800537806F817302846FBF764FF40F6CA03F3
:104FE8009842A8BF184640F2EE23984206EB4706BF
:104FF800B8BF18460123A0F2EE211A46192091FBEA
:10500800F0F17170FEF713BA1346511C2960494E2E
:1050180013F8021B31702B60537873702846FBF726
:1050280041FF2B6870805A1C2A601B783371284610
:10503800FBF738FF2B68F0805A1C2A601B78337204
:1050480001231A46FEF7F3B91346511C29603A4E5C
:1050580013F8021BB1702B60384953780B70D31CBE
:105068002B60374F93783B71131D2B60D378092B36
:10507800A8BF09232846BB70FBF714FF2B686A6892
:105088003880D11A012905DD2846FBF70BFF2B686C
:105098006A6878829A4240F0658209F0C5FE2B68FA
:1050A8006A689A423EF4C1A95A1C2A601B78FB70B0
:1050B80001231A46FEF7BBB9224B102F4FF000020E
:1050C80028BF10271A605A609A60DA601A74002F95
:1050D8003EF4ABA92A68174401322A6012F8011C71
:1050E80003F8011B9742F7D1FEF79FB9164E00232C
:1050F80033602846FBF7BEFE326801230243326064
:105108001A46FEF794B9531C2B60107813283FF603
:10511800AEA8931C2B6056780C4B00211EE000BFF4
:10512800F05A0020BC620020404D0020414D002074
:105138006C2E00203C73002080640020D47800206E
:10514800F055002004360020843600203C1A03085D
:105158000131242903F10C033FF489A81F7AB742CF
:10516800F6D1BF4EBF4B0C2707FB0161D61C91F847
:105178003C1003F820102E6003EB800391785970DF
:10518800111D2960D0789870501D2860B649127991
:105198000868DA7028F0ECFEFEF747B92846FBF7F6
:1051A80081FEB24E30602846FBF77CFE70602846D0
:1051B800FBF778FE0123B0601A46FEF738B9531C96
:1051C8002B601678FF2E00F09081FE2E00F0E08014
:1051D8002846FBF767FE95E80C009B1A002B06DDB6
:1051E800531C2B60137813B90B2E40F2A081242E88
:1051F8003FF63DA89E4A4FF0FF3322F816001A46A4
:10520800FEF715B91346511C29609A4E13F8021B74
:1052180071702B6053783370D31C2B609378B37004
:105228002846FBF73FFE2B68F0801A46591C296078
:1052380012F8021B31712A605B7873714FF0FF33EB
:105248001A46FEF7F4B82368B1788B4A581C2060D8
:10525800197023681278591C21601A70FEF7A0BBD8
:10526800D9F8003013F48053B4EEE88A00F0A38034
:10527800F1EE10FAC0F2D180B4EEC98AF1EE10FA5C
:105288000DD8DFED7E7A9FED7E7A77EEC87AB4EEA0
:10529800C78AF1EE10FAB0EE678A00F2BE80F7EE28
:1052A800007A78EE677AB6EE007AF0EE696AE7EE91
:1052B800876A40F2E932FDEEE67A17EE901AB1F508
:1052C800FA6FA8BF4FF4FA619142B8BF114689B28C
:1052D800002B3EF440ADB5EE408AF1EE10FA40F2F4
:1052E800DC5308BF1946FEF736BD95F82420654BF8
:1052F800002A40F089803046FEF7AEBA21680123C3
:10530800CA1822601A460870FEF791B85A1C194646
:105318002A605D4811F8022B027229605B7843729B
:10532800042A06D9FF2A3EF4CAA921680020FEF7FC
:105338003DBA56490978994203D8022AF5D1FF2B7C
:10534800F3D122680123D11821601370B9F1000F3D
:105358003EF46BA84E4AC9F800201A46FEF767B813
:10536800069B43F001030693FEF7EDBF2846FBF7C3
:1053780099FD484EFEF784B923680322591C216021
:105388001A7023686A78591C21601A70FFF72FB8C1
:10539800931C2B605678022E3EF669AF2846FBF721
:1053A80081FD334A02EB46024FF0FF33A2F85E005C
:1053B8001A46FEF73CB8F1EE10FABFF670AF4FF49C
:1053C8007A71FEF7C8BC09EBC6072846B970FBF727
:1053D80069FD2B6829F836001A46591C296012F80D
:1053E800021BF9702A605A783A71DA1C2A609A7896
:1053F800BA711A1D2A600AF1010ADB787B71D0455F
:105408007FF481ACFEF711B85978022908D0032936
:105418000CBF04203046FEF71FBA4FF47A715AE7E2
:10542800042A34BF02200320FEF716BA4246FEF7CC
:105438008BB90DF11809484620F0F8FABDF8183074
:10544800B3423FF46AAD144B1B68002B3FF465ADC3
:105458001B689B69002B3FF460AD304698475CE5BC
:10546800001A030838330020C8340020DC4C002020
:1054780004340020D05B0020D478002000C0884489
:1054880000C08244548200205C2200207140002029
:1054980075E50008D0780020BC6200202846FBF79C
:1054A80001FDA8F80A002846FBF7FCFCA8F80C0048
:1054B8002846D6F80090FBF7F5FCA9F82400284602
:1054C800D6F80090FBF7EEFC0D2FA9F826007FF622
:1054D800D6AB2846FBF7E6FCA8F80E002846FBF7F3
:1054E800E1FCA8F81000FFF7CABB931C2B602F4BF8
:1054F80051781970D31C2B602D4E937886F85C3048
:10550800131D2B60D37886F856302846FBF7CAFC63
:10551800A6F858002846FBF7C5FC2846FBF7C2FC4E
:105528004FF0FF33A6F85A001A46FDF780BF204B0C
:1055380000301E4418BF01204FF0FF3386F84A00A0
:105548001A46FDF774BF2B683168581C1A46286044
:1055580012F8020B81F831002A605B7881F832304A
:10556800FFF772BB5A1C2A601B78003318BF01234F
:10557800F37192E500F07F00032828BF002012F0A5
:1055880003FB01231A46FDF752BF2B68D8F8002009
:10559800591C2960197851720B2F3FF4A4AA991C41
:1055A80029605B785370FFF79EBA00BF4064002003
:1055B800043400202DE9F04FDFF80CB12DED0C8BF1
:1055C8009BF800309BB0012B079002F0EF84394C18
:1055D80094F80021002A41F04E83072B364D02F043
:1055E8000D84002303936B683348984700286ED0D6
:1055F800B5F8A880002285F84920B8F1000F40F0DE
:105608009682B5F926002A6BB5F92460E96AB5F9DE
:105618002830821A686BEA63711A284EA9631B1A2C
:1056280095F84A1026482B6414F076F9336813F07D
:10563800005302F05F84D5ED0F5AD5ED0E7A214A5A
:1056480094ED636AD4ED646A94ED657AD4F8983180
:105658001268B8EEE58AD5ED105AF8EEE77AF8EE5A
:10566800E58A013377EE867A38EE268A78EE878ADD
:105678009342C4ED637A84ED648AC4ED658AC4F804
:10568800983101F077869BF80080B8F1140F03F089
:1056980039840023D4F8A0110493062902F21E8548
:1056A800DFE811F0CD1AB01BBC14C61B301ABC19A8
:1056B800361900BF6822002094640020E879002091
:1056C800CC640020404E002081400020049C9BF8C0
:1056D8000090B9F1070F00F0E48294F8B031002B84
:1056E80040F0EA82D44B5B79002B40F01B82012307
:1056F8009BF8002084F8B031072A02F0DC850023EB
:105708000B93CE4BD4ED6E9A93ED007ACC4ADFF82A
:10571800ACA31268CB4BDFF8A8830492F7EE007AAB
:1057280037EEE98AC84A089328EE078A0592B4EE4C
:10573800E78AC64A039300255346F1EE10FAD4EDE2
:105748006D8ADFF88093DFEDC2AA9FEDC29A9FEDC4
:10575800C2BADFEDC2CA9FEDC2AADFEDC2BAC24F1C
:105768000692C24688BFB0EE678A2E469846BF4B5F
:105778002B44D3ED007ABE4BF5EE407A2B44F1EE84
:1057880010FA93ED00CA17D0BA4B2B4493ED007A68
:105798007CEE476AB0EEE66AF4EEC67AF1EE10FAED
:1057A80008D5F5EEC06AF1EE10FACCBF37EE87CA1D
:1057B80037EE67CA83ED00CA059BB3F800E01EF018
:1057C800030F00F08182022E04F006870499AA4B89
:1057D80091F8322007EE102A91F831202B44D3EDAE
:1057E800006A5342B8EEC77A07EE903A27EE267A57
:1057F800F8EEE77AB4EEE77AF1EE10FA0AD407EE9B
:10580800902AF8EE677AF4EEC77AF1EE10FA88BFBC
:10581800F0EE477A994B0993994A03EB460332F91C
:105828001610B3F90A30C81A07EE100AB8EEC77A8C
:105838001EF0010FE7EE497A00F09682DFF888E261
:105848009EED00CA27EE8CCA94F8C8E1BEF1000F9D
:105858001FD0DFF874E2D4F8CC019EED007ADFF8AF
:105868006CE25B1A07EE903A079BDEF8001027EE11
:10587800097AF8EEE77A1B1A8B4227EE87CA01F3FA
:10588800BF81F7EE007AF4EEE79AF1EE10FA01F133
:1058980082817C4B2B44D3ED007A039BD3ED01DA54
:1058A80068EEA77A3CEE6DDA67EE8D7AC8ED007A7D
:1058B800069BD9ED006A93ED007A734BD7ED007A19
:1058C80026EE877A2B4467EE086A93ED007A26EE77
:1058D800877AF0EE676AE7EE0D6AB0EE667A94EDC5
:1058E8006E6AF7EE006AB4EEE66AF1EE10FAACBF43
:1058F8000123002343B1F0EEE77AF0EEC76AF4EE35
:10590800E76AF1EE10FA01D587ED007A022E04F06D
:1059180009865E4A5E4B52F826001B68B0EE6D0A97
:1059280098475C4A5C4B52F826001B689847049BD2
:1059380093F83A30632B04D8059B1B88002B01F0A1
:105948007F81F0EE6C7A554B99ED007A37EEC00AFC
:105958002B44D3ED007A83ED000A049B30EE670AEE
:1059680093F8482080EE07CADAB1F7EE007AF4EE31
:10597800E79AF1EE10FA14DB494BD3ED007AB0EE5A
:10598800CC7AB4EEE77AF1EE10FA0ADD454BD3EDA6
:10599800007AB0EECDDAB4EEE7DAF1EE10FA01F300
:1059A8006A82414B94F8D8212B44D3ED007A68EEF3
:1059B800A77A27EE8CCA8AED00CA2AB9C8ED00CAB0
:1059C800C7ED00CACAED00CA039B043504330C2D89
:1059D80006F101060AF1040A08F1040807F10407B0
:1059E80003937FF4C4AE9BF80030072B02F0898341
:1059F800012B02F06584002303932C4A104B116895
:105A08001B6893F82F0011F48053049300F0588218
:105A1800274D284E2B78DFF8B8E0F6889EED037AFC
:105A280013F0010F244B1A8B08BFA4F8E021A2EB56
:105A3800060E07EE90EA4DE0806400205C3F0020EF
:105A4800C8340020B86C00206C5E002018000020CC
:105A580000009642CDCCCC3DAE47813F000000000F
:105A68000000C842610BB63B80300020503F002048
:105A78006C23002024240020D4230020E078002078
:105A8800983D00200C3F0020183F0020886D002022
:105A9800846D0020EC6D0020E86D00203824002083
:105AA800703F00206C3F0020243F0020E879002050
:105AB800173C002014790020F05A00207430002090
:105AC8008C300020083F0020383F0020603F002035
:105AD80050410020F8EEE77AB4EEE77AF1EE10FADA
:105AE80042F25A83971906EE907AF8EEE66AB4EE17
:105AF800E67AF1EE10FA81F20384B4F8E0219645D3
:105B080083F23386DA4ADB4E92ED005AD6ED003A3C
:105B1800D94AC4ED793A84ED7A5AD2ED006ADFEDBC
:105B2800D77AE6E1D64B1B78013BDBB2E0E5D54BF3
:105B3800D549089391F801A01B68D44F9BF80090B1
:105B4800B7F906004FF47A71B1FBF3F3C3EB4316D0
:105B580003EB8603DE00B6B2B04503F05982E96F65
:105B6800B5F924E02B6E4A1C07EE90EA7344012A2B
:105B7800EA672B66F8EEE77A03F05482D5ED1B5AF4
:105B8800D5ED1D6A07EE102A37EEE56AB8EEC75A5A
:105B9800B8F1010F86EE057A37EE257A77EEC77AE7
:105BA80085ED1C7AE6EE276A85ED1B7AF0EE667ABB
:105BB800C5ED1E6AC5ED1D6A03F04686D5F890103E
:105BC800B5F926E06B6E4A1C07EE90EA7344012A89
:105BD800C5F890206B66F8EEE77A03F03C82D5EDC5
:105BE800205AD5ED226A07EE102A37EEE56AB8EE9C
:105BF800C75AB8F1010F86EE057A37EE257A77EEA7
:105C0800C77A85ED217AE6EE276A85ED207AF0EEEF
:105C1800667AC5ED236AC5ED226A03F06986D5F870
:105C2800A410B5F928E0AB6E4A1C07EE90EA73445D
:105C3800012AC5F8A420AB66F8EEE77A03F02582BE
:105C4800D5ED255AD5ED276A07EE102A37EEE56A15
:105C5800B8EEC75AB8F1010F86EE057A37EE257A05
:105C680077EEC77A85ED267AE6EE276A85ED257AFE
:105C7800F0EE667AC5ED286AC5ED276A03F0D88587
:105C8800F880B5F8A8309BF80090013BA5F8A8303B
:105C980008990023B9F1070F4B608B60CB607FF444
:105CA8001CAD05F09FF8039B784FC01A94F8B031EB
:105CB8003880002B3FF416AD013B84F8B0311BB09F
:105CC800BDEC0C8BBDE8F08F94F8C83163B1022E9F
:105CD80004F064846E4B09936E4A03EB460332F971
:105CE8001610B3F90A30B4E56B4B2B4493ED000A58
:105CF800039BD3ED01DA28EE800A3CEE6DDA022E22
:105D080020EE0D0A88ED000A7FF4D2AD634A644B99
:105D180010681B689847069BD9ED006A93ED007AD6
:105D2800604BD7ED007A1A785F4B83ED020A5F4B20
:105D380026EE877A2B4427EE087A93ED006A27EE41
:105D4800067AF0EE676AE7EE0D6A012AB0EE667A27
:105D580002D0192A7FF4C3ADB4EEEADAF1EE10FAF4
:105D6800CCBF01230023C5E5B2F900C0D4ED5E6ABB
:105D780094ED5F7AB2F902000A908CEAEC70B4EE06
:105D8800E67AA0EBEC70F1EE10FA0C900A984BBF93
:105D9800B7EE007AF7EE006A77EE665A76EEC75AE3
:105DA8000028B8BF40420D900C9886460D9886454D
:105DB80041F31F80BCF1000FD6BFCCF1000007EE05
:105DC80010CA07EE100ADFF8E8E0B8EEC77A9EF8C6
:105DD80000E027EE097ABEF1000F01F01C80DFF821
:105DE800D4E09EED005AB5EEC05AF1EE10FA42F337
:105DF800EF80DFF8C4E0DEED004AF5EEC04AF1EED0
:105E080010FA42F3E58034EEC77AB7EE006AC7EEBF
:105E1800246A75EEC65AF4EEC66A65EE8A5AF1EE41
:105E280010FA85EE857A88BFF0EE466AF5EEC06A0C
:105E3800F1EE10FA37EE067AB8BFF0EE6C6A66EE4D
:105E4800876AF4EEC66AF1EE10FA88BFF0EE466A89
:105E5800F5EEC06AF1EE10FAB8BFF0EE6C6ADFF842
:105E68005CE09EED007A67EE877AA7EEA6CAEBE4BF
:105E7800287300208078002038730020000000007C
:105E8800D4780020B86C0020806400208440002072
:105E9800E0780020983D00200C3F00204C72002044
:105EA80060720020943D002074300020183F0020CC
:105EB800443F0020403F0020483F00203C3F002056
:105EC800E14BE24A5D8B92ED037AE14A07EE905A84
:105ED800E04DD2ED003AE04A95ED005AD2ED006A65
:105EE800DE4D84ED7A5AF8EEE77AC4ED793A77EE2A
:105EF800677A87EEA66ADA4EDA4AD6ED005ADA4EA3
:105F0800DFEDDA6A96ED003AD94EDFEDDA4A96ED22
:105F1800004A92ED007AF7EE007AB4EEE76A75EE81
:105F2800835AF1EE10FA88BFB0EE676A75EE845AAC
:105F3800B4EEE66AF1EE10FA65EEA45AB8BFB0EE18
:105F4800666AF1EE476A73EEC52AF4EEE65AF1EE98
:105F580010FA84ED7B6AC4ED7D2A00F1A384F4EE87
:105F6800C75AF1EE10FA88BFF0EE475ABC4ADFED87
:105F7800C14AD2ED017ABC4A92ED013ABC4A77EEA9
:105F8800837A92ED014A77EE847A67EEA47AF4EE8A
:105F9800E76AF1EE10FA08DCB4EEE77AF1EE10FAEF
:105FA8008CBFF0EE676AF0EE476AAD4A9FEDB14AE2
:105FB800D2ED027AAC4AD2ED024AAF4A77EEA47A21
:105FC80092ED007A67EE847AF1EE474AF4EEE47ACD
:105FD800F1EE10FA08D4F4EEC77AF1EE10FA8CBF9D
:105FE800F0EE474AF0EE674A002841F04F82F7EE9C
:105FF800007AA24AA24E527894F8F801002ABFEE1D
:10600800003AB7EE007A327814BFB0EE472AB0EE05
:10601800432A002814BFB0EE434AB0EE474A002A8C
:1060280003F0ED80F4EEC77AF1EE10FA64EE824ADE
:10603800944841F36D8290ED027A90ED011AD0ED0B
:10604800031A9FED8A2A26EE877A27EE843AA5EE70
:10605800817AA1EEA47A27EE037AB4EEC27AF1EE41
:1060680010FAB4BFF0EE427AF0EE477A8DED0E7A70
:1060780088BFB0EE427A012A00F0BF8190ED064A4F
:10608800D0ED051A90ED072A26EE844AA5EEA14A1E
:10609800A4EE824A24EE034AB4EEC74AF1EE10FA9F
:1060A800B4EEE74A8CBFB0EE472AB0EE442AF1EED0
:1060B80010FA98BFB0EE427AA8BFF0EE447A022AEE
:1060C8008DED0F4A00F0998190ED0A4AD0ED091A3A
:1060D80090ED0B2A26EE844AA5EEA14AA2EE244AA8
:1060E80024EE034AB4EEC47AF1EE10FAF4EEC47A60
:1060F8008CBFB0EE442AB0EE472AF1EE10FA58BF32
:10610800B0EE427AB8BFF0EE447A032A8DED104A19
:1061180000F0738190ED0E4AD0ED0D1A90ED0F2A24
:1061280026EE844AA1EEA54AA4EE824A24EE034A4A
:10613800B4EEC47AF1EE10FAF4EEC47A8CBFB0EE85
:10614800442AB0EE472AF1EE10FA58BFB0EE427A70
:10615800B8BFF0EE447A042A8DED114A00F04D8163
:1061680090ED124AD0ED111A90ED132A26EE844ACA
:10617800A1EEA54AA2EE244A24EE034AB4EEC47A5C
:10618800F1EE10FAF4EEC47A8CBFB0EE442AB0EE09
:10619800472AF1EE10FA58BFB0EE427AB8BFF0EED7
:1061A800447A052A8DED124A00F0278190ED164AAF
:1061B800D0ED151A90ED172A26EE844AA5EEA14ACD
:1061C800A2EE244A24EE034AB4EEC74AF1EE10FACE
:1061D800F4EEC47A8CBFB0EE472AB0EE442AF1EE52
:1061E80010FA58BFB0EE427AB8BFF0EE447A062AE9
:1061F8008DED134A00F0018190ED1A4AD0ED191A7D
:1062080090ED1B2A26EE844AA5EEA14AA4EE824A06
:1062180024EE034AB4EEC47AF1EE10FAF4EEC47A2E
:106228008CBFB0EE442AB0EE472AF1EE10FA58BF00
:10623800B0EE427AB8BFF0EE447A072A8DED144AE0
:1062480000F0DB8020E000BFF05A00205041002021
:10625800807800207C78002030730020173C0020D4
:1062680074300020743F00208030002000000000BF
:106278008C3000206F12833A783F0020343300209E
:10628800714000206872002090ED1E4AD0ED1D1A62
:1062980090ED1F2A26EE844AA5EEA14AA4EE824A72
:1062A80024EE034AB4EEC47AF1EE10FAF4EEC47A9E
:1062B8008CBFB0EE442AB0EE472AF1EE10FA58BF70
:1062C800B0EE427AB8BFF0EE447A082A8DED154A4E
:1062D80000F0938090ED224AD0ED211A90ED232A08
:1062E80026EE844AA5EEA14AA4EE824A24EE034A89
:1062F800B4EEC47AF1EE10FAF4EEC47A8CBFB0EEC4
:10630800442AB0EE472AF1EE10FA58BFB0EE427AAE
:10631800B8BFF0EE447A092A8DED164A6DD090ED9B
:10632800264AD0ED251A90ED272A26EE844AA5EEB6
:10633800A14AA4EE824A24EE034AB4EEC47AF1EEEE
:1063480010FAF4EEC47A8CBFB0EE442AB0EE472AB5
:10635800F1EE10FA58BFB0EE427AB8BFF0EE447AC8
:106368000A2A8DED174A48D090ED2A4AD0ED291A0D
:1063780090ED2B2A26EE844AA5EEA14AA4EE824A85
:1063880024EE034AB4EEC47AF1EE10FAF4EEC47ABD
:106398008CBFB0EE442AB0EE472AF1EE10FA8DED2C
:1063A800184A58BFB0EE427AA8BFB0EE674A0B2A27
:1063B80003F0F581D0ED2E7AD0ED2D1A90ED2F2A2D
:1063C80066EEA77AE1EEA57AE2EE247A67EE837AA2
:1063D800F4EEC77AF1EE10FAF4EEC47A8CBFF0EE60
:1063E800476AF0EE676AF1EE10FACDED197A98BFB8
:1063F800B0EE667AB8BFF0EE447A77EEC77AF7EE79
:10640800006AF4EEE67AF1EE10FAC4ED6E7A43F320
:10641800938186EEA77A012ADDED0E7A67EE877AF8
:10642800CDED0E7A55D0DDED0F7A67EE877A022A28
:10643800CDED0F7A4DD0DDED107A67EE877A032A1D
:10644800CDED107A45D0DDED117A67EE877A042A12
:10645800CDED117A3DD0DDED127A67EE877A052A07
:10646800CDED127A35D0DDED137A67EE877A062AFC
:10647800CDED137A2DD0DDED147A67EE877A072AF1
:10648800CDED147A25D0DDED157A67EE877A082AE6
:10649800CDED157A1DD0DDED167A67EE877A092ADB
:1064A800CDED167A15D0DDED177A67EE877A0A2AD0
:1064B800CDED177A0DD0DDED187A67EE877A0B2AC5
:1064C800CDED187A05D0DDED197A27EE877A8DEDB6
:1064D800197AE248006810F0805000F08584B6EE22
:1064E800006A84ED7B6A002A02F0A4862D78DFF822
:1064F8008493DFF88483DFF884A3DFF884E394F8D7
:10650800F0C15B8B0593FDEEE37AD9ED005A9AF85A
:1065180003A0B8F906909EF800E005F0010301F029
:10652800100817EE905A01F48001BCF1000F40F0FA
:10653800BD81B8F1000F40F06B85C948DDED0E7ADA
:1065480090ED007AC749E7EE067ABAF1000F42F0FB
:10655800E586BDEEC57A17EE107AB0EE457AA2EE62
:10656800A77AFDEEC77A17EE90CA17EE90EAAC4507
:10657800A8BFAE466745C8BFBE4607EE90EAF8EE2C
:10658800E77A012AC1ED007A00F04A8190ED047A99
:10659800DDED0F7AE7EE067AB0EE457AA2EEA77A3D
:1065A800FDEEC77A17EE90CA17EE90EAAC45A8BF81
:1065B800AE46BC45B8BFBE4607EE90EAF8EEE77AAD
:1065C800022AC1ED017A00F02B8190ED087ADDED09
:1065D800107AE7EE067AB0EE457AA2EEA77AFDEEDB
:1065E800C77A17EE90CA17EE90EAAC45A8BFAE4638
:1065F800BC45B8BFBE4607EE90EAF8EEE77A032A34
:10660800C1ED027A00F00C8190ED0C7ADDED117A83
:10661800E7EE067AB0EE457AA2EEA77AFDEEC77AE3
:1066280017EE90CA17EE90EAAC45A8BFAE46BC4537
:10663800B8BFBE4607EE90EAF8EEE77A042AC1ED45
:10664800037A00F0ED8090ED107ADDED127AE7EE36
:10665800067AB0EE457AA2EEA77AFDEEC77A17EE73
:1066680090CA17EE90EAAC45A8BFAE46BC45B8BF85
:10667800BE4607EE90EAF8EEE77A052AC1ED047AFD
:1066880000F0CE8090ED147ADDED137AE7EE067A0D
:10669800B0EE457AA2EEA77AFDEEC77A17EE90CA59
:1066A80017EE90EAAC45A8BFAE46BC45B8BFBE469B
:1066B80007EE90EAF8EEE77A062AC1ED057A00F0CF
:1066C800AF8090ED187ADDED147AE7EE067AB0EE39
:1066D800457AA2EEA77AFDEEC77A17EE90CA17EEB2
:1066E80090EAAC45A8BFAE46BC45B8BFBE4607EE6B
:1066F80090EAF8EEE77A072AC1ED067A00F0908072
:1067080090ED1C7ADDED157AE7EE067AB0EE457A63
:10671800A2EEA77AFDEEC77A17EE90CA17EE90EAB6
:10672800AC45A8BFAE46BC45B8BFBE4607EE90EA2A
:10673800F8EEE77A082AC1ED077A71D090ED207A51
:10674800DDED167AE7EE067AB0EE457AA2EEA77A84
:10675800FDEEC77A17EE90CA17EE90EAAC45A8BFCF
:10676800AE46BC45B8BFBE4607EE90EAF8EEE77AFB
:10677800092AC1ED087A53D090ED247ADDED177A15
:10678800E7EE067AB0EE457AA2EEA77AFDEEC77A72
:1067980017EE90CA17EE90EAAC45A8BFAE46BC45C6
:1067A800B8BFBE4607EE90EAF8EEE77A0A2AC1EDCE
:1067B800097A35D090ED287ADDED187AE7EE067A79
:1067C800B0EE457AA2EEA77AFDEEC77A17EE90CA28
:1067D80017EE90EAAC45A8BFAE46BC45B8BFBE466A
:1067E80007EE90EAF8EEE77A0B2AC1ED0A7A17D09D
:1067F80090ED2C7ADDED197AE7EE067AA2EEA75A2B
:10680800FDEEC57A17EE900A8542A8BF0546874275
:10681800D8BF2F4607EE907AF8EEE77AC1ED0B7AEB
:10682800002B00F0DD83104B1B68002B40F0E58344
:106838000E4B1B784BB3307868B10A4FDFF84480B1
:106848000025E8B2D8F80030B7EC010A984730784C
:1068580001358542F5DB064B1B6815E068300020E2
:1068680068720020A8300020043F0020805A0020D1
:106878001456002064720020445E0020DC5B002077
:10688800185600200C56002098479BF80030072B1C
:1068980001F0BC83012384F800311BB0BDEC0C8BE4
:1068A800BDE8F08FF0EE665AFFF760BBB8F1000F55
:1068B80040F03C83DB48DDED0E7A90ED007ADA4952
:1068C800E7EE067AF1EE626AB0EE637AA6EEA77A90
:1068D800F0EE477ABEF1000F41F02E85BAF1000FB5
:1068E80043F06680BDEEC57AFDEEE77A17EE107AC2
:1068F80017EE90CA17EE90EAAC45A8BFAE466745BA
:10690800C8BFBE4607EE90EAF8EEE77A012AC1ED65
:10691800007A85D090ED047ADDED0F7AE7EE067AFD
:10692800B0EE637AA6EEA77AFDEEC77A17EE90CAA4
:1069380017EE90EAAC45A8BFAE46BC45B8BFBE4608
:1069480007EE90EAF8EEE77A022AC1ED017A3FF401
:1069580067AF90ED087ADDED107AE7EE067AB0EED3
:10696800637AA6EEA77AFDEEC77A17EE90CA17EEFD
:1069780090EAAC45A8BFAE46BC45B8BFBE4607EED8
:1069880090EAF8EEE77A032AC1ED027A3FF448AFBD
:1069980090ED0C7ADDED117AE7EE067AB0EE637AC7
:1069A800A6EEA77AFDEEC77A17EE90CA17EE90EA20
:1069B800AC45A8BFAE46BC45B8BFBE4607EE90EA98
:1069C800F8EEE77A042AC1ED037A3FF429AF90ED97
:1069D800107ADDED127AE7EE067AB0EE637AA6EE6B
:1069E800A77AFDEEC77A17EE90CA17EE90EAAC4583
:1069F800A8BFAE46BC45B8BFBE4607EE90EAF8EE63
:106A0800E77A052AC1ED047A3FF40AAF90ED147ACB
:106A1800DDED137AE7EE067AB0EE637AA6EEA77A92
:106A2800FDEEC77A17EE90CA17EE90EAAC45A8BFFC
:106A3800AE46BC45B8BFBE4607EE90EAF8EEE77A28
:106A4800062AC1ED057A3FF4EBAE90ED187ADDED3C
:106A5800147AE7EE067AB0EE637AA6EEA77AFDEE30
:106A6800C77A17EE90CA17EE90EAAC45A8BFAE46B3
:106A7800BC45B8BFBE4607EE90EAF8EEE77A072AAB
:106A8800C1ED067A3FF4CCAE90ED1C7ADDED157AB7
:106A9800E7EE067AB0EE637AA6EEA77AFDEEC77A3D
:106AA80017EE90CA17EE90EAAC45A8BFAE46BC45B3
:106AB800B8BFBE4607EE90EAF8EEE77A082AC1EDBD
:106AC800077A3FF4ADAE90ED207ADDED167AE7EE69
:106AD800067AB0EE637AA6EEA77AFDEEC77A17EECD
:106AE80090CA17EE90EAAC45A8BFAE46BC45B8BF01
:106AF800BE4607EE90EAF8EEE77A092AC1ED087A71
:106B08003FF48EAE90ED247ADDED177AE7EE067A43
:106B1800B0EE637AA6EEA77AFDEEC77A17EE90CAB2
:106B280017EE90EAAC45A8BFAE46BC45B8BFBE4616
:106B380007EE90EAF8EEE77A0A2AC1ED097A3FF4FF
:106B48006FAE90ED287ADDED187AE7EE067AB0EEB2
:106B5800637AA6EEA77AFDEEC77A17EE90CA17EE0B
:106B680090EAAC45A8BFAE46BC45B8BFBE4607EEE6
:106B780090EAF8EEE77A0B2AC1ED0A7A3FF450AEB4
:106B880090ED2C7ADDED197AE7EE067AE6EEA73A73
:106B9800FDEEE37A36E6099BB2F900E0B3F90A3074
:106BA8002249AEEB0300096880EAE073A3EBE073C7
:106BB8008B42BEF66EAEB2F90230099AB2F90C20D9
:106BC8009A1A82EAE273A3EBE27399427EF761AE06
:106BD8000899174BD1ED017A93ED007AF0EEE77A38
:106BE800F4EEC77AF1EE10FA7EF553AED1ED027AE3
:106BF800F0EEE77AB4EEE77AF1EE10FA7EF749AEF6
:106C08000C4B1A88002384F8C831002A40F09C8372
:106C1800094A0A4B1178186881F0010104F0A6FFAF
:106C2800FEF737BE68720020A8300020643F0020BD
:106C3800683F0020D8990020DA990020DC990020CC
:106C4800A64BA74A2B44D3ED006A92ED007AA54BD8
:106C580026EE877AF7EE006AB4EEE67AD3ED007A8C
:106C6800F1EE10FA88BFB0EE667A27EE277A67EE63
:106C78000C7AFEF768BE072B02F02F8400230393DB
:106C8800994E9A4D3368590501F1A482984B1B78A7
:106C9800002B40F00681974B94F8127127B1964A61
:106CA8001288920742F0DA8294F81881DA7FB8F1F4
:106CB800000F41F0A5829E7F002E00F0EB85022E8A
:106CC80002F09682032E01F012868C49498802321E
:106CD800D2B2B8F1000F02F03682002902F03382F6
:106CE80087480668B1FBF6F10EB2A4F84861002A9D
:106CF80003F09B8107EE906AF8EEE77AF7EE006AF8
:106D080086EEA77A7F49012AD4ED576AD1ED007A39
:106D180077EEE67A67EE877AC4ED537A21D0D1ED23
:106D2800017AD4ED586A77EEE67A022A67EE877A16
:106D3800C4ED547A15D0D1ED027AD4ED596A77EEC4
:106D4800E67A032A67EE877AC4ED557A09D0D1ED41
:106D5800037AD4ED5A6A77EEE67A67EE877AC4ED5D
:106D6800567A9BF80000092803F02B82002E40F386
:106D7800988592B3D4ED577A94ED537A77EE877A63
:106D8800012AC4ED577AC1ED007A21D0D4ED587AA2
:106D980094ED547A77EE877A022AC4ED587AC1EDD9
:106DA800017A15D0D4ED597A94ED557A77EE877A31
:106DB800032AC4ED597AC1ED027A09D0D4ED5A7A82
:106DC80094ED567A77EE877AC4ED5A7AC1ED037A54
:106DD800013A022AB8BF0222D2B2B8F1000F0CBFA2
:106DE8001046022000F05EBD4F023FF578ABFFF77A
:106DF8007ABB0A98DFF828E10028D8BF404207EE9E
:106E0800100A9EF800E0B8EEC77A27EE097ABEF1BC
:106E1800000F7EF4E4AFDFF80CE19EED006AB4EEFB
:106E2800CB6AF1EE10FA41F1CF81B7EE005A35EE98
:106E3800465ADFED356ADFF8F0E036EEC77A25EE20
:106E48002B5ADEED006AA5EE076A26EE267AB5EE25
:106E5800C07AF1EE10FA41F2BB80CAEE076AB7EECB
:106E6800006A35EEC67AF0EE465AE7EE265AF0EE9C
:106E7800656AFEF7E6BF01230799C4F8CC11022A18
:106E880084F8C8317EF48DAD204A1288002A43F078
:106E9800D2801F4A1F4B1178186804F067FEFEF76E
:106EA80080BD1D4A134BB2F906105A8B91423FF729
:106EB800F3AE1A4A1278012A02F03081192A02F038
:106EC8002D810E2A3FF4E8AE082A3FF4E5AE0D49BD
:106ED80000228A60C4F80C21DEE600BFE02300200F
:106EE800343F0020303F0020E879002094640020DF
:106EF8002C200020F05A00206C5E0020742C00200A
:106F08001C3300205041002000003443D899002051
:106F1800DA990020DC990020445E002034330020F8
:106F2800443F00204C3F0020403F0020002B42F00F
:106F38007E82BEF1000F41F07184FDEEC57A0DF13D
:106F4800380C17EE90EAFDEEE57A0CEB8203049319
:106F58002B48DFF8B49006944FFA8AF317EE907A2C
:106F6800F1EE626A8AF0010805921C46034693ED29
:106F7800007AFCEC017AE7EE067A1030B0EE637A1C
:106F8800A6EEA77AFDEEC77A17EE903A17EE902A8A
:106F9800AB42A8BF2A469F42CCBF00210AF001019C
:106FA800002914BF114639469E45CCBF002308F07E
:106FB800010307EE901A002B14BF13467346B8EE70
:106FC800E77A07EE903A049BF8EEE77A002C18BFB0
:106FD800F0EE477A9C45E9EC017AC7D1059A069C00
:106FE800002A3FF420AC92000649074828F0FEF832
:106FF800064B1B68002B3FF41BAC15F0B9FE17E4D9
:10700800687200201C790020A8300020043F00206E
:10701800002B42F0BE81BAF1000F42F0D283CF4874
:10702800DDED0E7A90ED007ACD49E7EE067ABDEEF9
:10703800C57A17EE103AB0EE457AA2EEA77AFDEEC1
:10704800C77A17EE90EA17EE907AAE45A8BF2F469A
:107058007345C8BF1F4607EE907AF8EEE77A012A13
:10706800C1ED007ABFD090ED047ADDED0F7AE7EE3E
:10707800067AB0EE457AA2EEA77AFDEEC77A17EE49
:1070880090EA17EE907AAE45A8BF2F469E45B8BF46
:107098001F4607EE907AF8EEE77A022AC1ED017AE8
:1070A800A1D090ED087ADDED107AE7EE067AB0EE21
:1070B800457AA2EEA77AFDEEC77A17EE90EA17EEA8
:1070C800907AAE45A8BF2F469E45B8BF1F4607EE2B
:1070D800907AF8EEE77A032AC1ED027A83D090ED30
:1070E8000C7ADDED117AE7EE067AB0EE457AA2EE7B
:1070F800A77AFDEEC77A17EE90EA17EE907AAE45BA
:10710800A8BF2F469E45B8BF1F4607EE907AF8EEF7
:10711800E77A042AC1ED037A3FF465AF90ED107A5F
:10712800DDED127AE7EE067AB0EE457AA2EEA77A9E
:10713800FDEEC77A17EE90EA17EE907AAE45A8BF33
:107148002F469E45B8BF1F4607EE907AF8EEE77ABD
:10715800052AC1ED047A3FF446AF90ED147ADDEDCF
:10716800137AE7EE067AB0EE457AA2EEA77AFDEE3C
:10717800C77A17EE90EA17EE907AAE45A8BF2F4669
:107188009E45B8BF1F4607EE907AF8EEE77A062AC2
:10719800C1ED057A3FF427AF90ED187ADDED147A4A
:1071A800E7EE067AB0EE457AA2EEA77AFDEEC77A48
:1071B80017EE90EA17EE907AAE45A8BF2F469E4587
:1071C800B8BF1F4607EE907AF8EEE77A072AC1EDB6
:1071D800067A3FF408AF90ED1C7ADDED157AE7EEFC
:1071E800067AB0EE457AA2EEA77AFDEEC77A17EED8
:1071F80090EA17EE907AAE45A8BF2F469E45B8BFD5
:107208001F4607EE907AF8EEE77A082AC1ED077A6A
:107218003FF4E9AE90ED207ADDED167AE7EE067AD6
:10722800B0EE457AA2EEA77AFDEEC77A17EE90EA9D
:1072380017EE907AAE45A8BF2F469E45B8BF1F46A9
:1072480007EE907AF8EEE77A092AC1ED087A3FF45A
:10725800CAAE90ED247ADDED177AE7EE067AB0EE45
:10726800457AA2EEA77AFDEEC77A17EE90EA17EEF6
:10727800907AAE45A8BF2F469E45B8BF1F4607EE79
:10728800907AF8EEE77A0A2AC1ED097A3FF4ABAEB4
:1072980090ED287ADDED187AE7EE067AB0EE457AB9
:1072A800A2EEA77AFDEEC77A17EE90EA17EE907A6B
:1072B800AE45A8BF2F469E45B8BF1F4607EE907A39
:1072C800F8EEE77A0B2AC1ED0A7A3FF48CAE90ED1E
:1072D8002C7ADDED197AE7EE067AA2EEA75AFDEED2
:1072E800C57A17EE900A8542A8BF05468342D8BFE3
:1072F8002B4607EE903AF8EEE77AC1ED0B7A6FE687
:1073080007EE902AF8EEE77ADFF85CE0DFF85CC079
:107318009EED005ADCED003ADFF854E0C4ED793A0E
:1073280077EE677A06EE906ABCEEC77AF8EEE66A00
:1073380017EE102A77EEE67A84ED7A5AA4F8E0215F
:10734800DEED006AFEF7D5BD06494A69002A3EF41B
:10735800A0AA0A6813604B74FEF79BBA68720020F3
:10736800A8300020E09900202873002080780020B1
:107378003873002007EE103A9BF800305C4FC4F8D1
:107388009881B8EEC77AF7EE006A132B86EE879AD3
:10739800B7F90400B4F89C8195ED080A01F0C2859C
:1073A800544B554A93ED001A93ED093A93ED162A7A
:1073B80093ED1F6AD3ED0B1A93ED144AD3ED015ADE
:1073C800D3ED0A3A93ED0C7A93ED155AD3ED172ABB
:1073D800D3ED206AD3ED044AD3ED030A69EE277A88
:1073E80069EE288A29EE088AA7EE813A02EB880E10
:1073F8000021A2EE286AC4F88C11C4F89011A8EEF6
:10740800214AE7EEA53AA8EE075A93ED1A7AD3ED8A
:107418000F5A93ED021AD3ED0E1A8EED003AE2EEF2
:10742800A86A64EEC34A27EE467A93ED0D2AD3ED97
:10743800192A8EED204AE3EE603A65EEC45A93EDC0
:10744800183AC3ED093AE7EE814AF0EE477AA4EE1E
:10745800615AE8EE025AE2EEC66AE3EE287AC3ED14
:107468000A4A83ED145AC3ED155A8EED406AC3EDEE
:107478001F6AC3ED207AC4F8941108F1010303F0E0
:107488001F03A4F89C31B880FEF7FDB81B4A107999
:1074980000283EF4ACAD1A48007800283EF4A7ADA9
:1074A80012789FED182A07EE102A174A07EE900A5D
:1074B8001288F8EEE77A04EE102AB8EE477AB8EEAA
:1074C800444A27EE277AB7EE003AC7EE047AF4EE7C
:1074D800C27AF1EE10FA88BFF0EE427AF4EEC37A7F
:1074E800F1EE10FAB8BFF0EE437AFEF782BD00BFA6
:1074F8008440002000510020644E0020D05B002012
:107508004F410020713DAA3F1841002000000000B3
:1075180090ED027A90ED012AD0ED037A1FED053A3D
:1075280026EE877AA2EE257AA7EEA47A27EE047AC9
:10753800B4EEC37AF1EE10FAB4BFF0EE437AF0EE8F
:10754800477A8DED0E7A88BFB0EE437A012A3EF471
:1075580054AF90ED063AD0ED051A90ED072A26EEC5
:10756800833AA1EEA53AA2EE243A23EE043AB4EE09
:10757800C73AF1EE10FAB4EEE73A8CBFB0EE472AFC
:10758800B0EE432AF1EE10FA98BFB0EE427AA8BFE7
:10759800F0EE437A022A8DED0F3A3EF42EAF90EDCD
:1075A8000A3AD0ED091A90ED0B2A26EE833AA1EE9D
:1075B800A53AA2EE243A23EE043AB4EEC73AF1EE25
:1075C80010FAB4EEE73A8CBFB0EE472AB0EE432A81
:1075D800F1EE10FA98BFB0EE427AA8BFF0EE437A07
:1075E800032A8DED103A3EF408AF90ED0E3AD0ED37
:1075F8000D1A90ED0F2A26EE833AA1EEA53AA2EED7
:10760800243A23EE043AB4EEC73AF1EE10FAB4EE97
:10761800E73A8CBFB0EE472AB0EE432AF1EE10FAF3
:1076280098BFB0EE427AA8BFF0EE437A042A8DEDF7
:10763800113A3EF4E2AE90ED123AD0ED111A90ED07
:10764800132A26EE833AA1EEA53AA2EE243A23EEB7
:10765800043AB4EEC73AF1EE10FAB4EEE73A8CBF4A
:10766800B0EE472AB0EE432AF1EE10FA98BFB0EE1A
:10767800427AA8BFF0EE437A052A8DED123A3EF41D
:10768800BCAE90ED163AD0ED151A90ED172A26EEFD
:10769800833AA1EEA53AA4EE823A23EE043AB4EE78
:1076A800C37AF1EE10FAF4EEC37A8CBFB0EE432A37
:1076B800B0EE472AF1EE10FA58BFB0EE427AB8BFE2
:1076C800F0EE437A062A8DED133A3EF496AE90ED2D
:1076D8001A3AD0ED191A90ED1B2A26EE833AA5EE38
:1076E800A13AA4EE823A23EE043AB4EEC73AF1EE98
:1076F80010FAB4EEE73A8CBFB0EE472AB0EE432A50
:10770800F1EE10FA98BFB0EE427AA8BFF0EE437AD5
:10771800072A8DED143A3EF470AE90ED1E3AD0ED86
:107728001D1A90ED1F2A26EE833AA5EEA13AA4EE83
:10773800823A23EE043AB4EEC73AF1EE10FAB4EE08
:10774800E73A8CBFB0EE472AB0EE432AF1EE10FAC2
:1077580098BFB0EE427AA8BFF0EE437A082A8DEDC2
:10776800153A3EF44AAE90ED223AD0ED211A90ED4A
:10777800232A26EE833AA5EEA13AA2EE243A23EE76
:10778800043AB4EEC37AF1EE10FAF4EEC37A8CBF81
:10779800B0EE432AB0EE472AF1EE10FA58BFB0EE29
:1077A800427AB8BFF0EE437A092A8DED163A3EF4D4
:1077B80024AE90ED263AD0ED251A90ED272A26EE34
:1077C800833AA1EEA53AA2EE243A23EE043AB4EEA7
:1077D800C73AF1EE10FAF4EEC37A8CBFB0EE472A3E
:1077E800B0EE432AF1EE10FAA8BFB0EE427AB8BF65
:1077F800F0EE437A0A2A8DED173A3EF4FEAD90ED8D
:107808002A2AD0ED291A90ED2B3A26EE822AA1EEEB
:10781800A52AA3EE242A22EE042AB4EEC72AF1EE02
:1078280010FAF4EEC27A8CBFB0EE473AB0EE423AA4
:10783800F1EE10FA8DED182AA8BFB0EE437AA8BF72
:10784800B0EE672A0B2A02F0CE83D0ED2E7AD0ED67
:107858002D1A90ED2F3A66EEA77AE5EEA17AE4EEBE
:10786800837A67EE847AB4EEE77AF1EE10FAB4EE32
:10787800E72A8CBFF0EE676AF0EE476AF1EE10FA7D
:10788800CDED197A58BFB0EE667AA8BFF0EE427A0D
:10789800FEF7B3BDA4F84861B8F1000F00F0788195
:1078A800DF490220DF4ADFEDE06AD2F800E09BF80A
:1078B80000C09EF800209EF8028007EE902AF8EE9D
:1078C800E77AB0EE007A67EEA67AF4EEC77AF1EEC0
:1078D80010FA40F35D8437EEC77ADFEDD46AB0EE74
:1078E800676AA7EE266AB0EE467A9FEDD16AD1EDB7
:1078F800006A66EE866AB0EEE66AC4ED5B6A84EDFD
:107908005E6AB8F1000F13D005EE908AB8EEE55A1A
:10791800DFEDC55A66EEA64A25EE255AF7EE005A5F
:1079280075EEC55A64EE864AE5EE245A66EEA56AF7
:10793800DFEDC05A9EF8052027EE257A27EE267A35
:10794800CAB1DFEDB96ADFEDBC5A26EE266A06EE4B
:10795800902AF8EEE66A66EE866AF4EEE56AF1EEDB
:1079680010FA00F35787F7EE005A75EEE66A85EECF
:10797800A66A27EE067ABCF10C0F9FEDB08ADFED00
:10798800B06A00F0ED86B4EEC87AF1EE10FA98BF4E
:10799800B0EE478AB4EEE68AF1EE10FAB8BFB0EE60
:1079A800668A84ED418A002800F0E680B0EE007A0D
:1079B800F4EEC77AF1EE10FA05DD37EEC77ADFED9F
:1079C8009B6AE7EE267A91ED017ADFED996A27EE58
:1079D800267AB0EEC76A84ED5C7A84ED5F6AB8F106
:1079E800000F13D006EE908ADFED8F5AF8EEE66AA4
:1079F80027EE075A66EEA56AF7EE005A75EEE65AC4
:107A080025EE065AE6EE855A27EE257ADFED896AD5
:107A18009EF8062067EEA67A67EE877AAAB107EE87
:107A2800102AB8EEC77ADFED805ADFED836A27EEB9
:107A3800067A27EE257AB4EEE67AF1EE10FA40F3EC
:107A4800DB86DFED806A67EEA67ABCF10C0F00F0EA
:107A5800A286DFED7A6A9FED7A7AF4EEE67AF1EEA5
:107A680010FA88BFF0EE667AF4EEC77AF1EE10FAF3
:107A7800B8BFF0EE477A0128C4ED427A7CDD9EF863
:107A88000120DFED696A07EE902AF8EEE77AB0EE9A
:107A9800007A67EEA67A9EF80920F4EEC77AF1EE2E
:107AA80010FA05DD37EEC77ADFED606AE7EE267A71
:107AB80091ED027ADFED5E6A27EE267AB0EEC76AAC
:107AC80084ED5D7A84ED606A9AB106EE902ADFED66
:107AD800565AF8EEE66A27EE075A66EEA56AF7EEFA
:107AE800005A75EEE65A25EE065AE6EE855A27EE56
:107AF800257ADFED506A9EF8072067EEA67A67EED2
:107B0800877A0AB307EE102AB8EEC77ADFED465A2D
:107B1800DFED496A27EE067A27EE257AB4EEE67A93
:107B2800F1EE10FA0CDCB5EEC07AF1EE10FA01F1C4
:107B3800FC82B7EE006A36EE477AC6EE076A01E0C5
:107B4800DFED406A67EEA67ABCF10C0F00F04286C2
:107B5800DFED3A6A9FED3A7AF4EEE67AF1EE10FA42
:107B680088BFF0EE667AF4EEC77AF1EE10FAB8BF85
:107B7800F0EE477AC4ED437ABCF1090F00F0E785CF
:107B880093F82160002E40F09C85002384F818317A
:107B98002D4EDFF8B88096F82420DFF8B490531EF5
:107BA800082B00F20E81DFE813F02E018501A300F7
:107BB8000C01550009009B010C01870199F8003060
:107BC800002B41F0EB823368317A4FF4807203EB7B
:107BD8000121002025F046F9337A0133DBB2022B6C
:107BE800337240F06381002025F07CF9002025F0F5
:107BF80079F9FF2025F076F900F01F00052802F03A
:107C0800718317F033FBF768002F00F069830022B7
:107C1800336971680120B84796F82420BFE700BF90
:107C280050410020E09A00200AD7233CD7A368419E
:107C38006F12033B00004843A4707D3F00C0F94425
:107C480000C0F9C40000C842E0960020009A002055
:107C5800664400204FF40071306817F0B9FA012823
:107C680001F05383C1F03B83022840F01F8117F0D5
:107C780035FB17F0FBFAF768002F00F0318300227C
:107C8800104633697168B84796F8242087E71021B1
:107C9800D14817F09DFA002840F006810490012190
:107CA8007F2023F0C1F901288246049B40F0FC8024
:107CB8001846022123F0B8F9002801F05C86012853
:107CC80040F0F28016213A2023F0AEF9431C9B02C3
:107CD800F36317F003FB386803F03CFF00210A2028
:107CE80017F094FA002841F0AA82032386F824307A
:107CF80010210EA817F06CFA002840F0D7809DF8E4
:107D080042209DF841009DF844109DF845309DF8AB
:107D18004370120442EA00620A431B019DF84610B0
:107D28009DF83900DBB243EA111342EA072203F552
:107D3800FA63726333879DF83A209DF8403042EA2F
:107D4800002201F00F01180903F00F0386F83A101A
:107D580072859DF838109DF83B2086F832309DF8E2
:107D68003C3086F8281086F82C209DF83D109DF8A8
:107D78003E2086F82D309DF83F3086F8303086F862
:107D8800310086F82E1086F82F2017F0A7FAB37E58
:107D980073B9924F386803F0DDFE4FF4007110207C
:107DA80017F034FA074617F099FA002F40F093803D
:107DB8008B4825F0EBF800230422336286F8242050
:107DC8000323DBB2022B40F20F82042A00F0BA81AF
:107DD800082A00F0B781834B1B7823B9824B9B7824
:107DE800002B41F08D829BF80030072B00F0FA84BD
:107DF8000022072B84F800217DF4F3AB02F0F2FF98
:107E08000390FDF7F0BB754F386803F0A3FE00211F
:107E1800084617F0FBF9824617F060FABAF1010F2D
:107E280044D1002338687376049303F093FE40F23C
:107E3800AB11082017F0EAF90528049B01F08C849F
:107E4800012801F02A8517F049FA737E002B02F009
:107E5800FE81022386F82430386803F07BFE737EA7
:107E6800022B14BF4FF0000A4FF0804A0021372040
:107E780017F0CCF95146292017F0C8F9824617F0B7
:107E88002DFABAF1000F11D1737E022B01F059853A
:107E980086F81AA0386803F05DFE0021092017F063
:107EA800B5F900283FF4F3AE17F018FA96F8242035
:107EB800531E86E7494FCFE70827FF2025F012F821
:107EC800FF2801F0C481013FF7D17369D8F8002079
:107ED800FA339342EAD217F0C9F996F824205EE6FD
:107EE8000827FF2024F0FEFFFF2800F01D81013F36
:107EF800F7D1EAE73D4A08920027B246DFF8088141
:107F0800DFF8F890089E04943C46B8EC018AD5ED59
:107F1800087AB8EEC88A28EE278A002C02F009836E
:107F28006BBB9BF80030082B39D007F5D260B0EE58
:107F3800480A2844D5F88C36984707F5E360D5F801
:107F48001437284498479BF80030032BB0EE408A3A
:107F580020D0D5F8AC30D8F84406B0EE480A984797
:107F680006EB84030134032C07F12C0783ED010A87
:107F78003DF4ACABDAF8003003F00053C5E707F581
:107F8800F460B0EE480A2844D5F89C379847B0EE1C
:107F9800408AC6E727F034FB29F81400D9E7B0EE89
:107FA800480A27F02DFB29F81400BEE7104B114CA6
:107FB8001A68114B114F94F80001D2691B883A8056
:107FC8007B8000287EF45AAE03900D4DFDF70BBB65
:107FD800DFED0C6AFDF743BF2097002068440020BE
:107FE800003800406E5E0020414D0020B86C002033
:107FF8006044002068220020B2290020844000202C
:108008009464002000000000CC64002002F0EAFE26
:10801800039AB54B801AD880FEF73CBCDFF80C9366
:10802800D4ED017A94ED006AB9F80070D9F81430EB
:1080380077EEA77AF0EE006AB0EE677AA6EE267AB7
:10804800013F04EBC702D6EE267A083A1033F6EE63
:10805800003A27EE237A67EEA37A84ED207AC4EDFE
:10806800217AA24CA64604F1800092ED027A92EDA4
:10807800036ADEED036ADEED027A53ED014A13ED81
:10808800025A37EE674A76EEC65A77EE277AE4EE5A
:10809800845A013FA2F10802E5EE047A0EF1080EB7
:1080A80003F1080336EE267A00F10800E4EE877A39
:1080B800E5EE475A67EEA37A25EEA37AC0ED007A7B
:1080C80080ED017AD1D1B8F1140F07D102F08AFE00
:1080D800049B854FC01A7880D4F8A011844B08936C
:1080E800844A3368013182FB01025018CA17C2EB77
:1080F800A002C2EBC202891AC4F8A01103F000530F
:10810800FAE602F06FFE9BF800300B9A764F801A61
:10811800012B788000F0D580072B7DF46CAC02F041
:1081280061FE0390FDF769BC336A0022012B3276A9
:1081380042F26681F269013B013233620823F2613F
:1081480086F824306C4E17F07FFC7378022B01F010
:10815800E181032B7FF43FAE41F2B813F35C002BAF
:1081680041F04A8741F2A403F35C002B41F03F87BA
:1081780041F2E803F35C002B41F0438741F22C13F2
:10818800F35C002B3FF427AE5C481AF0EDFB22E6C7
:10819800B0EE677AFFF7A9BB594EDFF894E1594A68
:1081A80096ED005ADEED003A574E1278C4ED793A52
:1081B80084ED7A5AD6ED006A12B1012284F8F021D2
:1081C800D4ED7B7AFDF795BEDFF868E19EED007A85
:1081D800FEF73DBEAB68002B3EF458AD05F14401F7
:1081E80028469847FEF752BD484B71691B685B1AD1
:1081F800C82B7FF6EDAD17F039F896F82420E4E5A2
:1082080043494448D1F8EC10076844F6206081429D
:10821800A8BF0146B1F57A7FB8BF4FF47A7188B22A
:10822800FF06A4F81A01316841F19A82C90400F1E5
:1082380068833949D1F800C0BCF936703749384EDF
:10824800D1ED037AD4F81C11A6FB006086096420DE
:1082580090FBF6F01428BDEEE77A04EB410EA8BFB8
:10826800142001318142C4F81C1117EE109AA4BFE2
:108278000021C4F81C1104EB4101AEF82091B1F9BA
:10828800201107EE101AB8EEC77A77EEC77AFDEE1E
:10829800E77ACDED047ABDF9100080EAE071A1EB30
:1082A800E071B94201F3B2861E4908464FF07E518B
:1082B8000160FEF700BD02F095FD0B90FDF721BAB5
:1082C800094F02F08FFD184AD4F8DC311268039088
:1082D800C31A9A1AC4F8DC01BB80FA80FDF78DBB7B
:1082E80096F824205BE400BF844000206822002028
:1082F800B86C002093244992548200208093002077
:108308007C7800201856002034730020009A002042
:10831800A408002068300020C83400205041002004
:10832800D34D6210180000201C3300204C4E002052
:108338002C730020403F0020BAF1000F3EF4D2AA6F
:10834800F4EEC57AF1EE10FAB8BFF0EE657AFDEEFC
:10835800E77ABDEEE57A17EE90EA17EE90CAAE45D9
:1083680017EE107AA8BFAC467745C8BFBC4607EEE3
:1083780090CAF8EEE77A012AC1ED007A3EF450AAD5
:1083880090ED047ADDED0F7AE7EE067AB0EE637AC7
:10839800A6EEA77AB4EEC57AF1EE10FAF0EE477AB7
:1083A800B8BFF0EE657AFDEEE77A17EE90EA17EEC1
:1083B80090CAAE45A8BFAC46BE45B8BFBC4607EE9E
:1083C80090CAF8EEE77A022AC1ED017A3EF428AAAB
:1083D80090ED087ADDED107AE7EE067AB0EE637A72
:1083E800A6EEA77AB4EEC57AF1EE10FAF0EE477A67
:1083F800B8BFF0EE657AFDEEE77A17EE90EA17EE71
:1084080090CAAE45A8BFAC46BE45B8BFBC4607EE4D
:1084180090CAF8EEE77A032AC1ED027A3EF400AA80
:1084280090ED0C7ADDED117AE7EE067AB0EE637A1C
:10843800A6EEA77AB4EEC57AF1EE10FAF0EE477A16
:10844800B8BFF0EE657AFDEEE77A17EE90EA17EE20
:1084580090CAAE45A8BFAC46BE45B8BFBC4607EEFD
:1084680090CAF8EEE77A042AC1ED037A3EF4D8A957
:1084780090ED107ADDED127AE7EE067AB0EE637AC7
:10848800A6EEA77AB4EEC57AF1EE10FAF0EE477AC6
:10849800B8BFF0EE657AFDEEE77A17EE90EA17EED0
:1084A80090CAAE45A8BFAC46BE45B8BFBC4607EEAD
:1084B80090CAF8EEE77A052AC1ED047A3EF4B0A92D
:1084C80090ED147ADDED137AE7EE067AB0EE637A72
:1084D800A6EEA77AB4EEC57AF1EE10FAF0EE477A76
:1084E800B8BFF0EE657AFDEEE77A17EE90EA17EE80
:1084F80090CAAE45A8BFAC46BE45B8BFBC4607EE5D
:1085080090CAF8EEE77A062AC1ED057A3EF488A902
:1085180090ED187ADDED147AE7EE067AB0EE637A1C
:10852800A6EEA77AB4EEC57AF1EE10FAF0EE477A25
:10853800B8BFF0EE657AFDEEE77A17EE90EA17EE2F
:1085480090CAAE45A8BFAC46BE45B8BFBC4607EE0C
:1085580090CAF8EEE77A072AC1ED067A3EF460A9D8
:1085680090ED1C7ADDED157AE7EE067AB0EE637AC7
:10857800A6EEA77AB4EEC57AF1EE10FAF0EE477AD5
:10858800B8BFF0EE657AFDEEE77A17EE90EA17EEDF
:1085980090CAAE45A8BFAC46BE45B8BFBC4607EEBC
:1085A80090CAF8EEE77A082AC1ED077A3EF438A9AE
:1085B80090ED207ADDED167AE7EE067AB0EE637A72
:1085C800A6EEA77AB4EEC57AF1EE10FAF0EE477A85
:1085D800B8BFF0EE657AFDEEE77A17EE90EA17EE8F
:1085E80090CAAE45A8BFAC46BE45B8BFBC4607EE6C
:1085F80090CAF8EEE77A092AC1ED087A3EF410A984
:1086080090ED247ADDED177AE7EE067AB0EE637A1C
:10861800A6EEA77AB4EEC57AF1EE10FAF0EE477A34
:10862800B8BFF0EE657AFDEEE77A17EE90EA17EE3E
:1086380090CAAE45A8BFAC46BE45B8BFBC4607EE1B
:1086480090CAF8EEE77A0A2AC1ED097A3EF4E8A85A
:1086580090ED287ADDED187AE7EE067AB0EE637AC7
:10866800A7EEE27AB4EEC57AF1EE10FAF0EE477AA8
:10867800B8BFF0EE657AFDEEE77A17EE90EA17EEEE
:1086880090CAAE45A8BFAC46BE45B8BFBC4607EECB
:1086980090CAF8EEE77A0B2AC1ED0A7A3EF4C0A830
:1086A80090ED2C7ADDED197AE7EE067AE6EEA73A38
:1086B800B4EEE35AF1EE10FAC8BFF0EE653AFEF7F1
:1086C80067BA1E21C648F8F75DFE00283FF45DAA88
:1086D800C44B1B8858063FF558AA94F88431B34216
:1086E80041F00085C04BD4ED627A93ED010AD4EDD8
:1086F800435A9FEDBE6ADFEDBE6A27EEE57A68EE63
:10870800277AA8EE007AE5EE807AB4EEC67AF1EE22
:1087180010FA88BFB0EE467AB4EEE67AF1EE10FAB7
:10872800F4EEC67AB8BFB0EE667AF1EE10FA88BFFA
:10873800F0EE467AF4EEE67AF1EE10FAB8BFF0EE13
:10874800667A84ED417AC4ED437AFFF71EBAFDEEEE
:10875800C87AA84F17EE902ABE80FA80FFF710BAA1
:10876800B4EEC87AF1EE10FA98BFB0EE478ABDEEC3
:10877800C77AB4EEE68A9F4FF1EE10FA17EE102A88
:10878800B8BFB0EE668A84ED418A3A8000287FF44B
:108798000DA9FFF7F5B99FED957ADFED956A954F2D
:1087A800F4EEC77AF1EE10FA98BFB0EE677AFDEEF4
:1087B800E77AB4EEE67AF1EE10FA17EE902AB8BF2F
:1087C800B0EE667A012884ED427A7A803FF757A99D
:1087D800FFF7D6B9BDEEE77A864F17EE102ABA80B2
:1087E800FFF7B6B902F0FEFA039A824F9BF8003001
:1087F800801AB880FFF7FCBAB5EEC07AF1EE10FA2D
:1088080000F19784B7EE006A36EE477AC6EE076A3B
:10881800FFF719B99FED786AFFF7ABB8FDEEC57A97
:108828000EA817EE90EAFDEEE57A00EB82030493BA
:10883800DFF8E091DFF8E0C106944FFA8AF317EE0B
:10884800907AF1EE626A8AF0010805921C464B465E
:1088580093ED007AF0EC017AE7EE067A0AF001036C
:1088680009F11009B0EE637AA6EEA77AB4EEC75AFA
:10887800F1EE10FAD8BF0023002BF0EE477A18BFAC
:10888800B0EE657ABDEEC77AFDEEE77A17EE102AEC
:1088980017EE901AAA4217EE103AA8BF2B46974235
:1088A800CCBF00220AF00102002A08BF3B46A942B9
:1088B80017EE902A07EE103AA8BF2A468E45CCBF7D
:1088C800002308F00103002B08BF724607EE902A28
:1088D800B8EEC77AF8EEE77A049B002C18BFF0EEE2
:1088E800477A9842ECEC017AB1D1FEF777BB93F85E
:1088F8002010C1EB411001EB8001C90089B2FEF7DD
:10890800E6B93E49D1F800C0BCF836707F0895E456
:108918003B4BD4F8A4910893B4F89CA1CAF1200366
:10892800DFB2384B0AEB491E03EB8E0EBB0801F091
:10893800A28301331B013448344A05930EEB030C20
:108948000EF1100313ED024A13ED035A13ED016AF9
:1089580013ED047A50ED024A50ED035A50ED016AC6
:1089680050ED047A64EE244A65EE255A66EE266ACE
:1089780067EE277A1033634542ED024A42ED035A07
:1089880042ED016A42ED047A00F1100002F1100292
:10899800D8D1059B1E48A3F11002964400EB020CA7
:1089A800224417F0030309D0BEEC017AFCEC017AEB
:1089B80067EE277A013BE2EC017AF5D1BAF1000FB4
:1089C80041F0EE81B8F1140F7FF48AAB02F00AFA95
:1089D800049B084FD4F8A011C01A7880FFF780BB19
:1089E800683000206C5E00201800002000C0F944A8
:1089F80000C0F9C4844000200000C842C8340020E8
:108A0800B86C0020644E0020F44F0020782200202B
:108A1800E44F002068720020A8300020D4F8A49108
:108A2800EA4AEB4B089203EBC903126805929DEDE5
:108A3800057A9B88DFEDE77AE74A0691F8EE478AE0
:108A480009EE103A643BC82BA8BFC82368EEA78A72
:108A5800F8EE497A782BB8BF782368EEA78A07EE34
:108A6800903A2C27B0EE680A07FB0927B8EEE78A88
:108A780026F012FEB8EEC99AF0EE409AB0EE680AF7
:108A880026F06CFD38EE097A79EE487A28EE098AE4
:108A980067EE877AB7EE006A88EE277AB8F1140F86
:108AA8000699F8EE007A77EE076A60EE277A89EE83
:108AB800A67A77EE065A36EE477AC6EE256A67EE4C
:108AC800A67A27EE267AC7ED006A87ED047AC7ED05
:108AD800026AC7ED017AC7ED037A01F0A283BF4BA2
:108AE8009BF8008009F1010283FB0203A3EBE27902
:108AF80009EB49090131A2EB0909C4F8A011C4F82E
:108B0800A49109E7B64B1A78D4F8A4E1B04F9FEDC9
:108B1800B57A4FEACE0C07EB0C0383ED007A002AF6
:108B28007DD0B148B0EE476AF0EE476A0023F0EC1A
:108B3800017A013367EEA77A05EE903AB4EEE77A48
:108B4800F1EE10FAF8EEE55AB8BFB0EE677A934244
:108B580076EEA76AA7EEA56AE9D1F5EEC06A07EB3B
:108B68000C03F1EE10FA83ED007A58DDC6EE265AB2
:108B78009E4B9F4A1288F7EE007A75EEE75AD3EDBE
:108B8800007A65EEA77AFDEEE77A17EE903A812B28
:108B980041F3E6809342A8BF134607EE903AF8EEF9
:108BA800E77A944B2C2000FB0E3393ED097AD3ED32
:108BB800003A93ED0A6A93ED014AD3ED046AD3EDC6
:108BC800034A93ED025AA3EEA77AA4EE276A66EE4B
:108BD800C76AA7EE646ABDEEC77AE5EE276A17EEA4
:108BE800100A812883ED096AC3ED0A6A41F3B5804A
:108BF8008242A8BF024607EE902AF8EEE77AFCEE1A
:108C0800E77ACDED057ABDF8143007EB0C029380B6
:108C1800BEF1000F03D1B8F1130F01F01E82B8F1B5
:108C2800150F7FF450AABC44734FBCF8043027F8E2
:108C38001E30664BD4F8A0110893FFF751BADFF83D
:108C4800C091B9F800E0D9F804C04FEA5E0A4FEACB
:108C58008A0204EB8E085FEADE0E04EB020300F0E2
:108C6800A08010320EF1010E644803EB0E1E424440
:108C780010330CF1100708F1100151ED032A51EDE2
:108C8800043A10ED043A10ED032A51ED026A11ED91
:108C9800016A10ED020A10ED018A12ED044A12ED84
:108CA800035A53ED044A53ED035A13ED027A53ED78
:108CB800017A52ED020A12ED011A73EE238A72EE5E
:108CC800221A40ED048A40ED031A70EE268A78EEE7
:108CD800061A40ED028A40ED011A74EE848A75EE98
:108CE800851A43ED048A43ED031A77EE208A77EE5E
:108CF800811A43ED028A43ED011A73EE633A75EE69
:108D0800655A17ED035A32EE623A74EE644A65EE1C
:108D1800631A17ED044A23EE052A64EE652AE3EE8A
:108D2800041A1033734524EE843AA3EE842A00F122
:108D3800100007F11007A5EE853A01F1100102F1C4
:108D48001002E4EE852A41ED071A01ED082A02ED2A
:108D5800073A42ED082A57ED055A17ED065A70EE04
:108D6800666A38EE466A30EEC77A71EE677A26EEA2
:108D7800253A65EEE63A25EE674A67EE054AE6EEDD
:108D8800053AA6EE853AA7EE254AE7EEA54A01ED93
:108D9800063A41ED053A02ED064A42ED054A7FF4EE
:108DA8006CAF1FFA8AFA624651460F481DF0FEF969
:108DB8005146D9F8042040461DF0F8F99BF80030D8
:108DC800142B7FF489A9FFF781B900BFB86C002084
:108DD8006450002027D4D236346C0020565555559F
:108DE800464E00200000000068220020484E002067
:108DF800444E00207C50002084400020782200202F
:108E08004C4E0020DFF88093D548D9F80820B9F8EF
:108E18000C1025F081FB9BF80080B8F1140F01F0CD
:108E28000C82D4F8A0110131C4F8A011FFF7F8B8EA
:108E3800DFF858A39AF800205FEA920901F0C1828E
:108E4800DFF84CC309F101077F010CEB070E0CF1A9
:108E58002003ACF1700013ED076A53ED056A13EDBA
:108E6800037A53ED017A53ED025A13ED084A53ED94
:108E7800064A13ED045A26EE066A66EEA66A27EE3F
:108E8800077A67EEA77AA4EE046A20337345E4EE06
:108E9800A46A00F11000A5EE057AE5EEA57AF1EED8
:108EA800C65AB1EEE66AF1EEC76AB1EEE77A40ED6E
:108EB800085A00ED076A40ED066A00ED057ACAD146
:108EC800203FBC4404EB091012F0030318BF0CF157
:108ED800080C0FD05CED017A1CED027A67EEA77AD8
:108EE800013BE7EE077A0CF1080CB1EEE77AA0EC4B
:108EF800017AEFD1B8F1140F01F085810131C4F87E
:108F0800A01101E601F06EFF9BF800800490B8F113
:108F1800140F05BF934FD4F8A011D4F8A0113980CD
:108F2800FCF7BBBBDFF86C92DFF86CA299ED004A46
:108F380099ED097AD9ED014A99ED0A6AD9ED046AE1
:108F480099ED035AD9ED025A69EE277A0AEB88039C
:108F5800A7EE847AA7EEA46A66EEC76AA7EE456A0A
:108F6800E7EEA56A20EE070A89ED096AC9ED0A6AE3
:108F780029EE088A69EE288A83ED007A26F040FBFC
:108F8800D9ED145AD9ED1F6A99ED0B1AD9ED161AB5
:108F980099ED155A99ED207A99ED0C2AD9ED172AF1
:108FA80099ED0F6AD9ED1A7A99ED0E3AD9ED0D3A85
:108FB80099ED194AD9ED184AE8EE015A00210AEB51
:108FC8008802E8EEA16A00B2C4F88C11A8EE025A31
:108FD800C4F89011C4F89411A8EEA27A26EE656A36
:108FE80067EEE67AA5EEC35AA8EE236AA6EEC47A1F
:108FF800E8EEA47A89ED145AC2ED205A89ED156A73
:10900800C2ED406A89ED1F7AC9ED207AFEF735BABC
:10901800B5F92430EA6207EE903A0122F8EEE77AD1
:109028002B66EA670023B8F1010FC5ED1C7AC5ED80
:109038001B7A6B6701F00E80B0457CF4BFADB5F9C3
:1090480026306B6607EE903A00220123F8EEE77AA5
:109058002A63C5F890300023B8F1010FC5ED217AD5
:10906800C5ED207AC5F8883000F0E287B0457CF479
:10907800D6ADB5F92830AB6607EE903A0022012349
:10908800F8EEE77A6A63C5F8A4300023B8F1010F57
:10909800C5ED267AC5ED257AC5F89C307CF4F0AD8F
:1090A8009FED318AB9F1030F47D0BAF1000F09D00B
:1090B80007EE90AAF8EEE77AF4EEC87AF1EE10FA25
:1090C80001F12B81294AAB6E126894F8A811F88037
:1090D80003EB560393FBF6F600236E639362136368
:1090E800D36221B1224B1B88002B7CF4CAAD214BE3
:1090F8001B6813F4003304D01F4B1B79002B41F07D
:1091080005811E481A46C15C012903F10C0300F0D1
:109118002B860132152AF6D1FCF7B3BD184A927B8B
:10912800002A3DF4D4AEFDF7B7BDF7EE006AFEF7AE
:1091380009BDF7EE006AFEF786BCB0EE480A26F0D5
:109148005FFA00B2B1E7B4F84861013E36B2002ECA
:10915800A4F848617EF7A0AB0A49FDF70ABE00BF34
:1091680068220020844000200000000060440020A5
:10917800005C002098290020D05B0020081F03080D
:10918800E8530020504100204C4E0020464E00205D
:10919800E822002000510020644E0020D14B1968BD
:1091A80089037EF515AE4FF400325A60CE4B1A682B
:1091B800CE4B4FF6FE710A40CB490A601A89D20796
:1091C80011D41DF0F7FB0028FBD1C84A938823F07F
:1091D80002031B041B0C938099F80030002B7EF4CB
:1091E80002ADFEF7F0BC9A891A89D207FBD4E8E7EA
:1091F800B4F81A1101F57A7189B2FDF768BDBC4857
:10920800DFEDBC7A0068C4ED6E7A10F0805000F093
:10921800CA82B7EE007A77EE677AF4EEC67AF1EE94
:1092280010FA88BFF0EE467AB0EE676AC4ED7B7A32
:10923800FDF759B92B7803F00103FDF7F1BA16F0E1
:109248004DF816F013F896F82420FEF7A8BC16F08F
:1092580045F8042386F82430FEF774BFA64ADFEDEC
:10926800A77A92ED080AB4EEE70AF1EE10FA40F296
:109278009385049326F05AFAD4ED457A20EE270A0E
:1092880026F0BEF9B0F5617F049B00F3DF8507EE99
:10929800900AF8EEE76ADFED9A7A66EEA76A07EEBB
:1092A800907AB8EEE77AFDEEE67A17EE902A203249
:1092B800402A40F2D0879FED930A049326F0A0F944
:1092C80000B207EE900A049BB8EEE77A8E49D1ED1A
:1092D800037A77EE877AC1ED037AFDF7E5BC15F0DE
:1092E800FDFFF7680423002086F824303076002F2D
:1092F8003EF428AF336932687168B847FEF7D6BDC7
:10930800079820F0FBF9FEF76EBD7369D8F80020C6
:1093180064339342FEF4ABACFEF7C8BDBDEEE57A0C
:1093280017EE107AB0EE457AA2EEA77AF0EE477AF9
:10933800BEF1000F40F04083FDEEC77A17EE90CAE9
:1093480017EE90EAAC45A8BFAE466745C8BFBE4613
:1093580007EE90EAF8EEE77A012AC1ED007A3DF4CB
:109368005FAA90ED047ADDED0F7AE7EE067AB0EEAB
:10937800457AA2EEA77AFDEEC77A17EE90CA17EEE5
:1093880090EAAC45A8BFAE46BC45B8BFBE46FDF79F
:1093980013B9049B002B00F0CE85FDEEE57A0EA9EB
:1093A80001EB820217EE908AFDEEC57A91462346BC
:1093B800524674465548564F17EE90CA9E46CA46BE
:1093C80013E0FDEEC77A17EE909ACC4503DCA94569
:1093D8004B46A8BF2B4607EE903AF8EEE77A514580
:1093E800E7EC017A00F110001ED090ED007AF1EC64
:1093F800017AE7EE067A6346B0EE457AA7EEA27ADE
:10940800F0EE477A002ADCD034B1B4EE475AF1EED8
:1094180010FAC8BFF0EE657AFDEEE77A434617EE1C
:10942800909AC845D3DDD6E77446FDF7FCB9049B8E
:10943800002B00F02585FDEEC57A0EA901EB82020E
:1094480017EE90CAFDEEE57A9146234652467446D9
:109458002E482F4F17EE908AF1EE626A9E46CA4652
:1094680013E0FDEEC77A17EE903A634503DBAB4293
:10947800A8BF2B46994607EE909AF8EEE77A514531
:10948800E7EC017A00F11000CED090ED007AF1EC13
:10949800017AE7EE067AE146B0EE637AA6EEA77A9D
:1094A800F0EE477A002ADCD0434634B1B4EE457A70
:1094B800F1EE10FA48BFF0EE657AFDEEE77A17EEA6
:1094C800909AC14504DBA94517EE903AA8BF2B46F0
:1094D80007EE903AF8EEE77AD1E701F083FC0390C3
:1094E800FDF7CEBB000002405800024000380040A3
:1094F8006830002000000080206D00208FC2753C7D
:10950800D06D393A000000005041002068720020F8
:10951800A8300020B3784FF00109072B3EF65BAC6A
:10952800DFE803F0A2BB968B523C4604032373701A
:10953800FEF751BC33690622652B3C46B27037D919
:109548003278032A14BF6FF0FF026FF07F02A3F195
:10955800650303EA020303F1010314BF4FF48072A9
:1095680080229A42336123D2DAF80020F768023267
:1095780003EB0708904502D321F09EFE3369CD4ADC
:109588007760D16FC6F80880490203FB01F3052113
:10959800176042F81C3C42F8183CB170B268C649E2
:1095A800012022F051FC012840F0EB870623B3701C
:1095B8000021C24821F0BCFF012840F0E287B378BF
:1095C8000133DBB2B370A8E73278337DDFF814A338
:1095D800032A14BF4FF480784FF080082746002BE9
:1095E80000F08F80012BFAD1B54BD6F804E0D3F800
:1095F80000C0DAF800204FF0FF3300244FEA4C2C6B
:10960800B3FBFCFC1CEB0E0044F100010024A1425A
:1096180002F1020208BF904238BF0EEB0C02A949C2
:10962800022015F0A9FF032800F25986DFE800F0B0
:10963800025302533C46FEF7CEBB41F27013F35C73
:10964800002B3EF4C8AB9D4819F08EF9FEF7C3BB5A
:109658009D4B00930320B070302305229B49974807
:1096680022F060FBFEF7B7BB00230DF13808414636
:109678001846092215F040FE01287EF4ACAB0E9B7B
:1096880093F8FE21552A00F0598641F2B4120221BE
:109698000123B1547370FEF79EBB0DF1380841F2F7
:1096A800FC174146F0590023092215F025FE012830
:1096B8007EF491AB00230E993370B1F80B30B3F5FB
:1096C800007F00F0C98641F2B41203210123B1548E
:1096D8007370FEF780BB7468B36831691A1B8A42DD
:1096E80084BFF460326103283FF424AF0133B3FB35
:1096F800F8F208FB12320AB143449B1A0022736045
:109708003275DAF800206C490232002015F034FF77
:10971800032800F2E48501A353F820F03D960008E1
:10972800359700083D9600083D950008736886F84F
:1097380014900133B36057E76548006810F0805013
:1097480031D0B6EE007A67EE877AB4EEE76AF1EECA
:1097580010FA3FF569AD5CE586F819A0FEF773BB12
:10976800CE003EF563ADFDF7A6BA5A4EDFF878E1B4
:10977800594A96ED005ADEED003A584E1278C4ED7B
:109788007B7AC4ED793A84ED7A5AD6ED006A002ADC
:109798003CF4AFAB012284F8F021FCF7AABBF0EE51
:1097A800447AFCF72ABE11F4800001D00020C8E7F3
:1097B800B6EE007AB4EEC76AF1EE10FAC1DCFCF737
:1097C80092BEFDEEE57A28460EAB4549DFF81CC18E
:1097D80017EE907A754603EB82088646D1ED007A3B
:1097E800B3EC017AA7EE867A1031F0EE456AE7EE1F
:1097F800226A07EE907AB0EE667A35B1F4EE456AE1
:10980800F1EE10FA48BFB0EE657ABDEEC77A17EEF2
:10981800100A874204DC7045A8BF704607EE900A1C
:10982800F8EEE77A9845ECEC017AD7D1FDF7D8BB8A
:10983800012A7FF735AC07EE101AB8EEC77AC7EEE3
:10984800876AB1EEE68A2DE4012A40F3038407EE25
:10985800101AB8EEC77AC7EE876AB1EEE68AB9F190
:10986800030F14D0BAF1000F09D007EE90AAF8EE52
:10987800E77AB4EEE78AF1EE10FA00F34E852B6E24
:1098880003EB560393FBF6F3EB62FFF7D5BBB0EEA1
:10989800480A25F0B5FE00B2E4E7194604220EA8EE
:1098A80023F0E0FA9DF83B30AB2B04BF022373761C
:1098B800FEF7C9BAE893002058820020C49300201C
:1098C800649400205C82002085B20208A04403084A
:1098D800683000207C78002018560020347300205F
:1098E800687200205C9400202C730020A8300020AF
:1098F800012A40F39D8307EE101AB8EEC77AC7EE27
:10990800876AB1EEE68AB9F1030F14D0BAF1000FF5
:1099180009D007EE90AAF8EEE77AB4EEE78AF1EEFE
:1099280010FA00F3FA846B6E03EB560393FBF6F31D
:109938002B63FFF79BBBB0EE480A25F061FE00B22F
:10994800E4E7386802F006F951463A2015F05EFC63
:109958005146049004220EA823F084FA049B002B9D
:109968007FF46DAC15F0BAFC0E9B1BBAC3F3807381
:10997800B376FEF78FBA04212C2021F055FB032182
:1099880005904E2021F050FB0C210490362021F048
:109998004BFB049A059B911C421C8A400AFA03F36C
:1099A800A2FB0301420A42EAC152F263FEF791B9EF
:1099B800BDEEE57AFCF798BFB4EEC57AF1EE10FA81
:1099C800B8BFF0EE657AFDEEE77A17EE90EA17EE8B
:1099D80090CAAE45A8BFAC467745C8BFBC4607EE9F
:1099E80090CAF8EEE77A012AC1ED007A3CF418AF84
:1099F80090ED047ADDED0F7AE7EE067AB0EE457A5F
:109A0800A2EEA77AB4EEC57AF1EE10FAF0EE477A34
:109A1800B8BFF0EE657AFDEEE77A17EE90EA17EE3A
:109A280090CAAE45A8BFAC46BE45B8BFBC4607EE17
:109A380090CAF8EEE77A022AC1ED017A3CF4F0AE5A
:109A480090ED087ADDED107AE7EE067AB0EE457A09
:109A5800A2EEA77AB4EEC57AF1EE10FAF0EE477AE4
:109A6800B8BFF0EE657AFDEEE77A17EE90EA17EEEA
:109A780090CAAE45A8BFAC46BE45B8BFBC4607EEC7
:109A880090CAF8EEE77A032AC1ED027A3CF4C8AE30
:109A980090ED0C7ADDED117AE7EE067AB0EE457AB4
:109AA800A2EEA77AB4EEC57AF1EE10FAF0EE477A94
:109AB800B8BFF0EE657AFDEEE77A17EE90EA17EE9A
:109AC80090CAAE45A8BFAC46BE45B8BFBC4607EE77
:109AD80090CAF8EEE77A042AC1ED037A3CF4A0AE06
:109AE80090ED107ADDED127AE7EE067AB0EE457A5F
:109AF800A2EEA77AB4EEC57AF1EE10FAF0EE477A44
:109B0800B8BFF0EE657AFDEEE77A17EE90EA17EE49
:109B180090CAAE45A8BFAC46BE45B8BFBC4607EE26
:109B280090CAF8EEE77A052AC1ED047A3CF478AEDB
:109B380090ED147ADDED137AE7EE067AB0EE457A09
:109B4800A2EEA77AB4EEC57AF1EE10FAF0EE477AF3
:109B5800B8BFF0EE657AFDEEE77A17EE90EA17EEF9
:109B680090CAAE45A8BFAC46BE45B8BFBC4607EED6
:109B780090CAF8EEE77A062AC1ED057A3CF450AEB1
:109B880090ED187ADDED147AE7EE067AB0EE457AB4
:109B9800A2EEA77AB4EEC57AF1EE10FAF0EE477AA3
:109BA800B8BFF0EE657AFDEEE77A17EE90EA17EEA9
:109BB80090CAAE45A8BFAC46BE45B8BFBC4607EE86
:109BC80090CAF8EEE77A072AC1ED067A3CF428AE87
:109BD80090ED1C7ADDED157AE7EE067AB0EE457A5F
:109BE800A2EEA77AB4EEC57AF1EE10FAF0EE477A53
:109BF800B8BFF0EE657AFDEEE77A17EE90EA17EE59
:109C080090CAAE45A8BFAC46BE45B8BFBC4607EE35
:109C180090CAF8EEE77A082AC1ED077A3CF400AE5C
:109C280090ED207ADDED167AE7EE067AB0EE457A09
:109C3800A2EEA77AB4EEC57AF1EE10FAF0EE477A02
:109C4800B8BFF0EE657AFDEEE77A17EE90EA17EE08
:109C580090CAAE45A8BFAC46BE45B8BFBC4607EEE5
:109C680090CAF8EEE77A092AC1ED087A3CF4D8AD33
:109C780090ED247ADDED177AE7EE067AB0EE457AB4
:109C8800A2EEA77AB4EEC57AF1EE10FAF0EE477AB2
:109C9800B8BFF0EE657AFDEEE77A17EE90EA17EEB8
:109CA80090CAAE45A8BFAC46BE45B8BFBC4607EE95
:109CB80090CAF8EEE77A0A2AC1ED097A3CF4B0AD09
:109CC80090ED287ADDED187AE7EE067AB0EE457A5F
:109CD800A2EEA77AB4EEC57AF1EE10FAF0EE477A62
:109CE800B8BFF0EE657AFDEEE77A17EE90EA17EE68
:109CF80090CAAE45A8BFAC46BE45B8BFBC4607EE45
:109D080090CAF8EEE77A0B2AC1ED0A7A3CF488ADDE
:109D180090ED2C7ADDED197AE7EE067AB0EE457A09
:109D2800A7EEA27AB4EEC57AF1EE10FAF0EE477A11
:109D3800B8BFF0EE657AFDEEE77A17EE900A854235
:109D4800A8BF0546B842A8BF2F4607EE907AF8EE9E
:109D5800E77AC1ED0B7AFCF763BD8223FEF755BFA6
:109D6800DFEDC77AFEF71DBFD4F8AC6151003EB1F4
:109D78008B1800EB830376785B78B342BBF481AF32
:109D88000A4400EB82000022C4F8AC01A4F8FA21CE
:109D9800C4F8FC21FBF775BF9FEDD17AFFF796BA9F
:109DA800BB0000EB030C04EB030EB64B03EBC91925
:109DB8005FEA9A0300F0108301331B01059309EB56
:109DC80003070CF1100009F110030EF1100213ED56
:109DD800024A13ED035A13ED016A13ED047A50EDAC
:109DE800024A50ED035A50ED016A50ED047A64EED0
:109DF800244A65EE255A66EE266A67EE277A1033FE
:109E0800BB4242ED024A42ED035A42ED016A42ED7D
:109E1800047A00F1100002F11002D8D1059B103B22
:109E280009EB03000CEB030273441AF0030A3EF437
:109E3800C9ADB0EC017AF2EC017A67EE277ABAF193
:109E4800010AE3EC017AF4D1FEF7BCBD07EE907A83
:109E5800DFED8D6AB8EEE77A66EEA65A9FED8B5A6B
:109E68009FED8B6ADFED8B7AA5EE856A26EEA55A03
:109E7800E5EE867AE5EE276A26EE870AFFF71DBA31
:109E8800FDEEE57A0EABCDED067AFDEEC57A0994C6
:109E9800814FDFF84082CDF81C90544617EE90CAE7
:109EA800DDF818A00891F1EE626A03EB8202CDF8A2
:109EB80010E097ED007AF3EC017AE7EE067AB0EE5F
:109EC800637AA6EEA77AF0EE477ADCB9FDEEC77A98
:109ED800E64617EE909ACC4504DCA94517EE90EAC1
:109EE800A8BFAE4607EE90EAF8EEE77A002800F041
:109EF80019829342E8EC017A07F11007D9D1099C3D
:109F0800FCF791BC049931B1B4EE475AF1EE10FA5E
:109F1800C8BFF0EE657AFDEEE77A17EE90EAF245F3
:109F280007EE90AA04DCAE45A8BFAE4607EE90EA5D
:109F3800F8EEE77ADAE7FDEEC57A0EAB17EE90CACF
:109F4800FDEEE57A0994544FDFF88881CDED067A65
:109F5800544603EB8202CDF81C900891CDF810E02E
:109F680017EE90AA05E09342E8EC017A07F1100792
:109F7800C5D097ED007AF3EC017AE7EE067AB0EEF9
:109F8800457AA2EEA77AF0EE477ADCB9FDEEC77AF9
:109F9800E64617EE909ACC4503DCA945CE46A8BF05
:109FA800AE4607EE90EAF8EEE77A0028DBD108998A
:109FB8000029D8D107998E4605998E45B8BFF0EE8D
:109FC800657AD0E7049931B1B4EE475AF1EE10FA48
:109FD800C8BFF0EE657AFDEEE77AD64617EE909A9E
:109FE800CA45DEDCD9E7F0EE427AFCF706BA2B4820
:109FF80018F0BAFCFEF7BCB8294818F0B5FCFEF713
:10A00800B1B8284818F0B0FCFEF7B8B8BCF838105A
:10A018009FED257A07EE901AF8EEE77A234967EE66
:10A02800877AC1ED007AFCF746BE2149FCF799BE54
:10A038009FED2B8A67E41F4A516900293BF4B1ACB4
:10A048001D4908881D4991FBF0F11068016053749F
:10A05800FBF7A7BC9FED228A01E49FED190A194B73
:10A06800089325EE800A25F0CBFA174FD4F8A011F3
:10A07800F880FEF735B81548154A8446FEF791BCB6
:10A0880000000243644E002084F9223F92E741B960
:10A098009730083C15A82ABE68720020F892002064
:10A0A8000C9400203C9300206F12833A1800002083
:10A0B80050410020E0990020F899002020A10700D5
:10A0C8000000C842B86C002084400020E44F002003
:10A0D80068220020A830002035FA8E3CDB0FC93FEB
:10A0E8000000000007EE906AF8EEE78A5FED067A56
:10A0F8001FED060A84F8846168EEA78A38EE800AA4
:10A10800FDEEC07A17EE903A2033402B40F25E8184
:10A118001FED0D0ABE4BFDEEE87A83ED010A17EE3E
:10A12800903A2033402B00F25481DFEDBA7AF4EEF6
:10A13800E78AF1EE10FA40F32182DFEDB76ADFED2E
:10A14800B77A01E0F0EE478AF4EEE78AF1EE10FA0A
:10A1580038EEE67AF6DCDFEDB27AB4EEE77AF1EEC5
:10A1680010FA40F118829FEDAC6ADFEDAE6A01E0AB
:10A17800B0EE677AB4EEE67AF1EE10FA77EE067A88
:10A18800F6D49FEDA97AF4EEC77AF1EE10FA40F30F
:10A198002B819FEDA07A77EE677A27EEA76ADFED2D
:10A1A800A35ADFEDA36A9FEDA37AE6EE256A67EE70
:10A1B800865AA6EE267AE5EE877AC4ED627AFEF72D
:10A1C80096BA91ED000A06930592049125F018FAC3
:10A1D800DFF87CE2984FDEF8ECE0DFF878C23880F0
:10A1E8008CFB0E3C4FEAEE70C0EBAC1007EE900A09
:10A1F800F8EEE77A04A9FDEEE77A0EC917EE900AA1
:10A208007880FCF7B3BD00F0EDFD049B8A4F9AF807
:10A218000020D4F8A0119BF80080C01AB880FEF77F
:10A228006DBE00F0DFFD049B834FD4F8A491D4F8F1
:10A23800A011C01A7880FEF752BC00F0D3FD049B31
:10A248007D4F9BF80080C01A7880FEF7EABD86F83B
:10A258002430FDF7C0BDDFED6F7AF4EEE76AF1EE6A
:10A2680010FA40F3B681DFED6C5A9FED6C6A01E09D
:10A27800F0EE676AF4EEC66AF1EE10FA76EEE57A69
:10A28800F6DCDFED676AF4EEE67AF1EE10FA40F1FB
:10A298009D81DFED615A9FED636A01E0F0EE667A19
:10A2A800F4EEC67AF1EE10FA77EEA56AF6D4DFED91
:10A2B8005E7AF4EEE76AF1EE10FA04DDDFED557A26
:10A2C80077EEE66AC8E5DFED5D7AF4EEE76AF1EE6F
:10A2D80010FA44BFDFED527A77EEE66ABCE5337DCB
:10A2E800FFF77DB9564BF7681B687361072386F83B
:10A2F8002430002F3DF46FAD336932687168012056
:10A30800B84796F82420531EFDF75BBD4D4B1B78CC
:10A31800002B65D00023FEF7F4BEF880A5F8A860EE
:10A32800FBF7B6BC089900297FF4E3AD07998E4680
:10A3380005998E45B8BFF0EE657ADAE593F8FF2106
:10A34800AA2A7FF4A2A9D3F8C6214AB193F8C21168
:10A35800A1F10B0001282DD901F0F701062929D018
:10A36800D3F8D6214AB193F8D211A1F10B000128F4
:10A3780020D901F0F70106291CD0D3F8E6214AB10B
:10A3880093F8E211A1F10B00012813D901F0F701AC
:10A3980006290FD0D3F8F621002A3FF476A993F8BE
:10A3A800F231A3F10B01012904D903F0F703062BBD
:10A3B8007FF46BA941F2FC1101237250B370FFF7CF
:10A3C8006EB9214800F1800CFEF77EBDF6F7B6FEA7
:10A3D800A0E6DFED1E7AF0E673466246484624E5BD
:10A3E8001EF030FFFBF74DBC9FED147AF4EEC77AF0
:10A3F800F1EE10FA44BF9FED0A7A77EE677ACCE661
:10A4080000F0DD80042386F82430FDF74DBD00BF41
:10A4180018000020DB0F4940DB0FC940E4CB164190
:10A42800DB0F49C0E4CB16C1DB0FC93F92E741B946
:10A438009730083C15A82ABE84400020DB0FC9BF0E
:10A44800009A00204F4100206822002000000000F0
:10A45800A4080020D34D62100B7C022B7FF433A993
:10A4680091F8FE31552B7FF42EA991F8FF31AA2BD4
:10A478007FF429A9B1F80EE0F759674B77441F60BC
:10A4880091F80D8041F2102208F1FF337F2B46F836
:10A4980002803FF618A9C8F1000338EA03037FF4E5
:10A4A80012A94FEA482341F21822013BB350C88A47
:10A4B80000B9486A594B41F20422B050B1F8112052
:10A4C800520102F2FF1252121A60B1F8133003B9A6
:10A4D8000B6A400096448644A3EB0E0341F2082C15
:10A4E80040F6F47EB3FBF8F3734546F80C3040F2BF
:10A4F8008F804FF6F47E734540F2868003233370D5
:10A50800CB6A47493A44104441F20C2741F21C22D5
:10A518000978F051B350002973D0B3780133B37080
:10A52800FDF759BC94F8D831002B7BF45CAAFBF7F3
:10A5380045BA9BF80010132917D04BB107F5F46002
:10A54800B0EE480A2844D5F89C379847B0EE408AC0
:10A558009BF80030132B7DF4E6ACB0EE480A25F0EA
:10A568004FF8A9F80200FDF7E0BCB0EE480A0593E1
:10A5780025F046F8059BA9F80000DEE7B0EE687AFA
:10A58800E9E502287DF427AC41F2B4120123B35463
:10A598007370FDF720BCF0EE477AF2E5089BD3ED27
:10A5A80003DA204B93ED020A1F4B3CEE6DDA28EEDE
:10A5B800800A20EE0D0A83ED020AFBF7A7BB14F010
:10A5C80087FD02287DF472ACFDF76EBCF0EE676A79
:10A5D8006DE6F0EE667A54E694F8C831002BDDD1CA
:10A5E800104B2B4493ED000A039BD3ED01DA28EEC0
:10A5F800800A3CEE6DDA20EE0D0A88ED000AFBF7C2
:10A6080085BB24F09DFD88E702233370002378E79B
:10A6180001233370FFF757B8549400207494002036
:10A62800349400200C3F002074300020436A826973
:10A6380070B4D154436A0469426B0133A34228BF02
:10A6480000234362DAB1116811F0010101D070BC36
:10A658007047856A86699D422E44D6600BD3641B79
:10A66800546081621368002143F0010380F84410AC
:10A6780070BC136070475D1B55608362F2E7026D22
:10A68800136843F080031360E1E700BF026B10B466
:10A6980062B1036CC2684469D11A013B615C5DF820
:10A6A800044B08BF13460364C8B27047016A436984
:10A6B800C4685B5C0131A14228BF114601625DF8A4
:10A6C800044BD8B2704700BF436B13B190F84400F5
:10A6D8007047836A406A181AB0FA80F040097047D8
:10A6E800416A836A99420AD3CB1A416B026961B104
:10A6F8004968501E0B4483420AD2C01A7047026947
:10A708001144CB1A416B0029F2D1501EC01A704770
:10A7180000207047036B43B1026C5B6893422FBF04
:10A72800981AC0689B1AC0187047C269036A9A428F
:10A738002FBFD01AC0688018C01A70470A4B30B5AE
:10A7480003F1140493F900205D78072AC8BF143A6E
:10A75800811804330D7313F8025C855413F8012C27
:10A768000A76A342EED130BDF01B030803682DE939
:10A77800F041DF691FB13B46BDE8F0411847002AA8
:10A78800164611DD04460D460E4400E023689B681A
:10A79800204698470028F9D0236815F8011B1B6844
:10A7A80020469847AE42F1D1BDE8F08100230370FE
:10A7B80043708370C3707047232303702423C370CE
:10A7C800252383712D2343702E2303712F23C371F7
:10A7D800704700BF2DE9F041446814B12568A4888A
:10A7E8002C8541F08001046840F2E93501E0002D34
:10A7F8005AD02689013D16F0020FADB2F7D0217369
:10A8080004F10C0640F2E93101E000295DD0258908
:10A81800013915F0010F89B2F7D031780468A189A0
:10A828004FF0000C4FF47A714FF6FF764FF0FF0EA1
:10A83800624502D130E0B1421ED02589013915F0B8
:10A84800020589B2F7D084F80CE004F10C084FF443
:10A858007A7102E0B9B2B1420ED0258915F001052E
:10A8680001F1FF37F6D098F80050EDB20BB11D702A
:10A8780001330CF1010CDBE71C4B9C4204D0A3F51F
:10A8880078439C4208D10125194B03EB05156B89C8
:10A8980001339BB26B816B89436813B11A689B883B
:10A8A80093610120BDE8F08110498C4204D0A1F5E4
:10A8B80078418C42B3D101250D4901EB0515698911
:10A8C800013189B269816989A9E7084DAC4203D091
:10A8D80008498C42A2D10121054C04EB01114C8995
:10A8E8000134A4B24C814989046898E700300140DA
:10A8F8002C9A00200038004030B4436813B11C681B
:10A908009B882385036840F2E93401E0002C37D0A6
:10A918001D89013C15F0020FA4B2F7D0197303F199
:10A928000C0540F2E93101E000294BD01C890139BE
:10A9380014F0010F89B2F7D02B78036840F2E9319F
:10A9480001E000292DD01C89013914F0020F89B2C9
:10A95800F7D01A7303F10C0440F2E93201E0002A3F
:10A9680041D01989013A11F0010F92B2F7D023783A
:10A97800436813B11A689B889361012030BC704703
:10A9880021498B4204D0A1F578418B42D6D10124CC
:10A998001E4901EB04146189013189B26181618921
:10A9A800CCE7194A934204D0A2F578429342DFD10A
:10A9B8000121164B03EB01114B8901339BB24B81EB
:10A9C8004B89D5E7104CA34203D011498B42B4D12F
:10A9D80001210E4B03EB01114B8901339BB24B81D3
:10A9E8004B890368AAE708498B4203D0084A934277
:10A9F800BED10122054B03EB0212538901339BB2EE
:10AA080053815389B4E700BF003001402C9A0020DD
:10AA18000038004030B50446006D61710368A268D3
:10AA280023F00103036087B0A379009213F00402B6
:10AA38003DD04FF4805213F00203019244D10293A7
:10AA48004FF480630022039311F00103059237D17C
:10AA5800049308238D07694648BF049315F046F907
:10AA68006079236DA17900F00202002A15BF4FF426
:10AA780040324FF480324FF40034002410F0010FBC
:10AA8800586808BF2246CC074CBF024320EA02029E
:10AA98005A609A6809074CBF42F0080222F008027F
:10AAA8009A601A6842F001021A6007B030BD13F0CC
:10AAB800020301920BD04FF4005513460295C1E7EB
:10AAC800042304930C23C5E74FF40053B7E702931C
:10AAD800B8E700BF10B50446006DA160036823F015
:10AAE80001030360A37986B013F00402009141D0FA
:10AAF8004FF4805213F00203019244D102934FF4B1
:10AB0800806362790393D1074FF0000304930593A0
:10AB180045BF0423049308230C236946920748BFC2
:10AB2800049315F0E3F86079236DA17900F002022F
:10AB3800002A15BF4FF440324FF480324FF40034EE
:10AB4800002410F0010F586808BF2246CC074CBFFC
:10AB5800024320EA02025A609A6809074CBF42F091
:10AB6800080222F008029A601A6842F001021A608C
:10AB780006B010BD13F00203019207D04FF4005144
:10AB880013460291BDE74FF40053B7E70293B8E7C5
:10AB98002DE9F04F013085B0C3B203930B46029103
:10ABA8008B4C8C4E002B00F099808B4D8B4FDFF82F
:10ABB800309221F05DFD4FF4FA7A4FF0100C4FF40B
:10ABC8007A70D9F80430C3F30803002B40F0DE8014
:10ABD800EFF31183002B40F0D9802968A26800BFE9
:10ABE8002B689942F9D1D7F800E000FB0EF39B1AC5
:10ABF800B3FBFEF300FB01314FF0010E0191D9F8D0
:10AC08000430C3F30803002B40F08780EFF311836F
:10AC1800002B40F082802B68A16800BF2A6893420D
:10AC2800F9D1D7F800B000FB0BF2521AB2FBFBF2D5
:10AC380000FB0323019A9B1AB3F57A7FDFD3BAF19D
:10AC4800010ABED1039B002B40F0BD804FF47A7AF5
:10AC5800DFF88C9150464FF0100CD9F80430C3F34C
:10AC68000803002B75D1EFF31183002B71D12968EC
:10AC7800A26800BF2B689942F9D1D7F800E000FB21
:10AC88000EF39B1AB3FBFEF300FB01314FF0010EEC
:10AC98000191D9F80430C3F3080313BBEFF3118310
:10ACA800FBB92B68A16800BF2A689342F9D1D7F88D
:10ACB80000B000FB0BF2521AB2FBFBF200FB0323BD
:10ACC800019A9B1AB3F57A7FE3D3BAF1010AC4D18A
:10ACD800029B013B0293002B7FF467AF05B0BDE8F0
:10ACE800F08FEFF311888CF31288A1682368DB03D7
:10ACF80044BFC6F800E0A1682B6832685FFA88F89C
:10AD080088F31188D7F800801A4400FB08F35B1A0F
:10AD1800B3FBF8F300FB0233D2E7EFF311888CF3AF
:10AD28001288A1682368DB0344BFC6F800E0A16865
:10AD38002B6832685FFA88F888F31188D7F80080A2
:10AD48001A4400FB08F35B1AB3FBF8F300FB023369
:10AD580070E7EFF311828CF31288D4F808E02368C7
:10AD6800D90303D501233360D4F808E02B68316890
:10AD7800D2B282F311883A68194400FB02F3A3EBBC
:10AD88000E03B3FBF2F300FB01317FE7EFF311820F
:10AD98008CF31288D4F808E02368D90303D501237B
:10ADA8003360D4F808E02B683168D2B282F3118896
:10ADB8003A68194400FB02F3A3EB0E03B3FBF2F36A
:10ADC80000FB013118E7184621F0D2FA3EE700BF30
:10ADD80010E000E0FC990020009A0020049A00206E
:10ADE80000ED00E0204B5B68C3F3080330B4BBB947
:10ADF800EFF31183A3B91D4B1D4C1868A16800BF60
:10AE08001A689042F9D11B4B1C684FF47A7202FB06
:10AE180004F3591AB1FBF4F130BC02FB001070477F
:10AE2800EFF31182102383F3128811498C680B68A1
:10AE380013F4803F104B02D0012018608C680B4936
:10AE4800D2B20D68186882F311880A4B19684FF45A
:10AE58007A72284402FB01F31B1B30BCB3FBF1F3ED
:10AE680002FB0030704700BF00ED00E0009A0020B0
:10AE780010E000E0049A0020FC9900202DE9F84F2A
:10AE88008046FFF7AFFF254E2549DFF8A0E0254AA9
:10AE9800254D844610274FF47A740120DEF80430DB
:10AEA800C3F30803D3B9EFF31183BBB90B68D2F826
:10AEB80008A000BFD1F800904B45F7D1D6F800B0F4
:10AEC80004FB0BF9A9EB0A09B9FBFBF904FB039393
:10AED800A3EB0C034345E1D3BDE8F88FEFF3118AE8
:10AEE80087F31288D2F808B01368DB0344BF2860E0
:10AEF800D2F808B00B68D5F800905FFA8AFA8AF39E
:10AF08001188D6F800A0994404FB0AF3A3EB0B03BD
:10AF1800B3FBFAF304FB0933DAE700BF049A002015
:10AF2800009A002010E000E0FC99002000ED00E00D
:10AF38002DE9F04FDFF830C1474A4849484E494D9E
:10AF48008046102718F1FF38C0F08480DCF8043000
:10AF5800C3F30803002B5CD1EFF31183002B58D106
:10AF68000B68946800BF08688342F9D1D6F800904E
:10AF78004FF47A7000FB09FEAEEB040EBEFBF9FE3F
:10AF880000FB03EEDCF80430C3F308034FF47A74D3
:10AF98000120FBB9EFF31183E3B90B68D2F808A0DD
:10AFA80000BFD1F800904B45F7D1D6F800B004FBAC
:10AFB8000BF9A9EB0A09B9FBFBF904FB0393A3EB13
:10AFC8000E03B3F57A7FBDD2DCF80430C3F308036F
:10AFD800002BDFD0EFF3118A87F31288D2F808B07C
:10AFE8001368DB0344BF2860D2F808B00B68D5F8B3
:10AFF80000905FFA8AFA8AF31188D6F800A099447B
:10B0080004FB0AF3A3EB0B03B3FBFAF304FB0933CA
:10B01800D5E7EFF3118487F31288D2F80890136804
:10B02800D80303D501232B60D2F808900B68286851
:10B03800E4B284F31188D6F800A04FF47A7400EBD8
:10B04800030E04FB0AF3A3EB0903B3FBFAF304FBB7
:10B058000E3E97E7BDE8F08F10E000E0009A002070
:10B06800049A0020FC99002000ED00E030B4EFF3D2
:10B078001183102282F312880649074C0A68074890
:10B08800013200250A602560DBB2026883F311886B
:10B0980030BC7047009A0020FC99002010E000E0C6
:10B0A8001D4B70B59C68236D226BDD69C2B1636B63
:10B0B8002BB12B0702D5236D08221A6270BD2A0610
:10B0C800F7D5A26A616A8A421FD0511CA069A162A1
:10B0D800825C2069266D81423285EAD3A362E8E763
:10B0E800A906E4D5E26A1AB1988C80B29047DEE7E7
:10B0F800E1699B8C6069DBB24E1CE6614354E169EF
:10B10800E368994228BFE261D1E7226D136823F012
:10B1180080031360CDE700BFBC4C00201D4B70B509
:10B128005C68236D226BDD69C2B1636B2BB12B07A1
:10B1380002D5236D08221A6270BD2A06F7D5A26AC5
:10B14800616A8A421FD0511CA069A162825C206991
:10B15800266D81423285EAD3A362E8E7A906E4D5E1
:10B16800E26A1AB1988C80B29047DEE7E1699B8C5D
:10B178006069DBB24E1CE6614354E169E3689942B9
:10B1880028BFE261D1E7226D136823F080031360C2
:10B19800CDE700BFBC4C00201D4B70B51C68236D6B
:10B1A800226BDD69C2B1636B2BB12B0702D5236D0E
:10B1B80008221A6270BD2A06F7D5A26A616A8A4215
:10B1C8001FD0511CA069A162825C2069266D814252
:10B1D8003285EAD3A362E8E7A906E4D5E26A1AB1A0
:10B1E800988C80B29047DEE7E1699B8C6069DBB29E
:10B1F8004E1CE6614354E169E368994228BFE26165
:10B20800D1E7226D136823F080031360CDE700BFF8
:10B21800BC4C002003685B6A03B11847704700BF45
:10B2280003681B6A03B11847704700BF03682DE91C
:10B23800F041DF691FB13B46BDE8F0411847002ADD
:10B24800164611DD04460D460E4400E023689B684F
:10B25800204698470028F9D0236815F8011B1B6879
:10B2680020469847AE42F1D1BDE8F08103689B695A
:10B27800184700BF0368DB68184700BF03689B686E
:10B28800184700BF03685B68184700BF03681B685E
:10B29800184700BF054B53F8203033B11A689B8814
:10B2A800918A0B4218BF1B0493617047CC99002008
:10B2B80010B50409013C052C17D80D4B33F81420A0
:10B2C80000F00F0042FA00F313F001030DD0012340
:10B2D80003FA00F00138104023F052FE054A064BED
:10B2E800125D104403EBC00010BD002010BD00BF6C
:10B2F8005428030860280308B85400202DE9F04FAB
:10B308004A484B4B4B4C4FF090414FF0010A4FF0DD
:10B3180002094FF004084FF0080C4FF0100E2027D8
:10B328004026802530F8022B12F0010F03D0196057
:10B33800A3F804A0083312F0020F03D01960A3F891
:10B348000490083312F0040F03D01960A3F80480A6
:10B35800083312F0080F03D01960A3F804C00833AB
:10B3680012F0100F03D01960A3F804E0083312F0AC
:10B37800200F02D019609F80083312F0400F02D0CE
:10B3880019609E80083312F0800F02D019609D80EA
:10B39800083312F4807F05D04FF4807B1960A3F83E
:10B3A80004B0083312F4007F05D04FF4007B196015
:10B3B800A3F804B0083312F4806F05D04FF4806B03
:10B3C8001960A3F804B0083312F4006F05D04FF4E5
:10B3D800006B1960A3F804B0083312F4805F05D03D
:10B3E8004FF4805B1960A3F804B0083312F4005FCF
:10B3F80005D04FF4005B1960A3F804B0083312F4C9
:10B40800804F05D04FF4804B1960A3F804B008337F
:10B41800D20B04D04FF4004219609A80083301F52A
:10B428008061A1427FF47EAFBDE8F08F5428030805
:10B43800B854002000180048002867D003682DE998
:10B44800F04F03F138445C4EA40A0125345D04F042
:10B458001F066409022C05FA06F558D0032C00F0E3
:10B46800A580012C58D08088B0FA80F4C4F11F045C
:10B47800A4B2E50803EB850504F007042E6AA400CE
:10B488000F27A74026EA07062E622E6A01F0030757
:10B49800A2407C1E3243012CC1F3810CC1F3001879
:10B4A8002A62C1F341113CD9C60700F1898085079A
:10B4B80000F19580440700F1A380020700F1B180F4
:10B4C800C60600F1BF80850600F1CD80440600F174
:10B4D800DB80020600F1E980C60500F1F7808505EA
:10B4E80000F10581440500F11381020500F1218175
:10B4F800C60400F12F81850400F13D81440400F168
:10B508004B81020400F15981BDE8F08F70472B4C44
:10B51800A6693543A561A6E7284C66693543656188
:10B52800A1E7002422464FF0010E4FF0030904E082
:10B538000132102A04F10204E6D00EFA02F636EAC5
:10B548000005F5D1D3F808A009FA04F5ED430AEA95
:10B55800050AC3F808A0D3F808B00CFA04FA4AEAB6
:10B568000B0AC3F808A0B3F804A01FFA8AFA2AEA5B
:10B5780006069E80B3F804A008FA02F646EA0A0610
:10B58800B6B29E801E682E401E60D3F800A007FA4F
:10B5980004F646EA0A061E60D3F80CA001FA04F67F
:10B5A80005EA0A0A46EA0A05DD60C1E7034CE669CE
:10B5B8003543E56157E700BF6828030800100240DB
:10B5C8001A6822F003021A601A683A431A60DA68A5
:10B5D80022F003020A438507DA607FF56BAF1A6829
:10B5E80022F00C021A601A6842EA87021A60DA68C6
:10B5F80022F00C0242EA81024407DA607FF55DAF6F
:10B608001A6822F030021A601A6842EA07121A60B1
:10B61800DA6822F0300242EA0112DA6002077FF5A6
:10B628004FAF1A6822F0C0021A601A6842EA8712FD
:10B638001A60DA6822F0C00242EA8112C606DA60AD
:10B648007FF541AF1A6822F440721A601A6842EA1C
:10B6580007221A60DA6822F4407242EA012285065B
:10B66800DA607FF533AF1A6822F440621A601A680C
:10B6780042EA87221A60DA6822F4406242EA8122AA
:10B688004406DA607FF525AF1A6822F440521A6042
:10B698001A6842EA07321A60DA6822F4405242EA2B
:10B6A8000132DA6002067FF517AF1A6822F44042C9
:10B6B8001A601A6842EA87321A60DA6822F440424D
:10B6C80042EA8132C605DA607FF509AF1A6822F4CA
:10B6D80040321A601A6842EA07421A60DA6822F4AD
:10B6E800403242EA01428505DA607FF5FBAE1A680E
:10B6F80022F440221A601A6842EA87421A60DA681D
:10B7080022F4402242EA81424405DA607FF5EDAE38
:10B718001A6822F440121A601A6842EA07521A603C
:10B72800DA6822F4401242EA0152DA6002057FF533
:10B73800DFAE1A6822F440021A601A6842EA875299
:10B748001A60DA6822F4400242EA8152C604DA60DA
:10B758007FF5D1AE1A6822F040721A601A6842EA80
:10B7680007621A60DA6822F0407242EA01628504D0
:10B77800DA607FF5C3AE1A6822F040621A601A6870
:10B7880042EA87621A60DA6822F0406242EA81621D
:10B798004404DA607FF5B5AE1A6822F040521A60A8
:10B7A8001A6842EA07721A60DA6822F0405242EADE
:10B7B8000172DA6002047FF5A7AE1A6822F04042EF
:10B7C8001A601A6842EA87771F60DA6822F04042F6
:10B7D80042EA8171D960BDE8F08F00BF002852D0DD
:10B7E800036803F138422DE9F04F920A504DAA5CE4
:10B7F80002F01F0552090124022A04FA05F443D075
:10B80800032A00F09080012A43D001F003077A1E32
:10B81800012AC1F3810CC1F300188088C1F34111DA
:10B828003CD9C60700F18880850700F19480440759
:10B8380000F1A280020700F1B080C60600F1BE80C8
:10B84800850600F1CC80440600F1DA80020600F19A
:10B85800E880C60500F1F680850500F104814405FD
:10B8680000F11281020500F12081C60400F12E8149
:10B87800850400F13C81440400F14A81020400F18E
:10B888005881BDE8F08F70472A4A95692C43946126
:10B89800BBE7284A55692C435461B6E70024224681
:10B8A8004FF0010E4FF0030904E00132102A04F1B1
:10B8B8000204E6D00EFA02F636EA0005F5D1D3F80E
:10B8C80008A009FA04F5ED430AEA050AC3F808A036
:10B8D800D3F808B00CFA04FA4AEA0B0AC3F808A02D
:10B8E800B3F804A01FFA8AFA2AEA06069E80B3F87B
:10B8F80004A008FA02F646EA0A06B6B29E801E6856
:10B908002E401E60D3F800A007FA04F646EA0A069D
:10B918001E60D3F80CA001FA04F605EA0A0A46EA02
:10B928000A05DD60C1E7034AD5692C43D4616CE799
:10B9380068280308001002401A6822F003021A60FF
:10B948001A683A431A60DA6822F003020A43850744
:10B95800DA607FF56CAF1A6822F00C021A601A6878
:10B9680042EA87021A60DA6822F00C0242EA81028F
:10B978004407DA607FF55EAF1A6822F030021A6079
:10B988001A6842EA07121A60DA6822F0300242EABC
:10B998000112DA6002077FF550AF1A6822F0C00280
:10B9A8001A601A6842EA87121A60DA6822F0C0023E
:10B9B80042EA8112C606DA607FF542AF1A6822F4BD
:10B9C80040721A601A6842EA07221A60DA6822F49A
:10B9D800407242EA01228506DA607FF534AF1A68C0
:10B9E80022F440621A601A6842EA87221A60DA680A
:10B9F80022F4406242EA81224406DA607FF526AFEB
:10BA08001A6822F440521A601A6842EA07321A6029
:10BA1800DA6822F4405242EA0132DA6002067FF51F
:10BA280018AF1A6822F440421A601A6842EA87324C
:10BA38001A60DA6822F4404242EA8132C605DA60C6
:10BA48007FF50AAF1A6822F440321A601A6842EA8F
:10BA580007421A60DA6822F4403242EA0142850558
:10BA6800DA607FF5FCAE1A6822F440221A601A6880
:10BA780042EA87421A60DA6822F4402242EA8142A6
:10BA88004405DA607FF5EEAE1A6822F440121A60B7
:10BA98001A6842EA07521A60DA6822F4401242EA47
:10BAA8000152DA6002057FF5E0AE1A6822F440021E
:10BAB8001A601A6842EA87521A60DA6822F4400269
:10BAC80042EA8152C604DA607FF5D2AE1A6822F0E3
:10BAD80040721A601A6842EA07621A60DA6822F04D
:10BAE800407242EA01628504DA607FF5C4AE1A68E2
:10BAF80022F040621A601A6842EA87621A60DA68BD
:10BB080022F0406242EA81624404DA607FF5B6AE10
:10BB18001A6822F040521A601A6842EA07721A60DC
:10BB2800DA6822F0405242EA0172DA6002047FF5D4
:10BB3800A8AE1A6822F040421A601A6842EA87776B
:10BB48001F60DA6822F0404242EA8171D960BDE89C
:10BB5800F08F00BF10B1036882881A85704700BF54
:10BB680010B1036882889A61704700BF38B1002914
:10BB78008388026814BF002110218B4093617047AD
:10BB88000E4B1B8801463BB90D4B0E4A1B781068BB
:10BB98000BB981F00101E9E70B4B5A691AB118B9E1
:10BBA8001A68106058747047084A18681188084A5B
:10BBB80092FBF1F20121026059747047D899002074
:10BBC800DA990020DC990020E0990020F8990020FB
:10BBD80020A1070010B40A4B0A4A1C7801238340AD
:10BBE800234052F8200029B9B3FA83F149095DF8D6
:10BBF800044BBBE7191C18BF01215DF8044BB5E7DE
:10BC0800CB990020CC99002030B1036882881B8A28
:10BC18001A4214BF01200020704700BF2DE9F041EF
:10BC28000B4E346873691C400FD0DFF82880012759
:10BC3800B4FA84F3C3F11F0307FA03F558F8230095
:10BC480003689847AC437561F2D1BDE8F08100BF45
:10BC580000040140849900202DE9F0410B4E34681E
:10BC680073691C400FD0DFF828800127B4FA84F3E9
:10BC7800C3F11F0307FA03F558F823000368984730
:10BC8800AC437561F2D1BDE8F08100BF000401400A
:10BC9800849900202DE9F0410B4E346873691C40EB
:10BCA8000FD0DFF828800127B4FA84F3C3F11F030B
:10BCB80007FA03F558F8230003689847AC43756101
:10BCC800F2D1BDE8F08100BF000401408499002052
:10BCD8002DE9F0410B4E346873691C400FD0DFF832
:10BCE80028800127B4FA84F3C3F11F0307FA03F588
:10BCF80058F8230003689847AC437561F2D1BDE852
:10BD0800F08100BF00040140849900202DE9F04132
:10BD18000B4E346873691C400FD0DFF82880012768
:10BD2800B4FA84F3C3F11F0307FA03F558F82300A4
:10BD380003689847AC437561F2D1BDE8F08100BF54
:10BD480000040140849900202DE9F0410B4E34682D
:10BD580073691C400FD0DFF828800127B4FA84F3F8
:10BD6800C3F11F0307FA03F558F82300036898473F
:10BD7800AC437561F2D1BDE8F08100BF0004014019
:10BD8800849900202DE9F0410B4E346873691C40FA
:10BD98000FD0DFF828800127B4FA84F3C3F11F031A
:10BDA80007FA03F558F8230003689847AC43756110
:10BDB800F2D1BDE8F08100BF000401408499002061
:10BDC8000D490E488A6908B542F001020C4B8A6198
:10BDD8001A6842F400621A601A6842F480521A60C3
:10BDE8000021402225F019FD064B4FF0FF321A6062
:10BDF800C3F8032008BD00BF00100240849900204A
:10BE080000000140C49900202DE9F041044618467D
:10BE18000D461646984622F0E9FB2768E672284444
:10BE2800A07229467D69434632462046AC46BDE8A5
:10BE3800F0416047036810B504461B6898472368BB
:10BE480020469B689847A37B0133A37310BD00BFAE
:10BE580010B5036804469B689847FF230122637363
:10BE6800227310BD08B5FFF723FA38B12C2282716E
:10BE78000022C2712021BDE80840AFE408BD00BF20
:10BE880030B4436813B11A689B88138541F0800168
:10BE9800026840F2E93301E0002B48D01589013BE4
:10BEA80015F0020F9BB2F7D0117302F10C0540F2A6
:10BEB800E93301E0002B4AD01189013B11F0010F51
:10BEC8009BB2F7D02B780268938940F2E93300E0FF
:10BED800EBB11189013B11F0020F9BB2F8D0FF239F
:10BEE800137302F10C0540F2E93300E07BB11189CC
:10BEF800013B11F0010F9BB2F8D02C78E4B24368F3
:10BF080013B11A689B889361204630BC7047184962
:10BF18008A4203D0174B9A42F1D10123164A02EB09
:10BF280003135A89013292B25A815B89E7E71049B3
:10BF38008A4203D00F4B9A42C6D101230E4901EB26
:10BF480003135989013189B259815B89BCE70849D2
:10BF58008A4203D0074B9A42B5D10123064A02EB25
:10BF680003135A89013292B25A815B890268ABE79E
:10BF780000300140003800402C9A0020F8B5050137
:10BF88005A4C5B4B625961199A4204EB050704BF8E
:10BF980001230B730646387A20F0E4FC3B7A03F061
:10BFA8001F015B090122022B02FA01F278D0032B50
:10BFB80071D0012B67D0631901361879FFF778F92A
:10BFC800F6B2074610B11223C67183716319587906
:10BFD800FFF76EF910B11323C6718371631998794D
:10BFE800FFF766F910B11423C671837166190E2123
:10BFF800F2793846FFF720FA7079FFF759F9F279A4
:10C008000E21FFF719FAB079FFF752F9F2790E21EC
:10C01800FFF712FA6359374A934251D0344A934290
:10C0280059D0354A934240D02C44227B002A2FD144
:10C03800012002249A8822F480521204120C9A8059
:10C04800998889B241F4805199801A8802F4415242
:10C0580042F44572024322431A809A8822F470629D
:10C068001204120C42F4E0629A809A8B22F4006265
:10C078001204120C07219A8319821A8892B242F08C
:10C0880040021A80F8BD1D4B996A0A439A6292E7EA
:10C0980000200446CEE7194B19690A431A618AE75A
:10C0A800164BD9680A43DA6085E702F5EA32116966
:10C0B80041F400411161116921F400411161B3E7B4
:10C0C80002F56042D16841F48051D160D16821F411
:10C0D8008051D160A8E702F5EC32116941F4804142
:10C0E8001161116921F4804111619DE72C9A0020AA
:10C0F8000038004000300140003C00400010024081
:10C10800427A02B9704710B504460368406804F1E2
:10C118000A0198470023637210BD00BF437A5A1C76
:10C128000344D2B242729972037A934200D802B998
:10C13800704710B504460368406804F10A0198473F
:10C148000023637210BD00BF30B40B4D002305F10E
:10C15800140101E0272B0BD011F8132082424FEA7B
:10C16800430403F10103F5D12C44607D30BC7047D2
:10C17800002030BC704700BFF01B03082DE9F341D5
:10C18800056906460F467DBBD0F80080C8F30A0350
:10C1980023B30023D6F80080019318F02FFC04285D
:10C1A80019D1224C236943F001032361BBB2A8F8DB
:10C1B800003018F023FC04282ED108F10203019363
:10C1C800019B3F0C1F8018F019FC2369042823F0F9
:10C1D8000103236125D06FF0010505E018F00EFC7E
:10C1E800042805D04FF0FF35284602B0BDE8F0819D
:10C1F8000E4C236943F002032361C4F814802369B9
:10C2080043F04003236118F0F9FB2369042823F065
:10C2180002032361BDD0E5E7236923F0010323610D
:10C22800D9E7336804333360DEE700BF00200240FB
:10C23800F8B504460D468E180027B54201D120698D
:10C24800F8BDE368591CE160234415F8012B1A7204
:10C258000429F2D1A1682046FFF790FFE76020612A
:10C26800EBE770B5448806460D46C4F30B04224636
:10C278000021284625F0D1FA33690A4A934209D3A6
:10C28800094A934206D2224628461946BDE870401C
:10C2980022F0ACBF23B121462846BDE870401847BC
:10C2A80070BD00BFB07C0308547D0308064B0749E6
:10C2B8008B4202D30023184670471A88C2F30B0238
:10C2C8009042F8D01433F3E7A0780308B07C030851
:10C2D800024A136823EA0000106070478436002081
:10C2E8002DE9F04F2DED028B8FB0064612F066FA5D
:10C2F8009C4B1F7827B10FB0BDEC028BBDE8F08FC7
:10C30800DFF8C0B2DBF800305C05F4D5964B974DEA
:10C318001B78002B40F05C81954B1B78002B6BD071
:10C32800944C954AD4F86431F31A934201F2398057
:10C3380094F86C81B8F1000F31D1904F3868FEF74E
:10C34800A1FFC0B201280ED9022841F0B5838C4B59
:10C358001A78002A41F0A385D4F87021B21AB2F5F0
:10C368007A6F81F0A686D4F87431002B44D094F803
:10C378006C31BBB9834B1B689B7801211E3B0022A3
:10C388008B4284F86C1184F8802141F2E985386881
:10C398000221043012F00BF994F878310FE0D4F848
:10C3A80074314BB3D4F87C3140F6B732F31A934268
:10C3B80022D994F87831002B01F0B3826F4F013BFA
:10C3C800DBB284F87831002B01F04480D4F8741182
:10C3D80094F8802111F801EB94F88131C4F87411B4
:10C3E80072440133386884F88021714684F88131B9
:10C3F800FEF74CFFC4F87C61634B2F681B7853B180
:10C40800DFF8C481D8F8000028B1604B1B78013BE5
:10C41800012B41F22E805E4B1B7863B15D4F3B6868
:10C428004BB1544CD5F80090D4F8B832A9EB0303BB
:10C43800632B00F21B87584C2378022B01F05282A1
:10C44800DFF8888198F80030032B00F0EF87534B12
:10C458001B7873B1524F3B685BB1464CFEF7C2FC88
:10C46800D4F8C032009044F61F62C31A934200F217
:10C478007D814C4B1B78002B4BD14B4B1B7843B128
:10C488003C4CD4F8103403F5C333A0339E4280F0FB
:10C498004987464B1B78002B3FF42DAF354E444C53
:10C4A800444D06F231472068FEF7ECFE00283FF4C1
:10C4B80022AF2068FEF7DEFE2B7880465A1E33B185
:10C4C80020682A70FEF7DEFE0028F2D113E7032267
:10C4D8003946781E25F087F996F8303496F83124D5
:10C4E80086F8338483F47F4383F0FF039B1A1FFA93
:10C4F80088F89BB2B8EB132FD5D196F83224DBB26B
:10C508009A42D0D1781E11F065FF2B781844287014
:10C51800C9E7294C2278002A40F0E886154CD4F85F
:10C52800083403F5C333A0339E42A6D3234A94F8B4
:10C538000C34C4F80864D55CE90701F1B083AA0794
:10C5480001F16C836B0701F183821D4A94F80C3466
:10C558001178013393FBF1F201FB123384F80C34A8
:10C568008BE700BF6E5E0020BC410020009A0020CF
:10C57800C64100206C2400203F0D030060410020CC
:10C588002000002064410020C8410020D041002044
:10C59800D8410020789400207E2D0020E041002022
:10C5A800E44100204C4200205A420020EA41002089
:10C5B800F0410020F4410020B44100205442002002
:10C5C80059420020E87900202C410020E901002090
:10C5D8005C4C2A68D4F85C31D31A7C2B7FF69CAE6D
:10C5E80094F86031DFF87C919FED578AC4F85C219C
:10C5F800013384F860314FF02408404612F08AF87D
:10C60800524BF9EC016A1B8A07EE103AF8EEE66A1B
:10C61800B8EEC77A08F10108C6EE877A5FFA88F89B
:10C6280067EE887AFDEEE77ACDED007ABDF900A0D5
:10C638005FFA8AF012F044F8CAF3072012F040F8C3
:10C64800B8F1270FD9D1302012F064F8DFF818813B
:10C65800002012F035F8002012F032F8D8F8000067
:10C668005E21FEF713FE94F8603113F003092DD113
:10C67800D4F85C2141F288339A4201F2FE841420F6
:10C6880012F048F8324B334AB3F9043082FB0312F4
:10C698004FEAE379C9EBA2090FFA89F95FFA89F041
:10C6A80012F00EF8C9F3072012F00AF81C2012F055
:10C6B80031F8002012F004F8002012F001F85E2191
:10C6C800D8F80000FEF7E2FD94F8603113F007098E
:10C6D80001F05C83282B7FF41FAE00271720D5F8C4
:10C6E800009084F8607112F015F8384611F0E8FFF0
:10C6F800194B1A4CA3FB09239B0BA4FB03125209E9
:10C70800C2EB0212A3EB8203D8B211F0D9FF1820B2
:10C7180012F000F8124BA3FB09239B09A4FB031298
:10C728005209C2EB0212A3EB8203D8B211F0C8FF80
:10C73800384611F0C5FFD8F800005E21FEF7A6FDC7
:10C74800EAE500BF6C24002000007A4484780020C9
:10C75800983D00206766666673B2E74589888888D1
:10C76800D34D6210B87800206841002094F8C63292
:10C77800002B41F04B81E34B1A6802F00803002BB1
:10C7880048F603414AF60B404BF60F4349F6074873
:10C7980004BF0346884612F0040F4FF0190118BF72
:10C7A8009846920684F8C61203D548F4804848F0A3
:10C7B8002008D54B1A79C8F309010191002A41F0E4
:10C7C800DD845B79002B41F0B1849A4664204FF0F8
:10C7D800FF330A464FF00009CDF81880CDF81C80C9
:10C7E8000892ADF826A0ADF828308DF83600ADF8DF
:10C7F8002490CDF82A90CDF82E90CDF832900DF1F6
:10C80800180CBCE80F00DFF810E384F85190AEE88C
:10C818000F009CE80F00AEE807002EF8023B7146B7
:10C828004FF0010C1B0C4FF0FE0E1F20C82201F820
:10C838001E3984F84EE084F8522084F853C084F8F6
:10C848004F0094F8D60284F8500080F0F10383EA90
:10C858000313DAB2130983F0E70343EA022383EAF6
:10C86800C2031BB283EA0312D2B2C3F3072383EADB
:10C87800121343EA022383EAC2031BB283F0C802FD
:10C8880082EA0212D2B2C3F3072383EA121343EAFD
:10C89800022383EAC2031BB283EA0C0E8EEA0E1E41
:10C8A8005FFA8EFEC3F3072282EA1E1242EA0E22C4
:10C8B800604482EACE0E84F8D602A4F84CE001F176
:10C8C8001F0011F8013B83EA0E0383EA0313DBB26E
:10C8D8001A0982EA1E2242EA032282EAC3031BB231
:10C8E8001FFA83FE8142A4F84CE0EAD183F07C036E
:10C8F80083EA0313DBB21A0982EA1E2E8EEA032E9C
:10C908008EEAC30E0FFA8EFE1FFA8EF34FEA132A31
:10C918005FFA8EFEA4F84C30DFF8009284F874A019
:10C9280004F16E0384F873E004F14E0C0193DCF813
:10C938000C30DCF80000DCF80410DCF80820C846ED
:10C94800A8E80F00019B0CF1100C9C45C146EED1E4
:10C95800DCF80000C8F80000DFF8C4819CF8043057
:10C9680089F8043008F1270984F825E384F826A318
:10C9780018F8011F3868FEF789FCC145F8D194F80A
:10C98800C722002A41F0478060492B6808780A21AD
:10C9980084F8C712002801F03781DFF888C1012820
:10C9A800BCF80010059141F25985BCF802100291BB
:10C9B800022801F0FF83BCF804100391032801F05A
:10C9C8003385BCF806100191042801F02785052855
:10C9D800BCF8081001F01D850628BCF80AA001F073
:10C9E80014850728BCF80CE001F00085BCF80E900F
:10C9F80094F8D6220693104680F0300383EA031396
:10CA0800DBB20490424A9DF810C0128884F850C0E6
:10CA1800180980F07A0040EA032080EAC3033D4801
:10CA2800C2EB022280FB02C01044D217C2EB602284
:10CA380005988DF82D204FF0000860F30F08039833
:10CA48004FF0000C60F30F0C00201BB261F30F00D5
:10CA580000216EF30F0183EA031EC3F30723039338
:10CA6800029B63F31F48019BCDF81C8063F31F4CA6
:10CA7800039BCDF820C05FFA8EFE6AF31F4069F36E
:10CA88001F4183EA1E134FF0000A09900A918DF89E
:10CA98002CA043EA0E2C0DF11809B9E80F008CEA16
:10CAA800CE0E0FFA8EFE8EF0C808DFF86CC084F840
:10CAB80051A088EA08185FFA88F8CEF3072EACE888
:10CAC8000F008EEA181E4EEA082399E8030083EA4D
:10CAD800C8080FFA88F383F023024CF8040B82EAA3
:10CAE8000210C0B2C3F3072282EA1012049B2CF88A
:10CAF800141942EA0022591C82EAC0004FF02308A8
:10CB0800162211E03C4E0020D05B0020742C00203F
:10CB1800C85B002003082080C02400206C27002068
:10CB28006B270020445E00204FF0FE0EC82384F8D7
:10CB3800D612A4F84C000CEB020184F8538084F858
:10CB48004EE084F84F2084F852301CF8013B4340F3
:10CB580083EA0313DBB21A0982EA102242EA0322AB
:10CB680082EAC3031BB298B28C45A4F84C00ECD1FE
:10CB780083F0F40383EA0313DBB24FEA131E8EEA51
:10CB8800102E8EEA032E8EEAC30EA0460FFA8EFEF2
:10CB98001FFA8EF958F84E0FDFF81CC4A4F84C9011
:10CBA8004FEA192A5FFA8EFE84F86AE084F86BA0CF
:10CBB800D8F80410D8F80820D8F80C30ACE80F00E2
:10CBC800D8F81000D8F81410D8F8182004F21D3935
:10CBD800ACE8070004F2FF2884F81DA384F81CE3DE
:10CBE80018F8011F3868FEF751FBC145F8D194F8D1
:10CBF800CEE2BEF1000F40F01787E84B94F8D6C29A
:10CC0800B3F90010B3F90220B3F904309FEDE46AD8
:10CC180084F851E007EE103A2B6806938CF06A030B
:10CC280083EA031306EE901AD9B20B0983F0D503F1
:10CC380043EA012383EAC1031BB283EA0311524288
:10CC4800C9B207EE902AC3F3072383EA111343EA14
:10CC58000123F8EEE77AF8EEE66AB8EEC77A83EAD7
:10CC6800C1031BB267EE867A66EE866A27EE067AFD
:10CC7800002083F0C805CDED087ACDED076A8DED6B
:10CC8800097A0A900B900C9085EA05150DF11809A0
:10CC9800EDB2C3F30728B9E80F0088EA151848EA87
:10CCA800052888EAC505DFF814832DB2A8E80F0027
:10CCB80085F01E0E99E807008EEA0E13DBB2C5F365
:10CCC800072E8EEA131E4EEA032E88E807008EEA26
:10CCD800C30EA8F110051C20C8214FF005091E231A
:10CCE8004FF0FE080CF1010284F8521084F8CE923D
:10CCF80084F8533084F84E8084F84F00291884F85B
:10CD080050C0A4F84CE084F8D62215F8013B83EA19
:10CD18000E0383EA0313DBB21A0982EA1E2242EAEF
:10CD2800032282EAC3031BB21FFA83FE8D42A4F8D2
:10CD38004CE0EAD183F0270383EA0313DBB21A0934
:10CD480082EA1E2E8EEA032E8EEAC30E0FFA8EFE9C
:10CD58001FFA8EF34FEA13295FFA8EFEDFF8588226
:10CD6800A4F84C3084F8719084F870E004F14E0C0B
:10CD780004F16E0ADCF80000DCF80410DCF8082086
:10CD8800DCF80C3045460FC50CF1100CD445A8460C
:10CD9800F0D1844DBCF80030A8F8003005F1240823
:10CDA80084F822E384F8239315F8011F3868FEF706
:10CDB8006DFA4545F8D194F8CF320193002B40F035
:10CDC8002F8694F8D682754B774AB3F90410B2F9D6
:10CDD8000620DFF8ECC1754DDFF8E09184F850804B
:10CDE80088F0220383EA0313DBB2180980F05900A4
:10CDF800B2F5FA6F40EA032080EAC303A8BF4FF4F4
:10CE0800FA621BB2B2F57A7F83EA0310B8BF4FF417
:10CE18007A72C0B24FF0640EA2F57A72C3F3072398
:10CE28000EFB02F283EA101385FB02E543EA0023B6
:10CE38008CFB01CED217C9174FF0000AC2EBA5121E
:10CE4800C1EBAE0183EAC0031DB2CDF818A00DF105
:10CE5800180CADF82A20ADF82810CDF81CA0CDF894
:10CE680020A0CDF824A085F0C80ECDF808C0BCE8F5
:10CE78000F008EEA0E1E5FFA8EFEC5F3072585EABF
:10CE88001E1545EA0E25A9E80F0085EACE0212B262
:10CE980082F04A0383EA0313DBB2C2F3072181EA73
:10CEA8001311DCF8002049F8102941EA0321052074
:10CEB80081EAC303142508F101029DF8041084F8DF
:10CEC800CF024FF04A0C4FF0FE0EC82084F85110E4
:10CED80084F8D62209EB050184F84F50A4F84C30A9
:10CEE8004A4684F853C084F84EE084F852001D4640
:10CEF80012F8010B684080EA0010C0B2030983EA07
:10CF0800152343EA002383EAC00000B285B28A42AF
:10CF1800A4F84C50ECD180F0140080EA0010C0B2A4
:10CF28004FEA101E8EEA152E8EEA002E8EEAC00EEB
:10CF380025460FFA8EFE1FFA8EF855F84E0FDFF8C9
:10CF480078C0A4F84C804FEA182A5FFA8EFE84F85D
:10CF580069A084F868E06968EB68AA68ACE80F0023
:10CF6800286969692B8BACE8030004F2FF25ACF84B
:10CF78000030A84684F81BA384F81AE304F21B3A8D
:10CF880018F8011F3868FEF781F9C245F8D1084B37
:10CF9800084A1B781278013B14E000BF983D002036
:10CFA80088C3E43A6B270020445E0020D34D62100A
:10CFB80034330020173C00206C270020C0240020B8
:10CFC8006766666612F00100DBB214BFC022402219
:10CFD800172B04D8CA490B4493F824300193C94B42
:10CFE80019888B071ABF002342F01002012311F49D
:10CFF800027F18BF022311F0100F18BF062311F08B
:10D00800200F18BF1023002841F04B80032194F80B
:10D01800D6E206938EF0460383EA0313D8B20309D7
:10D0280083F0920343EA002383EAC0031BB283EA36
:10D038000310C0B2C3F3072888EA101848EA00288A
:10D0480088EAC0080FFA88F888F0C80C9DF8040030
:10D058008DF81C008CEA0C1C00235FFA8CFC8DF800
:10D068001E200320029A8DF81D30C8F307288DF87A
:10D078001F108DF8200088EA1C1807CA48EA0C28F7
:10D0880088EACC0C0FFA8CFC8CEA0C18A9E803008F
:10D098005FFA88F8CCF3072181EA181141EA0821E0
:10D0A80081EAC80894F854C089F800200FFA88F279
:10D0B8008CEA020C8CEA0C1C5FFA8CFCC2F3072287
:10D0C80082EA1C1242EA0C2294F8550094F8561091
:10D0D80094F8579094F8588084F8533082EACC0238
:10D0E80012B2504080EA0010C0B2C2F3072282EAAE
:10D0F800101242EA002282EAC00212B2514081EACA
:10D108000111C9B2C2F3072282EA111242EA0122CE
:10D1180082EAC10212B289EA020989EA09195FFAA8
:10D1280089F9C2F3072282EA191242EA092282EA3D
:10D13800C90212B288EA020888EA08185FFA88F871
:10D14800C2F3072282EA181242EA082294F859C068
:10D1580094F85A0094F85B1094F85C9084F8513075
:10D1680082EAC80212B28CEA020C8CEA0C1C5FFA42
:10D178008CFCC2F3072282EA1C1242EA0C2282EAE1
:10D18800CC0212B2504080EA0010C0B2C2F30722AB
:10D1980082EA101242EA002282EAC00212B2514028
:10D1A80081EA0111C9B2C2F3072282EA111242EAE6
:10D1B800012282EAC10213B289EA030282EA021258
:10D1C800D2B2C3F3072383EA121343EA022383EAA2
:10D1D800C2031BB283F0320282EA0212D2B2C3F354
:10D1E800072383EA121343EA022383EAC2031BB22A
:10D1F8009AB24FF0FE0CDFF8208184F850E0092045
:10D20800C8210EF1010EDBB284F84EC04FEA122C91
:10D2180084F84F0084F8521084F8D6E2A4F84C2021
:10D2280084F85EC084F85D30D8F80000D8F804109F
:10D23800D8F80820B8F80CA008F2B22EAEE807001B
:10D2480008F2C2288EF80290AEF800A084F810C345
:10D2580084F80F3315F8011F3868FEF717F8A8454A
:10D26800F8D1009BC4F8C032FFF703B9DFF8ACA0CF
:10D27800DFF8AC80412011F04DF9BAF9023088FB93
:10D288000320DB17C3EBA00080B211F029F9BAF92B
:10D29800003088FB0320DB17C3EBA00080B211F03D
:10D2A8001FF9BAF9043088FB0320DB17C3EBA00091
:10D2B80080B211F015F9144B38681978FDF7E6FFBC
:10D2C80094F8BC3213F0010800F0FD830F4AC4F84B
:10D2D800B8920133DBB2A2FB0312D20802EB82023E
:10D2E800A3EB420384F8BC32FFF7A5B8084B094901
:10D2F8001868FDF79BFF00232370FFF70FB900BFE5
:10D30800541C03086C5E002080990020CDCCCCCC46
:10D318005042002090410020BA240020983D00206F
:10D328006766666694F81434BA4AC4F8106402EB67
:10D338008302D26B42B30EAD04F21B43B64E45F8DE
:10D34800203D002104F22D433180079380211523CD
:10D35800A52784F81A34284684F8191484F8187410
:10D36800904728463188F3F7D9FD069DAB4804F568
:10D3780083616D1A152DA8BF15252A4621F036FFA1
:10D38800A74A94F814341570A64A013382FB031295
:10D39800A2EBE37202EB42029B1A84F81434FFF703
:10D3A80078B8A14BA14AD4F868112868128893F874
:10D3B8000BE09F4B401A4FF47A71D7B201FB0EF184
:10D3C800120A9F771F7588424FF00007DA775A755F
:10D3D8009F701F7180F02E83964A97481168926853
:10D3E800C4F8646180FB01E7C91780FB02E0C1EB68
:10D3F800A701D217C2EBA00208124FEA222C4FF065
:10D40800F40E19770127587783F8202030207521EA
:10D41800782283F821C083F81AE0DF7683F82200A7
:10D4280083F8231083F82420FEF782BF834F3868DF
:10D4380003685B69984700283FF409A838680368BF
:10D4480001219B6998470222002388F80020237055
:10D45800FEF7FDBF94F8801194F8813138684A1CB2
:10D46800013384F8802184F88131FDF70FFFFEF73E
:10D47800C1BF734CDFF8D0914FF0000A0BE01B2BB3
:10D4880000F043820D2B00F00C824FF0010389F865
:10D498000130D8F80000FDF7F5FE002837D0D8F89D
:10D4A8000000FDF7E7FE83B27E2B2A6828D099F8A2
:10D4B8000120002AEDD194F882110029DFD07D2BBC
:10D4C80000F0038294F886E1BEF1000F04D080F0EA
:10D4D8002003DBB284F886214A1CD2B2092A63549D
:10D4E80084F8822100F0E581082AD2D8B4F8842192
:10D4F800134403EB132303F0FF03A4F88431C8E7B4
:10D5080084F882A184F883A189F801A0C1E794F87E
:10D5180087312BB1637884F88701302B00F03E8582
:10D5280094F883213B4BDFF82491DFF824C1DFF81E
:10D5380024A14FF0010E002A3EF46DAF2968C91BE3
:10D54800012900F2A98194F89C82B8F1000F40F0FB
:10D55800F38194F8B41233F8110010B984F8B4E2E6
:10D56800E9E70131B0F5826F84F8B41200F0188150
:10D578001ED9B0F5E26F00F0BC8033D9B0F5046F66
:10D5880000F0C580B0F5116F00F0CD80B0F5E46F04
:10D59800D1D12C4AD76B118A642303FB07F393FB81
:10D5A800F1F110F0EAFF002384F88331FEF733BF6E
:10D5B800B0F5007F00F0D1804ED8B0F5807F00F044
:10D5C8004281B0F5887FB6D1D9F800104907B2D5A5
:10D5D80000214FF4887010F0D0FF002384F88331C5
:10D5E800FEF719BFB0F5C06F00F0CA80B0F5E06F64
:10D5F800A1D1144A506B118A642303FB00F34FF442
:10D60800E06093FBF1F110F0B8FF002384F8833158
:10D61800FEF701BF541C030816410020642F0020A8
:10D62800792F0020565555553041002018410020CB
:10D63800F84100201C410020676666661C2E002009
:10D648006C24002084780020200000203C4E00201C
:10D65800D05B00204F410020B0F5047F00F002812C
:10D66800B0F5806F7FF467AF94F8B5320133DBB261
:10D67800032B00F22F8142F2107184F8B53201FBBE
:10D6880003F1BD4B1B88002B40F02A810131BB4BB5
:10D698001B78D807BA4B1B8848BF0431DA0748BF44
:10D6A8000A31980748BF14311A0648BF2831D805EF
:10D6B80048BF28315A0748BF6431180748BFC831E6
:10D6C8009A0548BF01F5C871980648BF01F57A71F7
:10D6D800DA0648BF01F5FA61580648BF01F57A61D4
:10D6E8004FF4806010F049FF002384F88331FEF77F
:10D6F80092BEA44A976B118A642303FB07F393FB3A
:10D70800F1F110F03AFF84F88381FEF784BE9E4B56
:10D71800B3F9041001EB8101490010F02EFF84F8E1
:10D728008381FEF778BE9CF8041000293FF403AF0C
:10D738009AF8001000293FF4FEAE944B1B8803EBC7
:10D7480083035B004FF4116093FBF1F110F015FFB8
:10D75800002384F88331FEF75EBE9CF8051000298B
:10D768003FF4E9AE8A4B8B491B6881FB0321DB1729
:10D77800C3EBA10110F001FF84F88381FEF74BBED3
:10D788009CF8051000293FF4D6AE814B4FF4C060D9
:10D79800996810F0F2FE002384F88331FEF73BBE4F
:10D7A800D9F8001011F020087FF4C5AEDBF800109E
:10D7B800090600F1DD837849097B00293FF4BBAEF7
:10D7C80094F8B612032900F2B585DFE801F0322893
:10D7D8001902724B1B6859799A79DB7901F140710A
:10D7E80001EB022101EB0341002384F8B6324FF428
:10D7F800826010F0C2FE002384F88331FEF70BBE6E
:10D80800674B1A68137A507992781B0403EB00234C
:10D8180013444A1C84F8B62203EB0161E7E7604B26
:10D828001A68D379107952781B0403EB0023134448
:10D83800EFE75B4B1A689379D07812781B0403EBF7
:10D8480000231344E5E7D9F8001048077FF573AEC5
:10D8580000214FF4807010F090FE002384F883318B
:10D86800FEF7D9BD9CF8041000293FF464AE9AF87D
:10D87800000000283FF45FAE474B5B7B002B00F0B5
:10D88800F983424B198891FBF0F101EB81014900C2
:10D898004FF4047010F071FE002384F88331FEF712
:10D8A800BABD4FF0010284F882212370A4F88411D4
:10D8B800EFE5B4F88421C2F1FF0293427FF4E5ADAD
:10D8C8004FF0010384F88731DFE54FF0010384F856
:10D8D8008631DEE5012384F8B53242F21071D0E6D4
:10D8E8000231D4E6FDF77EFA2E4B1A6840F6B833BB
:10D8F800801A984200F27E812B4F3B793A2B00F038
:10D90800D48200232370FEF7A2BDD8F80000FDF7EB
:10D91800B9FC00287FF4B9AD4FF0010384F88331D6
:10D92800B7E5C4F8743184F86C31204F10F072FEFA
:10D9380094F87831FEF743BDD4F88C32DFF8709054
:10D9480094F8B2224B4500F0D183511C94F8B3E20D
:10D95800D4F890C284F8B21202F00F028DF81820A1
:10D968000DF11902ACEB0301002940F3EE8406A97E
:10D9780002910DF11E0720E0005C0020173C0020FA
:10D988006C5E002084780020983D0020184100201B
:10D998001C4100206766666630410020E09A00203E
:10D9A800C8340020842D00206C2D00206041002008
:10D9B800F8250020002840F31A810133C4F88C327E
:10D9C80013F8011C02F8011BBA42ACEB030081EA10
:10D9D8000E0EEFD384F8B3E200F0A684501CB842D0
:10D9E80082F800E005D20EAB9A1A1B3A002123F008
:10D9F80014FF0299322010F0A5FD4FF00008002313
:10DA080084F89C8284F88331FEF705BD013B84F8D5
:10DA1800C632FEF7B4BF013A84F8C722FFF7E7B869
:10DA2800013B84F8CF321CE40EF1FF3E84F8CEE2CD
:10DA3800FFF7C1B9C04A29681278C4F86811013AD9
:10DA4800012A3FF6C9AC1021022299701A71C3E469
:10DA5800BA4ABB4B12680793A3F12408002021217E
:10DA6800D50003F8240C88F8021040F1F782B54974
:10DA78000327B54B1B88580500F1ED82DA0700F142
:10DA8800968303F00203B14A002B1CBF03271146FB
:10DA9800AF4D3A46284621F0A9FB7B190EA8013361
:10DAA800A91E40F8203D00225B1A7A5588F80130FB
:10DAB80010F042FEFEF749BD10F09CFDA54B012277
:10DAC8001A70FEF750BCA04B1B88DA0515D4D8068F
:10DAD80000F17883990600F111845A0600F13B841D
:10DAE800180700F16A84D90700F17C8413F0020F4B
:10DAF8000CBF4FF004084FF00C08974B974A1B785F
:10DB0800D27803F001030AB143F0020353200093D3
:10DB180010F000FD924A128802EB820202EB8202A8
:10DB2800900080B210F0DCFC002010F0D9FC8D4A87
:10DB38008D4912883868C2EBC212520081FB02314B
:10DB480011444FEAE27ACAEB612A5FFA8AFA51462F
:10DB5800FDF79CFB854B38681A78009B48EA030858
:10DB6800824B8AEA020A002183F800A0FDF78EFBA7
:10DB780041463868FDF78AFB7C4B7C4A1B7838683D
:10DB880088EA0303DBB219461370FDF77FFB94F8AC
:10DB9800BC32002B7FF49AAB4F2010F0BBFC1DF079
:10DBA80061F91DF05FF91DF05DF901213868FDF795
:10DBB8006DFB6F4A6D4B92F800801B786B4A386892
:10DBC80008F00108414683F001031370FDF75EFB7E
:10DBD800664B38681B7888EA0308644B414683F82B
:10DBE8000080FDF753FB94F8BC32FFF76FBB84F855
:10DBF800B3E2F3E65F4AB2F8BE3200210133A2F87D
:10DC0800BE322170FEF723BC86468246014601904B
:10DC18000390029005908146FEF7EABE484B5049B2
:10DC280007930EAFA3F1210047F8200D4FF0080E1F
:10DC38004FF000080A2003F822EC03F8230C03F83D
:10DC4800248C38460988F3F743F94B4B4B491B683A
:10DC580081FB0321DB17C3EBA101384689B2F3F737
:10DC680037F9474BB3F8069012F0C6FB069B5A1CCF
:10DC7800069283F80080069B4FEA1922591C0691E8
:10DC88001A70069B5A1C069283F80090069B5A1C31
:10DC980006921870384610F04FFDFEF753BCDFF8B7
:10DCA800E8809FED388AB8F90230254A079207EED6
:10DCB800903AF8EEE77A0EAF67EE887AA2F124037D
:10DCC800FDEEE77AA2F12101002047F8201D02F8B5
:10DCD800240C0822CDED007A5A701E229A70BDF8E5
:10DCE80000103846F3F7F4F8B8F9003007EE903A28
:10DCF800F8EEE77A384667EE887AFDEEE77ACDEDFA
:10DD0800007ABDF80010F3F7E3F8B8F9043007EE2D
:10DD1800903AF8EEE77A384667EE887AFDEEE77AC9
:10DD2800CDED007ABDF80010F3F7D2F8384610F0C0
:10DD380003FDFEF704BC00BFCB5B00206830002069
:10DD480090410020EC4003086C5E0020004103086D
:10DD58006F41002020000020173C0020DC5B0020E1
:10DD680018410020C85B002003082080809900200B
:10DD7800703000206C2400201C4100206766666615
:10DD8800D05B002058A08B41983D0020022010F065
:10DD9800C1FCFF2010F0A6FA0378FF2B00F0B28236
:10DDA80090F901004FEAE0795FFA89F9C0B210F002
:10DDB80087FC484610F084FC032010F0ABFCFF20E1
:10DDC80010F090FA0378DFF89C93FF2B1BBFB0F993
:10DDD80008A05FFA8AF74FF0000ACAF3072A384604
:10DDE80010F06EFC504610F06BFC99F80430002BD4
:10DDF80040F0EB810DF118094946D04810F024FC99
:10DE0800132010F087FCBDF91870F8B210F058FC18
:10DE1800C7F3072010F054FC1B2010F07BFCBDF961
:10DE28001A70F8B210F04CFCC7F3072010F048FC49
:10DE3800232010F06FFC4E2010F042FC002010F060
:10DE48003FFC4946BD4810F0FFFB122010F062FC71
:10DE5800BDF91870F8B210F033FCC7F3072010F0C2
:10DE68002FFC1A2010F056FCBDF91A70F8B210F009
:10DE780027FCC7F3072010F023FC222010F04AFCEF
:10DE8800452010F01DFC002010F01AFC5E21D8F887
:10DE98000000FDF7FBF994F86031FEF71BBCC4F8ED
:10DEA800706183F80080FEF75EBABB78DBB103F1DE
:10DEB800FF3C5FFA8CFC0CF1010CBC44BE4600220E
:10DEC8001EF8013B534083EA0313DBB2120AD90060
:10DED80042EA0322F44581EA131382EA0302EFD1EE
:10DEE800002A7FF40EAD964B964ADFF87CE219685B
:10DEF800954B1288DFF87482D1F830C0CEF818201C
:10DF08001A68B8F8BE829B68CEF828200022CEF89E
:10DF18006800CEF84830CEF83820CEF85880BCF1EA
:10DF2800000F00F05682DCF80430086C83423BBFD7
:10DF3800CA681B1A1B1A9B18002B7EF481AA0B684F
:10DF4800DFF82C829B690846022198470423F87859
:10DF580088F8003007F0AEFF03232370FEF772BA8B
:10DF680002213868FDF782F994F87831FEF727BA6C
:10DF780010230422184606A98DF81A808DF81B80F4
:10DF88008DF81C808DF81D808DF818308DF81920BB
:10DF980010F0D8FA84F88381FEF73DBAA3785A09BD
:10DFA800012A40F0998103F00F0C13F0100300F0E0
:10DFB800AB81DFF8C081E37894F804E0A4F8AA0202
:10DFC80008EB03018EEA030084F888214346C4F86D
:10DFD800A082C4F8A412A8F1070284F8B002A4F839
:10DFE800A8E294F8B002DFF8908186460CE012F8B7
:10DFF800011BC4F8A002424581EA0E0E197007D22F
:10E00800D4F8A412D4F8A032994203F10100EED159
:10E01800424584F8B0E200F0EC81127894F8B0320E
:10E028009A4200F09C81494BC4F88C32002201339B
:10E03800B4F8A812C4F8903284F8882101234FF666
:10E04800F672A4F8941284F88C3184F89C32A4F8FF
:10E058009622FFF765BA03273D4919E5DBF800303A
:10E068003C4A3D4903F48003834216BF1146042706
:10E078000327FEE4334B198807E4102010F04AFB0D
:10E08800484610F01DFB484610F01AFB212010F0FE
:10E0980041FB484610F014FB484610F011FBFEF710
:10E0A800EEBA2E49C97800290CBF04210521FEF7D4
:10E0B800AEBF012238681A70FDF7DCF88046386870
:10E0C800FDF7D8F818F07F0F7EF44DA98E287EF45E
:10E0D8004AA994F86C31002B7EF461A9204BC4F84E
:10E0E80074312D2384F87831FEF744B9B4F99612C7
:10E0F800D4F890C294F894E2501C02F00F0242F057
:10E1080010020029B8BF42F020028DF81820ACEBAD
:10E11800090282EA0E0E5FFA8EFE8DF8192084F845
:10E12800B20284F8B3E20DF11A021BE4064B9246E0
:10E13800B3F9003064200A46FEF74CBB809698007D
:10E148001C2E0020184100201C410020F82500202A
:10E15800AC440308EC400308E4400308DC5B0020FF
:10E16800F8410020D05B0020780100206C240020BA
:10E17800E90100207824002074240020BC495A7941
:10E188000B8803EB830303EB83034FEA830A1FFA2D
:10E198008AFA002A40F05F814FF0FF331BB20293E6
:10E1A80012F02AF9029B019A40B2FEF713BBB1495B
:10E1B80004276DE4964692461146019203929146D1
:10E1C800FEF716BC4FF0340897E4DFF8C4A29AF8BB
:10E1D8000020002A3FF40EAEB4F86271A44B0092FE
:10E1E8001B883F016421BFB201FB03235100B3FB2D
:10E1F800F1F347EA0327BFB2C3F303231F43062003
:10E2080010F088FAF8B210F05BFA380A10F058FAF1
:10E21800B4F86231964A98491788009A01339BB23C
:10E2280093FBF2F002FB1033487AA4F8623101281C
:10E2380000F007814B7B6E2202FB07F7152297FB44
:10E24800F2F7002B40F0F7803A2010F063FABFB2E3
:10E258004FF0640AB7FBFAF293B2D8B20192009376
:10E2680010F02EFA009B180A10F02AFA3B2010F042
:10E2780051FA019A0AFB127080B20A23053090FB0A
:10E28800F3F0C0B210F01CFA002010F019FADFF811
:10E29800FCA1282010F03EFA0A23DAF8007097FB58
:10E2A800F3F7F8B210F00CFAC7F3072010F008FAE9
:10E2B800042010F02FFAB9F80630002B40F08180C6
:10E2C800DAF8087087F31007F8B210F0F9F9C7F315
:10E2D800072010F0F5F98DE5684B694AC4F88C32CF
:10E2E800591C012384F8880184F88C01C4F8901221
:10E2F800C4F8942284F89C32FFF712B94FF024082E
:10E30800FFF7FBBB484652E594F88821002A3FF402
:10E3180007A994F8B122013202F00F02624546D0F3
:10E3280084F88831FFF7FCB80299322010F00AF916
:10E33800FFF765BB4B1CDBB2042B84F8B6324FEAFF
:10E3480001617FF454AAFFF74FBA06AB02930DF1AF
:10E358001E07FFF743BB4FF01008FFF7CEBB494B32
:10E36800D4F8A022C4F8A4224FF0000E03F52072BE
:10E37800114603F5C079C4F8902203F5257072465A
:10E38800C4F8A032C4F894E2C4F88C9284F888E106
:10E39800F5F73AF8013030D0D4F88C32C4F890321E
:10E3A8000123C4F88C9284F89C32FFF7B9B8D4F8EA
:10E3B800A412D4F8A032344A13E64FF02008FFF72D
:10E3C8009CBB12F019F810F07BF9002010F078F9D6
:10E3D80010E5C8690B6A98423BBFCA681218C31A8D
:10E3E800D31AA9E54FF00808FFF787BB9146FEF757
:10E3F800FFBA84F8B1C2FFF793B8D4F88C3202227E
:10E40800591CC4F88C121A70C6E796469146FEF756
:10E41800EFBA964692469146FEF7EABA9646924673
:10E4280011469146FEF7E4BA964692461146019285
:10E438009146FEF7DDBABFB29AF8003097FBF3F7C2
:10E4480002E7392010F066F9F8B210F039F9380A05
:10E4580010F036F91BE70D4B1B689FE6964692466F
:10E4680011460192039202929146FEF7C1BA00BF8B
:10E4780018410020F840030830410020F82500200A
:10E488000000F6FF782400206F2400201C410020A3
:10E498004F41002003680A7A591C01601A707047BE
:10E4A80038B50B4C23688BB15A68821A002A054686
:10E4B80004DA0CE05A68AA1A002A07DB9A68226074
:10E4C80018461A6890472368002BF3D138BD38BD29
:10E4D800783100200B4B002210B4027203F1B4040F
:10E4E800012102E0072A09DC9979890702D51979FF
:10E4F800815401329C4203F11403F3D15DF8044BBB
:10E50800704700BFD83F030827230370704700BF38
:10E51800012310B415211424222244704171C270C1
:10E528000370037183705DF8044B704708B519F0E8
:10E53800D5FA024B024ADA60FEE700BF00ED00E0C0
:10E548000400FA0570B54E680546304620F04EF8CE
:10E55800314604460246286820F048FE2A68131906
:10E5680001333B212B60115570BD00BF024A034B9C
:10E57800127819780CF022B8642200206522002055
:10E588002DE9F0470569C3681D4028D00F460646A7
:10E598004FF000484FF00009B5FA85F328FA03F266
:10E5A800D2431B3B32611540042B16D8DFE803F039
:10E5B8003129211903007B6A002B32D003F1FF3A7D
:10E5C8001FFA8AFAC7F824903C6A34B123682046B7
:10E5D800514698476468002CF8D1002DDCD1BDE87D
:10E5E800F0873868716B036889B29847002DD3D1DA
:10E5F800F5E77868B16B036889B29847002DCBD1ED
:10E60800EDE7B868F16B036889B29847002DC3D16C
:10E61800E5E7F868316C036889B29847002DBBD1EB
:10E62800DDE7F36A1FFA83FACEE700BF38282DE941
:10E63800F04700F072820C462ED9802800F0E38063
:10E6480074D8522800F0898040F23681542800F0AE
:10E6580013826E2840F08782B74B0A681B88B74D33
:10E66800FF2BA8BFFF23511C21601370A96881F3F9
:10E678001001204689B2F2F751FCB14B20461988A7
:10E68800F2F74CFC296801F30F01204689B2F2F732
:10E6980045FC0120BDE8F087042800F0DC8140F249
:10E6A800DA80202800F08E8040F20F81242800F0C4
:10E6B8002181282840F057820B68DFF8BC82A14EE0
:10E6C800591C022221601A70236806275A1C2260EE
:10E6D8001F7023680A22591C21601A7023680125BB
:10E6E8005A1922601D70B8F800102046F2F716FC7F
:10E6F800B8F802102046F2F711FC23685A19226074
:10E708001F7023685022591921601A70236800224B
:10E71800591921601A7031882046F2F7FFFB20460C
:10E728007188F2F7FBFB2846BDE8F08782281CD0E9
:10E73800C0F03A81A02800F02581FE2840F013821D
:10E74800814D05F1080635F8021B2046F2F7E6FB75
:10E75800B542F8D10120BDE8F0870B680022591CAA
:10E7680021601A700120BDE8F0870B68774A734D65
:10E778001178774A581C20601970D1882046F2F722
:10E78800CDFB6D4B22681B88FF2B02F10101A8BF4E
:10E79800FF2321601370A96881F31001204689B214
:10E7A800F2F7BCFB296801F30F01204689B2F2F7A2
:10E7B800B5FB2368674A591C127821601A7001203A
:10E7C800BDE8F0870B68624D591C6A7821601A70A1
:10E7D80023682A78591C21601A702368AA78591C62
:10E7E80021601A70E9882046F2F798FB23682A7995
:10E7F800591C21601A7023686A79591C21601A70A3
:10E808000120BDE8F087DFF87481534F534EDFF8DD
:10E8180070A108F10D090A2514E0322D31D0A5F1B7
:10E828003C00C0B2132832D900232268511C216051
:10E8380015702268C14502F101012160137089D069
:10E8480018F8015B0A2DE8D1BAF80030FF2BA8BFF1
:10E85800FF23DBB2E9E7022865D053D8012840F04E
:10E8680082810B680022591C21601A7023685A1C87
:10E878002260187023682422591C21601A70BDE890
:10E88800F0873388FF2BA8BFFF23DBB2CDE70FF05B
:10E8980029FD0028C8D003780A2B00F26781B0F957
:10E8A800023087FB0312DB17C3EBA2039BB2FF2BDB
:10E8B800A8BFFF23DBB2B8E7442840F05481002A00
:10E8C8003FF448AF264B136044E7052840F04B81DE
:10E8D80020460B222349F2F7F1FA20460822224962
:10E8E800F2F7ECFA204607222049F2F7E7FA01206E
:10E8F800BDE8F0871E4B08461968F2F7F7FA0120C1
:10E90800BDE8F0870B680222591C21601A70236841
:10E9180001201A1822601870236800221918216033
:10E928001A70BDE8F087084604221249F2F7C6FAC1
:10E938000120BDE8F08700BF184100201C410020DD
:10E94800C85B0020B8440020844000204F410020CC
:10E95800D05B0020CB5B002067666666D044002051
:10E9680035E50008C0440308CC440308D84403082C
:10E9780084360020B0440308D0780020B11C030876
:10E98800004500207A4B08461968F2F7AFFA794B30
:10E9980020461968F2F7AAFA774B20461968F2F769
:10E9A800A5FA0120BDE8F087DFF8F091734F09F16F
:10E9B8000E064FF00A081DE0B8F1500F32D0B8F13A
:10E9C800320F31D0A8F13C00C0B213282FD900254E
:10E9D800294623685A1C2260204683F80080F2F7F3
:10E9E8009DFA29462046F2F799FA4E453FF4B2AE11
:10E9F80019F8018BB8F10A0FDED1614B9D681968CF
:10EA080005EB85054FF6FF736D009D42A8BF1D46B7
:10EA18009942A8BF194625EAE57521EAE171ADB228
:10EA280089B2D6E7574BE9E797E82200E8E70FF005
:10EA380059FC0028CBD003780A2BC8D8B0F9043089
:10EA4800B0F9061003EB830383F3500521EAE17163
:10EA5800ADB289B2BDE702464B492046F2F72EFA1D
:10EA680020460021F2F75AFA23680222591C216035
:10EA78001A700120BDE8F0870B68444A444F581CBF
:10EA880011212060197023681278591C21601A70AE
:10EA9800236897F85C20591C21601A70236897F83E
:10EAA8005620591C21601A70B7F858102046F2F702
:10EAB80035FA00212046F2F731FAB7F85A10204605
:10EAC800F2F72CFABD1E07F1480635F8021F20465A
:10EAD800F2F724FAAE42F8D122682E4B0C21501CD2
:10EAE80020605D181170226813F8011F501C9D42A8
:10EAF80020601170F7D123680222591C21601A7016
:10EB0800B7F85E102046F2F709FA2046B7F8601009
:10EB1800F2F704FA0120BDE8F0870B681E4A0120CD
:10EB28005C1C0C6018700B6805241D180D601C70A7
:10EB38000B680A241D180D601C700B6800241D1832
:10EB48000D601C700B6814781D180D601C700B6824
:10EB580054781D180D601C700B6892781C180C6096
:10EB68001A70BDE8F0870020BDE8F0870023A1E611
:10EB7800ACF7FF1FB0F7FF1FB4F7FF1FC844002012
:10EB88007C440020BC440020B844030840640020B2
:10EB9800043400204D340020BF340020A11C030899
:10EBA800F0B5434B1A6883B00123510241490093E1
:10EBB8005CBF03F1805300930968D7005CBF43F042
:10EBC800100300938E073C4948BF43F0C6030978F9
:10EBD80048BF0093D40548BF43F0006301F0EF003D
:10EBE80048BF009308286D4655D00E2953D0D0034E
:10EBF8003248009B00784CBF43F4204343F4005351
:10EC0800D7044CBF43F0C84343F0884300280CBFE7
:10EC180007200F20960648BF43F48073540748BF67
:10EC280043F4003343F400245205009402D5244AE7
:10EC38001279A2BB182936D001900027012639463F
:10EC48002846FCB2F2F79EFB60B11E4B002203F58A
:10EC5800D87103E08B420FD013F80C2C944203F1C7
:10EC68000C03F7D10137242FE9D195E80300164B9F
:10EC780083E8030003B0F0BD7A0904F01F0455F8D7
:10EC8800223006FA04F4013723EA0404242F45F855
:10EC98002240D4D1E9E743F480530093A7E743F433
:10ECA800C0130093C6E7009B43F060730093C3E76B
:10ECB800E87900203C4E002034330020185600200C
:10ECC80030410020481A03085C2200202DE9F84F43
:10ECD8004E014FF0000B174D8146904606F1200774
:10ECE8005C46594628465FFA8BFAF2F74BFBC0B1EF
:10ECF800A64215D8A74213D900200F4A014604E0BE
:10ED08000131242914D012F80C0C504502F10C02E0
:10ED1800F6D10A4B01EB410103EB81014846C0479C
:10ED280001340BF1010BBBF1240FDAD1BDE8F88FE8
:10ED38000021F3E75C220020481A03083C1A030864
:10ED480000210A4A0B4604E00133242B0BD012F8A9
:10ED58000C1C884202F10C02F6D1054803EB430370
:10ED680000EB830070470020704700BF501A03086B
:10ED78003C1A030800210A4A0B4604E00133242BFD
:10ED88000BD012F80C1C884202F10C02F6D105488F
:10ED980003EB430300EB830070470020704700BF7C
:10EDA800481A03083C1A030808B501210220FCF799
:10EDB80011FF094B1B7803F00503052B08D0002130
:10EDC8000120FCF707FF00210846FCF703FFFEE7D8
:10EDD80018F034FFF3E700BFB84C0020022828BF22
:10EDE800022010B4084C094B207000EBC00200EB65
:10EDF800820207495DF8044B013003EB4203C0B2BD
:10EE08000B601AF019BB00BF00360020D634002072
:10EE1800C834002008B506F079FCF1F72FFEBDE8EC
:10EE2800084006F05BBC00BF38B5414B5A89998948
:10EE3800914224BF00225A81198ADA89914224BF5B
:10EE48000022DA81DA788AB1072A0FD0394C3A4899
:10EE5800A27801210025062A01709970DD7150D928
:10EE68002379DFED366A002B3AD138BDDA79002AEA
:10EE78004CD09A783048DFED316A0178042A38BFDF
:10EE8800042207EE902AB8EEE77A07EE901A27EEEA
:10EE9800267AF8EEE77A9A7067EE877A254CA27898
:10EEA800062A2BD8264B03EB8203D3ED086AF4EE2F
:10EEB800E76AF1EE10FA10DDC6EE877AFDEEE77A22
:10EEC80017EE903A102BA8BF1023012BB8BF0123CF
:10EED800DBB28B4228BF0B4603702379002BC4D0CA
:10EEE800013A032AC1D8B7EE000A80EE260A20F0BC
:10EEF80087FB2388984238BF208038BDDFED0F6A32
:10EF0800D5E7DFED107AB0EE677ACBE79B780A4851
:10EF1800DFED0D6A017807EE103A07EE901AB8EEA9
:10EF2800C77AF8EEE77A27EE267A67EE877AB5E7AA
:10EF380080640020F0550020D47800206F12033838
:10EF4800A01C03086F12833A6F1203392DE9F047AA
:10EF5800A84FA94E06F0DAFBBE421ED2DFF8208386
:10EF6800DFF820934446258862197DB14A450DD2C1
:10EF7800052D0BD933886188C3F30B03994200F040
:10EF8800D880144625886219002DEFD17168304663
:10EF98001436FDF766F9BE42E4D3984A5378022B3B
:10EFA80040F2EC8000239649537013789548022B61
:10EFB800016000F2DF8003EBC301934A03EB810396
:10EFC80002EB4303914C184623600EF03DFB904A38
:10EFD8001378A3F1170102290FD98E4911F83300CC
:10EFE800002840F0D180D8000144497829B18A49E5
:10EFF80011F83330002B00F0F580884B9A78042AFA
:10F0080000F0E78032B91A88B2F5F07F84BF4FF478
:10F01800F0721A80824D834A2B681A40002A00F049
:10F02800E480DE0700F1D080580400F1C880190799
:10F0380000F1C0809A0100F1B7809B0400F1AD8017
:10F0480023689A8CD98C914224BF00229A84FFF7B6
:10F05800EBFE15F04DFA10B9734819F0F1FB1EF0EC
:10F06800F9FF00213022714822F0D7FB704B266847
:10F0780003F1500102E00433994279D01A78002A4A
:10F08800F9D19C78D8788442F5D26A496A4B91F8CC
:10F0980000E06A486A4D1C6B6A4B2860C8276421E7
:10F0A80011FB0E71DFF8E0E15960674F30F8041C7E
:10F0B800664DAEF8001000219960D9601961596158
:10F0C8009961D96183F8201083F821103A702E6075
:10F0D8000CB10AF09FFC5E4B9FED5E5A1B885E4A9E
:10F0E8009FED5E6A55795E4C5E495F48086006EEA2
:10F0F800903AF8EEE66A1388C5EE265A07EE103AFB
:10F1080053881279C4ED005A07EE903AB8EEC77AE0
:10F11800564BF8EEE77A1D725A7227EE067A67EEBA
:10F12800867ABDE8F04783ED017AC3ED007A06F0F0
:10F13800D5BA63799B077FF424AF716894F804A06B
:10F148003046FDF78EF83388BAEB133F0BD173883E
:10F158007068AA1FC3F30B039A4204F10601A8BF03
:10F168001A4620F043F81436BE42FFF4FBAE14E70B
:10F1780001228AE700231370234B23E7204903EB7E
:10F18800430301EB830110E7D8000D186D68002DCB
:10F198007FF42AAF1725157026E73548FDF798F84C
:10F1A8004020FDF795F84BE746F20900FDF790F887
:10F1B8002B6842E72F48FDF78BF82B683AE72E4873
:10F1C800FDF786F82B6832E72C48FDF781F82B68A5
:10F1D8002AE71A8BB2F57A7FBFF41CAF4FF47A7224
:10F1E8001A8317E71823137007E743F008032B6007
:10F1F80017E700BFB07C0308A0780308003600209A
:10F20800D2350020E09A0020D6340020C8340020EF
:10F2180034330020703C030804230308F055002011
:10F2280084360020096000024C6400206029002018
:10F23800383300203C73002084780020E4780020D4
:10F24800B89A0020DC5B00202C20002094290020A4
:10F2580078230020C0C9FB48A028002017B7D13860
:10F268007C2300206C6D00203661023D486D002033
:10F278000940000201600002092000020860000243
:10F2880007F0030800000408D830002008B506F08D
:10F298003DFAF1F7F3FB06F021FAFFF757FE0120DC
:10F2A800BDE808401AF0C8B838B50D4C0D4DAC4251
:10F2B80006D2616820461434FCF7D3FFAC42F8D379
:10F2C800094B0A4C0A481860002525700EF0BCF955
:10F2D800084B094A65701A60BDE8384016F01CBB37
:10F2E800A0780308B07C0308C8340020003600204A
:10F2F800D6340020E09A0020D235002008B5FFF768
:10F30800D3FF06F003FAF1F7B9FBBDE8084006F0B1
:10F31800E5B900BFF0B50C292BD8DFE801F06F2A5A
:10F328002A2A4C2A2A2A2B2A2A2A0700046AB2F8EF
:10F338000CE097881668674D24F480540462036AC9
:10F348004468C16923F4005343EA0E3321F4E641CB
:10F35800A84243EA073341EA062100F0B58005F5E3
:10F368000065A84200F0B08092684460C161026400
:10F378000362F0BD046A96899588D2F800E0554F7B
:10F3880024F480740462036A4468C16923F4007336
:10F3980043EA062321F07301B84243EA052341EA10
:10F3A8000E017ED04C4DA8427BD092684460C1616A
:10F3B800C2630362F0BD046A96899588D2F800E0BA
:10F3C800444F24F010040462036A4468816923F0FE
:10F3D800200321F0807143EA061321F4E641B84284
:10F3E80043EA051341EA0E2148D03B4DA84245D0D7
:10F3F80092684460816182630362F0BD046A938904
:10F40800B2F804E01768334E24F001040462056A78
:10F418004468816943EA0E0321F4803125F002052E
:10F428009BB221F07301B04243EA050341EA0701A8
:10F4380014D0294DA84211D005F54065A8420DD039
:10F4480005F58065A84209D005F58065A84205D074
:10F4580092684460816142630362F0BDD689158A6F
:10F46800578A23F0080333433D43D68824F4407475
:10F4780023F00403ADB233432C43E9E7D589178A57
:10F48800D68823F0800343EA051324F44064558AA0
:10F4980023F0400344EA870443EA061344EA850458
:10F4A800A6E7D589178AD68823F4006343EA05239B
:10F4B80024F44054558A23F4806344EA071443EA49
:10F4C800062344EA051470E7158A24F4804444EAC4
:10F4D800851449E7002C0140003401402DE9F84F1C
:10F4E8004FF4A07200218F488F4CDFF864928F4D43
:10F4F8008F4E904FDFF85C8222F08FF98E488F494B
:10F50800DFF854E2DFF854C200221359834200F0B6
:10F51800F880B3F1804F00F0F680AB4200F0F58040
:10F52800B34200F0F480BB4200F0F380734500F072
:10F53800F280634500F0F180434500F0F080DFF889
:10F5480020A2534500F0A7800AF5806A534508BFFA
:10F55800092300F0A1801432C82AD6D1DFF8C88167
:10F56800774F784D08F1C8064FF0030A4FF00209AB
:10F5780098F804301C09013C052C03F00F0300F235
:10F58800838037F8140040FA03F2D2077CD54FF095
:10F59800010B0BFA03F3013B18401FF0F1FC6A4B17
:10F5A8001B5D184415EBC0046ED055F83030674821
:10F5B80098F8081003F13842920A825C02F01F00A2
:10F5C8005209022A0BFA00FB00F09480032A00F08B
:10F5D8008A80012A05D1594A584852694BEA0202E1
:10F5E8004261B4F804E0BEFA8EF2C2F11F0292B290
:10F5F800D00803EB800002F00702046A92004FF083
:10F608000F0C0CFA02FC24EA0C040462046A01FAE6
:10F6180002F22243002402624FF0010C224603E06A
:10F62800102A04F102042FD00CFA02F030EA0E017D
:10F6380002F10102F4D1D3F808B00AFA04F1C9437F
:10F648000BEA010BC3F808B0D3F808B0C3F808B048
:10F65800B3F804B01FFA8BFB2BEA00009880988857
:10F6680080B29880186808401860D3F800B009FA8A
:10F6780004F040EA0B001860D868102A01EA00017B
:10F68800D96004F10204CFD108F1140846457FF48B
:10F698006FAFBDE8F88F082309EBC3034FF0010BE8
:10F6A80093F840A00AF01F034FEA5A1ABAF1020F62
:10F6B8000BFA03F30BD0BAF1030F0ED0DA457FF43F
:10F6C8004AAFD1F814A043EA0A034B6143E7D1F8E3
:10F6D80018A043EA0A038B613DE7D1F81CA043EA6E
:10F6E8000A03CB6137E7154A1448D2694BEA02028C
:10F6F800C26176E7114A114892694BEA02028261B7
:10F708006FE70023C8E70123C6E70223C4E7032302
:10F71800C2E70423C0E70523BEE70623BCE70723A7
:10F72800BAE700BFE8620020D83F030800040040A1
:10F738000008004000100040002C0140001002406A
:10F7480054280308B85400206028030868280308D0
:10F75800A01C030800400140001400400034014090
:10F768000044014001490248FEF70ABF0064002036
:10F778000048014001490248FEF702BFB06300207B
:10F788000040014001490248FEF7FABE88630020A4
:10F798000034014001490248FEF7F2BE88630020A8
:10F7A8000034014001490248FEF7EABE60630020C8
:10F7B8000008004001490248FEF7E2BE3863002015
:10F7C8000004004002494FF08040FEF7D9BE00BF58
:10F7D8001063002010B5064C06482146FEF7D0FEFF
:10F7E80004F1F0010448BDE81040FEF7C9BE00BFAF
:10F7F800E8620020002C0140004401400149024811
:10F80800FEF7BEBEE8620020002C01402DE9F04161
:10F818000468574DA30AAB4200F085805CD9554D6A
:10F82800AB426CD078D9544DAB4264D00135AB4271
:10F8380040F09A804FF49C7E072647794FEA970C50
:10F8480000297CD0B000634685190227D4F80C80C3
:10F858009F400CEB4503BFB2484D03F1040C47EA47
:10F86800080745F8231045F82C20E760EFF31181CD
:10F87800502282F31288821905EBC2021369002B09
:10F8880041D013620433821905EBC202576917B1DC
:10F898001F6053690433821905EBC202976917B1D7
:10F8A8001F6093690433821905EBC202D76917B147
:10F8B8001F60D36904330027CAB21F6082F311881E
:10F8C800304405EBC000036A03BBE3684FF6FE72E1
:10F8D8001340E360BDE8F0814A3DAB422BD00135CF
:10F8E800AB4204D0B3F5801F21D0BDE8F0814FF0C2
:10F8F800980E0326A1E74FF4887E06269DE74FF071
:10F90800E80E052699E705EB0E03BCE7E36843F02C
:10F918000103E360BDE8F081033DAB4226D14FF01F
:10F92800C00E042689E74FF0200E002685E74FF029
:10F93800480E012681E74FF0700E02267DE7BF08CA
:10F94800022306FA03F0BB40DB43E7680B4D9BB28A
:10F958003B4087190CEB470CE3600CF1040345F8B6
:10F968002C1045F8232081E7BDE8F081BDE8F0813F
:10F978004B0010005000100051001000E8620020F9
:10F9880030B503685C4D18885C4CB4FBF2F2013961
:10F99800013AAB4294B283B089B282B266D0584879
:10F9A800834263D0B3F1804F60D0A0F59830834292
:10F9B8005CD000F58060834258D0524883425BD0C7
:10F9C80000F5806083427DD022F4407200F58C30CF
:10F9D80092B283421A80D9621C850ED0484A93425B
:10F9E8000BD002F54062934207D002F58062934241
:10F9F80003D002F58062934201D100221A860122C7
:10FA08005A611A883C4992B242F001028B421A802C
:10FA180062D0B3F1804F61D03B4A934260D002F587
:10FA2800806293425ED002F5006293425CD002F598
:10FA3800806293425AD002F59032934258D002F530
:10FA48004062934256D002F5806293421ED002F57E
:10FA58008062934208BF092219D002A84FF00123FF
:10FA680040F8043D1DF00EF903B030BD254822F0E2
:10FA78007002834292B2A3D101201A80D9621C85F8
:10FA880058611A8892B202431A80C5E708221F4BB0
:10FA980003EBC20301A893F841408DF80440012309
:10FAA80000228DF805308DF807308DF806201DF0FE
:10FAB800E9F81B2CD8D1164B019301A81DF0E2F8E8
:10FAC80003B030BD01201A80D9621C8558611A889C
:10FAD80092B202431A809CE70022D8E70122D6E7B7
:10FAE8000222D4E70322D2E70422D0E70522CEE798
:10FAF8000622CCE70722CAE7002C014000A24A04EC
:10FB0800003401400010004000040040A01C03081D
:10FB180019010001204B98422DD0B0F1804F2CD014
:10FB2800A3F5943398422AD003F58063984228D0ED
:10FB380003F50063984226D003F58063984224D0E9
:10FB480003F59033984222D003F54063984220D0C1
:10FB580003F58063984207D003F58063984208BF95
:10FB6800092202D00020704708220C4B03EBC20385
:10FB780093F8400070470022F7E70122F5E70222D8
:10FB8800F3E70322F1E70422EFE70522EDE7062277
:10FB9800EBE70722E9E700BF002C0140A01C03089F
:10FBA8002DE9F04F2DED028B9B4A9C49137897B0B5
:10FBB80004460B9000F59C4020300E900860002B06
:10FBC80000F07E85964909688C4240F297809549F5
:10FBD800059109689448954D954C0491013B137023
:10FBE80001F4805303900A93002B40F09580039B07
:10FBF8005B7D002B40F00285049B180400F1E98727
:10FC0800049BD9050BD50B9A8A4BDFF858B29A4258
:10FC18009BF8022001F2AD81002A41F0AE81864BAB
:10FC28000693864E049B13F4805840F00885039B86
:10FC3800B4F906705B8B9F42B4BF00270127804B45
:10FC48001B6813F0805374D0069A127812F00102E0
:10FC580076D00399DFF81092898C99ED037A07EE34
:10FC6800901AF8EEE77AB4EEE77AF1EE10FA81F23C
:10FC78007680002F6BD195F8A410002967D17148C0
:10FC88007149006890F830004FF0000EC1F800E0AC
:10FC9800C1F804E0C1F808E06C49002858D10870A0
:10FCA800002A59D0049AD00656D5694A1278D10646
:10FCB80052D4B8F1000F4FD1002B4DD1049B5A02FA
:10FCC8004AD496F800E0BEF1000F01F08787614B37
:10FCD8009B78002F41F0AE873BB15F4A5F4B1268BB
:10FCE8001B689B1A002BC1F2CF87102019F0C6FAA7
:10FCF800012385F8A53096F800E02FE0494B0593DD
:10FD08001B680493484A494D039203F48053484CB6
:10FD18000A93002B3FF46BAF00214948F1F732FBFF
:10FD280000287FF464AF07F0CBFA059B1B680493A7
:10FD38005DE7049A520287D4069A127802F001020B
:10FD4800002185F8A410DFF82091002F97D03F49B3
:10FD580001200870002AA5D196F800E0039AB4F9AA
:10FD68000080518B928BB4F9020095F8A6B08845B3
:10FD7800CCBF4FF0800C4FF0000C4CF04003904586
:10FD8800A8BF63469B0843F0800C8842C8BF6346FF
:10FD980043F0400C9042B8BF63469B08B4F904C0D6
:10FDA800B4F9060043F080088C45C8BF434643F0C9
:10FDB80040089445B8BF43469B0843F0800C8842EE
:10FDC800C8BF634643F0400C9042B8BF63469B45AA
:10FDD80000F010864FF0000885F8A63085F8A78057
:10FDE800BEF1000F00F06787059B1B6803F0040352
:10FDF800002B40F07D850DF1500A194E0023CAF8FA
:10FE0800043006F1500B14934FF0190840F63303F1
:10FE180040F283372DE000BFCC2D0020802C00203D
:10FE2800C82D0020E8790020F05A0020B0280020D2
:10FE3800445E0020404B4C00173C00202C20002042
:10FE480068300020C8340020803000204024002082
:10FE58007030002004790020009A0020942E0020A1
:10FE680038330020DC5B00205041002004365E451A
:10FE780024D0B178F278914218FB0170F6D296F846
:10FE880001E00EF1040E18FB027134F91E209A42AB
:10FE9800A8BF1A46B2F5617FB8BF4FF461729042AD
:10FEA800E4DA9142E2DB31782329DFD85046043680
:10FEB8000493F1F757FA5E45049BDAD15C4B9AE854
:10FEC80003001F785B4B83E80300002F00F09B843E
:10FED800594B049357480121F1F754FA002840F090
:10FEE8005E82059B1B68DE0500F15482534B079325
:10FEF800534D2B881EB226F001061FFA86FA534589
:10FF0800A5F800A000F0E4854E4E4FF002080F203F
:10FF180014274FF0FF0B86F80080777086F802B040
:10FF280019F0ACF941464348B5F800A0F1F72AFAB0
:10FF3800002841F0B3812AF002039BB253452B807D
:10FF48000BD0404B1421FF2202260F201E7059703F
:10FF58009A7019F093F9B5F800A03B4B3B4A197811
:10FF6800506808931AF0030F08BF81F00201C1F32B
:10FF780040010992FBF7FAFD079B1B6813F00A0F73
:10FF88001AD006212B48F1F7FDF9002800F07F86EA
:10FF98002B88580641F1EE8007212648F1F7F2F93F
:10FFA80050B12B4B2B4AB3F904302B4982FB030287
:10FFB800DB17C3EBA2030B800C211E48F1F7E2F913
:10FFC8002A88002800F04F8242F480739A422B80DE
:10FFD80009D01C4B02261421FF220F201E705970D5
:10FFE8009A7019F04BF91D4B1B78082B00F04782CB
:08FFF8000E2B00F04482059B72
:020000040801F1
:100000001B68590561D5184B1B79002B00F018812E
:1000100014210A48F1F7BAF9002840F016810EF0D1
:10002000D1FB012019F080F800284ED0DFF83CA069
:1000300000264FF0CC0B1EE06E5E002068300020E2
:10004000E09A00203C4E00206C5E0020E02B002057
:10005000CB990020CC990020983D00206766666609
:10006000922E002034330020304100207C94002068
:10007000DEB2022E29D80BFB06F8731C5AF8087062
:10008000002FF5D1C378D84A90F9020052F82330F6
:1000900001970322009201213A4618F027FC0346FB
:1000A00006EB460000EB0010079353B139460AEB0C
:1000B0008000CC2221F0B5FB079B4AF808300136BE
:1000C000F6B216F0DDFC0028D3D1069B1E7816F0A0
:1000D000010600F01182C54B01221A70049BB4F98D
:1000E00006101B68C2485A8901279142077080F2A6
:1000F000E981C04B4FF07E521A60BF4A039BB4F9AE
:1001000000C01F8B92F9043092F801E01078002BA8
:10011000ACEB070314BF01224FF0FF32002B40F37A
:10012000C581B3F5FA7FC0F2C7814FF4FA731B1A89
:1001300007EE903AF8EEE77A6745C9ED007A03DDFD
:10014000F1EE677AC9ED007AB4F902C0ACEB0703AF
:10015000002B40F38081B3F5FA7FC0F282814FF427
:10016000FA731B1A07EE903AF8EEE77A6745C9ED85
:10017000017A03DDF1EE677AC9ED017AB4F9040082
:10018000C31B002BD8BF3B1AB3F5FA7F80F25E8108
:100190007345D8BF4FF0000E00F35A8102FB0EF2F8
:1001A00007EE902A059BF8EEE77AB8421A68C9ED87
:1001B000027ABCBFF1EE677AC9ED027A12F480527E
:1001C00000F00B82B1F5FA6FA8BF4FF4FA61B1F5F8
:1001D0007A7FB8BF4FF47A71A1F57A71874C88485D
:1001E00084FB013ECB17C3EB6E1303F1010E6FF0DE
:1001F000630C30F91EE030F913000CFB0313AEEB77
:10020000000103FB01F384FB0314DB17C3EB64134E
:1002100003441BB207EE903AB8EEE78A89ED038AF1
:10022000002A40F08C832B885B0624D4002E40F0FB
:10023000A8801EF0F4F817B0BDEC028BBDE8F08F7B
:10024000069B1B78DA077FF5EAAE3C201AF088FDA2
:1002500000283FF43AAF11F05DF83C201AF022FD7F
:1002600000283FF432AF11F055F83C201AF01AFD87
:100270000028F0D129E7634B634AB3F9043063499E
:10028000DFED636A09889FED637A82FB0302DB1767
:10029000C3EBA2035B1A1BB207EE903AF8EEE77AC3
:1002A00067EEA67A77EE876ABDEEE66A16EE103A3A
:1002B0002033402B40F26D87BDEEE77ADFED626AB6
:1002C00017EE103A2033402B00F2B0879FED527AA0
:1002D000F4EEC77AF1EE10FA41F32C83DFED4F5ABA
:1002E0009FED4F6A01E0F0EE477AF4EEC67AF1EE48
:1002F00010FA37EEE57AF6DCDFED4A7AB4EEE77A0B
:10030000F1EE10FA41F11283DFED445A9FED466A97
:1003100001E0B0EE677AB4EEC67AF1EE10FA77EE4D
:10032000257AF6D49FED3B7AF4EEC77AF1EE10FA17
:1003300040F330859FED387A77EE677A67EEA75AFB
:100340009FED3A5A9FED3A6A9FED3A7AA5EE856A9B
:1003500027EEA55AA5EE867AE5EE077A99ED016AB1
:10036000D9ED005A27EEC67A65EEA77AA5EEA67AF1
:10037000E6EE267A89ED007AC9ED017A002E3FF487
:1003800058AF089B1978099B01F001011868FBF729
:10039000F1FB17B0BDEC028BBDE8F08F264BDB788C
:1003A000002B3FF4A7AD254B07931B689D077FF5F6
:1003B000A3AD234DB5F800A01AF0010F7FF4BFAD37
:1003C0004AF001039A452B803FF4B9AD1D4B022240
:1003D00014211A700F20FF2259709A7018F052FFE2
:1003E000B5F800A0ABE500BF78240308183C002056
:1003F000802300201C240020D87800201F85EB518A
:10040000E49A0020983D002067666666922E0020E0
:1004100035FA8E3CDB0FC93FDB0F4940DB0FC9408B
:10042000E4CB1641DB0F49C0E4CB16C192E741B9DA
:100430009730083C15A82ABEDC5B00203C4E00200B
:100440006C5E0020E02B0020000000004FF4FA73E7
:10045000A3EB0E0EA2E6A7EB0C03B3F5FA7FBFF6F3
:100460007EAE9842FFF67DAE5FED097A7EE622F41D
:1004700080739BB29A422B807FF4AFAD7E4B1B788A
:10048000082B7FF4B9AD2A8822F040039BB29A4230
:100490002B803FF4B4AD794B02261421FF220F20AC
:1004A0001E7059709A7018F0EDFEA8E5A7EB0C03CA
:1004B000B3F5FA7FBFF639AE9842FFF638AEDFEDFE
:1004C000707A39E6B1F5FA6F80F22883187A8B1AC0
:1004D00003FB00F3C2F5FA6293FBF2F3C3F164038A
:1004E00007EE903AF8EEE77A9FED667A664B67EE94
:1004F000877AC3ED007A00E6644B1B780793002BE4
:100500007FF4ECADDFF8B8B1DFF8B8A11BF8030C4D
:100510009AF800805946ABF103071DF0FDFC002856
:1005200000F00283079BB8F1000F53D107F10801D7
:1005300078791DF0F1FC002841F06A825449B87ABC
:100540001DF0EAFC002800F00383B8F1020F41F02F
:1005500062825049F87B1DF0DFFC002841F05E828A
:100560004D49387D1DF0D8FC002800F00383B8F118
:10057000040F41F056824949787E1DF0CDFC0028D9
:1005800041F052824649B87F1DF0C6FC002800F0B9
:100590000383B8F1060F41F03882424997F82300EF
:1005A0001DF0BAFC002840F084873F4997F82800E6
:1005B0001DF0B2FC002800F00383B8F1080F40F0F2
:1005C00067873A4997F82D001DF0A6FC00283FF4F4
:1005D00085AD09231A4600F05DBF039B588B81420D
:1005E000C0F29A82B1F5FA6FD4BFC0EB0101C0F539
:1005F000FA614FF47A7303FB01F1C0F5FA60B1FBC5
:10060000F0F1EBE5039A013BD27D34F91330002A77
:1006100040F06E83A3F57A73B3F57A7FA8BF4FF4E9
:100620007A7323EAE37307EE903A9FED217AF8EEAE
:10063000E77A67EE877A1F4AFCEEE77A17EE903A80
:100640001380FFF7E1BA1D211B48F0F79FFE002839
:100650007FF4F1AA194A039BD2881B8BB4F9067068
:10066000991A8F4240F3C48613449F42B4BF0027B7
:100670000127FFF7E8BA00BF34330020E02B002049
:10068000000000000AD7233C1C240020183C002056
:10069000BB2B0020C02B0020C52B0020CA2B002024
:1006A000CF2B0020D42B0020D92B0020DE2B0020C4
:1006B000AAF1823FC85B0020683000201479002036
:1006C000B12B002022000020B34DB44B2E780393B1
:1006D000DFF8CC82002E00F02183B6B1DFF808935A
:1006E000DFF808B3AE4FCA460024072C3846E1B203
:1006F000D8F8043041F35282984700B20134A64240
:100700002BF8020F0AF1040AEFD1A64B05931A4603
:100710000B99A54B12680492A3FB013E42F2010320
:1007200013404FEA9E1E099300F0E7829F48A04ABB
:10073000A04B0078A049079012781A70079B0870A8
:1007400023B19C4B1B7883F0010307939B4A0399C9
:1007500012780D920D9A0C8D994BB1F8269091F864
:1007600022C010940C8B13941146A3FB01135B0859
:1007700003EB4303D31ADBB295F829400F93049B94
:1007800098F800002E7808900F2220460CF1040CF7
:1007900003F480538B4F8C4CDFF854A2CDF81890A3
:1007A0005FFA8CFCB34685F8282011920A93002149
:1007B00081460C95CDF8488036B9089B9C458DBF85
:1007C0009B46E34666465E46B14280F26383079BE2
:1007D000002B00F00D837D4B069833F911201FFA92
:1007E00082F880454FEA410303D31098804540F2D8
:1007F0004C835AF82120964580F00483E25E0998E4
:10080000002840F01B83E25201310637D4E7DFF8BD
:10081000E4B1DFF8E4810BF15A064FF0010A5946C2
:100820001BF8010C1DF078FBF8B19BF804009BF855
:1008300002309BF803E000EB400105EB8101013B36
:10084000D1F8B42003EB4303434493420DD095F811
:10085000E02081F8B0E00AFA00F022EA0000C1F8D6
:10086000B430C1F8B87085F8E0000BF1060B5E45B6
:10087000D5D1574B574A049319464F4BD2F800B085
:1008800009681B78544E0891DA4607930027AB4657
:10089000736853B31D7845B3B168AAEB0101002911
:1008A0000ADB9BF8E0100120B84021EA00010AF5BC
:1008B000FA708BF8E010B060079AB2B131785878CE
:1008C0000431C9B2002840F05382039A34F9111060
:1008D000108B00F1C80E714540F35E859BF8E01067
:1008E0009B783941C90740F1BE850137042F06F1D5
:1008F0000C06CDD1FFF7F2BA95F8AB3053B1069B99
:100900001B78D80706D5039BB4F906205B8B9A4267
:1009100000F39B8511213148F0F738FD002800F0E5
:10092000098295F8AE302BB995F8A93013B9322366
:10093000A5F8AC30012385F8AE30FFF760BA1D2171
:100940002648F0F723FD00283FF46DAC244BDB78FC
:10095000002B7FF468ACDFED237A134938EE678A09
:10096000C7F5FA63FDEEC87A1BB2CDED037ABDF987
:100970000C20120381FB0201D217C2EBA11203FB70
:1009800002F343F30F333B4407EE903AF8EEE77A75
:10099000C9ED037A47E400BFB0280020F05A0020D8
:1009A000742C0020E8790020D34D6210502C0020D8
:1009B0007401002075010020C15B0020CD2D0020B6
:1009C000ABAAAAAADC280020445E0020B42800209C
:1009D000E09A0020009A0020602900206830002062
:1009E000DC5B002000007A44382E0020B228002072
:1009F000D02D0020C92A00202C1D030895F8A780BF
:100A0000B8F1F90F00F2A88108F101085FFA88F83F
:100A100085F8A78085F8A630BEF1000F00F0508160
:100A2000B8F1140F7FF4E4A95F2B40F05C81069FBE
:100A30003B7813F0010300F0818706F045FC3B781A
:100A400003F00103002B7FF4D3A995F8A620572AC1
:100A500000F00087059B1B6813F0040302D05A2A9C
:100A600000F02A855D2A00F05D875B2A00F07F8711
:100A70005E2A00F0FE84562A00F0E18733782BB11D
:100A80006F2A00F0D487CA4B00211960972A00F022
:100A9000E587A72A00F0CE840021BB2A149101F03B
:100AA0000B80B72A00F0EA87BE2A01F00880BD2A31
:100AB00001F047809E2A01F031809D2A01F02680B6
:100AC000AE2A01F01B80AD2A7FF492A9FF210020FD
:100AD0000BF0AFFCFFF78CB90221B648F0F756FCDB
:100AE00000283FF42CAA2E801AF0020F7FF439AAB6
:100AF0004AF0020353452B803FF433AAAE4B022247
:100B000014211A700F20FF2259709A7018F0BAFB46
:100B1000B5F800A0FFF725BA11466EE51B7AC3F1C0
:100B2000640307EE903ADDE40BF1050178791DF0DE
:100B3000F3F900283FF402ADB8F1010F40F06887E7
:100B400007F10D01B87A1DF0E7F9002840F063873E
:100B50009A49F87B1DF0E0F900283FF401ADB8F1A7
:100B6000030F40F05B879649387D1DF0D5F90028CA
:100B700040F057879349787E1DF0CEF900283FF466
:100B800001ADB8F1050F40F04F878F49B87F1DF0D8
:100B9000C3F9002840F039878C4997F823001DF0ED
:100BA000BBF900283FF401ADB8F1070F40F0818494
:100BB000874997F828001DF0AFF9002840F06884B5
:100BC000844997F82D001DF0A7F900283FF486AA64
:100BD000B8F1090F3FF482AAFBE4D5F88C300B9AE8
:100BE000D31A002BFFF610A87B4A95F89030517C61
:100BF0007A4A039E32F811200E98B17DC5F88C0018
:100C0000013303F00F0385F890302B4492B292FB2E
:100C1000F1F283F8942095F8940095F8951095F8E2
:100C2000962095F8973001440A4495F8980095F875
:100C300099101344184495F89A2095F89B30014474
:100C40000A4495F89C0095F89D101344184495F8B3
:100C50009E2095F89F3001440A4495F8A00095F82D
:100C6000A1101344184495F8A23095F8A32001442C
:100C70000B441A4442F30B12642AF17DA8BF64228C
:100C800013B209B1C2F1640307EE903A9FED547AB2
:100C9000F8EEE77ACDE42A8822F040039BB29A422C
:100CA0002B803FF47DA9444B02261421FF220F2004
:100CB0001E7059709A7018F0E5FAFFF771B9F04696
:100CC00000213C48F0F762FBD8B1002385F8A8303A
:100CD00006F07AF995F8A730142B7FF489A83378B9
:100CE000002B40F0D187069B1B7803F00103A9E697
:100CF000C3F53B6308331BB28CE43A4B1B78079374
:100D00001EE5069B2A4A1B781060DB0700F17C85F4
:100D1000B8F1140F3FF499AEFFF76AB893F8223098
:100D200098F800600433DBB2B3428EBF2E702B7094
:100D30001E46D2E495F8A930002B3FF460A8069B2C
:100D40001B7813F001037FF45AA8012285F8A9301B
:100D500085F8AA20FFF753B885F8A6B0BEF1000FBA
:100D6000AED0FFF745B8012185F8A410FEF7F3BF18
:100D7000012800F083859BF8E0100123BB40013778
:100D80000B43042F8BF8E03006F10C067FF480ADA6
:100D9000FFF7A4B89FED147AF4EEC77AF1EE10FADB
:100DA00044BF9FED127A77EE677AFFF7C7BA00BFAC
:100DB000982E002068300020E02B0020C02B00205F
:100DC000C52B0020CA2B0020CF2B0020D42B0020C5
:100DD000D92B0020DE2B0020089A0020249A002026
:100DE00014AE2341C15B0020DB0FC9BFDB0F49C03C
:100DF000069B002B47D05AF8212096454FEA410325
:100E0000FFF4FCACBE4ABE48D25C00EB0308002AEB
:100E100000F01082022A40F0A58198F8012002EB30
:100E2000820202EB820202F2EE2292B2032940F326
:100E30009B80099812B200283FF4E5AC0F9803EBB1
:100E4000010880440C9800EB4808A8F82C20B9F160
:100E5000000F03D10D9802287FF6D5ACB7F80090AB
:100E60007A88B7F804804A449044A64A0FFA88F872
:100E700082FB0802A448A2EBE87220F8038012B2B9
:100E80004FF00109BFE41A464B000EF596784AF878
:100E90002180B4E411990C9D9C4BDDF8488085F8C5
:100EA00000B00F294A460CBF0122002285F8299084
:100EB00085F828101A7006D11B219548F0F766FABC
:100EC000002800F018859348934B82681968934B6B
:100ED000C1608A1A012119704368914F9A42039A9E
:100EE000397088BF002392F8227088BF80F82130C3
:100EF0000A9B98F80000B2F818C0B2F826800437B0
:100F0000FFB2002B00F0A38187427D4A40F220828D
:100F1000844F964600210EB983460646B1421ADA3E
:100F200012F8113093B1022B0ED19EF8013003EB71
:100F3000830303EB830303F2EE239BB227F8023B08
:100F400001310EF1020EE6E73B88F7E7CBB2032B47
:100F5000FAD86346F2E785F800B00D9B724A013378
:100F600013700A9BFEF744BE012000FA01F81198A5
:100F700020EA080012B2119041E412B901228BF864
:100F800002206A4B06931E789BF8219006F001031D
:100F90001B2004931CF0EAFFB9F1010F089000F048
:100FA0002A8206F0020307939BF82020604EDFF8A8
:100FB00088A1604FDFF86081052A00F29880DFE8A1
:100FC00002F0887C032E3E52B9F1010F04BF0523C5
:100FD0008BF82030049B002B00F0D880039BD8F8BE
:100FE0000000B3F91810BAF80230002261F30F02C2
:100FF00063F31F42002361F30F0361F31F43DBF828
:10100000141062608842236040F2738103230793C7
:1010100047F230520323CBF81C208BF820303B885A
:1010200043F002033B8006F04FF9D8F80020DBF8CC
:101030001C3013440422CBF818308BF82020B9F16F
:10104000010F40F06684D8F80030DBF818209A428F
:101050004DD2307818B91CF089FF002847D13B8861
:1010600023F002033B80D8F80020BAF80630642150
:1010700001FB03234FF4806000228BF820208BF8C3
:101080000320CBF8103018F0F3F99BF8202093E7F9
:101090001CF098FF012800F0AD84089B002B40F065
:1010A000AD81B9F1010F22D0D8F80030DBF8102063
:1010B0009A4259D301238BF82030B9F1010FD2D0D5
:1010C0009AF80830012B4FD017F096FA9BF82020A1
:1010D00072E7049B002BDBD1089B4FF48060002B50
:1010E00000F0F28018F0DCF90022CBF81020079B0A
:1010F000002B40F0FA80059B1B680493FEF797BD18
:101100006C2E0020565555552429002071300020A2
:1011100068300020DC5B0020009A00207401002071
:1011200075010020445E0020CD2D0020173C0020DA
:101130002C200020005C00203C730020E4CB1641F2
:10114000DB0F49C0DB0FC940E4CB16C1DB0FC93F41
:10115000DB0F494092E741B99730083C15A82ABEF9
:1011600000000000E25A61E617F046FA032240F65A
:10117000B8338BF82020CBF81C3050E743F0400206
:1011800093422A807FF48FADFEF70ABFD8F8003073
:101190003EE7F4EEC77AF1EE10FA40F323845FEDF8
:1011A000175A1FED1A6A01E0F0EE476AF4EEC66ABC
:1011B000F1EE10FA36EEE57AF6DC5FED1F6AB4EE7A
:1011C000E67AF1EE10FA40F111845FED225A1FED3C
:1011D000226A01E0B0EE667AB4EEC67AF1EE10FA59
:1011E00077EE256AF6D41FED277AF4EEC76AF1EEA2
:1011F00010FA6CDD1FED2A7A77EE666A66EEA65A63
:101200001FED2C5A1FED2C6A1FED2C7AA5EE856A76
:1012100026EEA55AA5EE867AE5EE076ABDEEE77AD8
:1012200017EE103A2033402B7FF650A85FED347A4A
:10123000FFF794B8CAB2022A40F2E382032A91D19E
:10124000139A0A98069D002808BF2A46EEE58742B1
:101250001946B64A55D8B64896460EB9BB463E46DC
:101260008E427FF778AE12F8113093B1022B0ED177
:101270009EF8013003EB830303EB830303F2EE23B9
:101280009BB220F8023B01310EF1020EE5E7038824
:10129000F7E7CBB2022B03D9032BF8D14346F0E793
:1012A0006346EEE72AF0010292B252452A803FF4EB
:1012B0001BAC0F2086F80080777086F802B017F01C
:1012C000E1FFB5F800A00FE418F0D2F80CE79FEDAD
:1012D000997AF4EEC76AF1EE10FA44BF9FED967A60
:1012E00077EE666A8AE703230793079817F0CAFF29
:1012F00001E7B9F1010FF6D103239BF820200793F2
:101300005AE68B4F96460EB983460646B142BFF663
:1013100022AE12F8113093B1022B0ED19EF801309B
:1013200003EB830303EB830303F2EE239BB227F863
:10133000023B01310EF1020EE5E73B88F7E7CBB245
:10134000022B03D9032BF8D14346F0E76346EEE7BF
:101350007748964600210EB9BB463E46B142BFF6DD
:10136000FAAD12F8113093B1022B0ED19EF8013074
:1013700003EB830303EB830303F2EE239BB220F81A
:10138000023B01310EF1020EE5E70388F7E7CBB22D
:10139000032BFAD86346F2E7C83881423DDA9BF85E
:1013A000E0109B783941CA073FF59FAAC3F10008B6
:1013B000012018F045F8691E162900F20B81DFE8BC
:1013C00011F0F8010C02E101BC0154012F010C01E4
:1013D000A3018E01790164010901BC01CD012F0136
:1013E0000C01A301B601B901CF00F900E300A1008F
:1013F0000127FEF728BC00230793D5E59AF80430AF
:10140000002B3FF44EAE17F0F7F803224FF47A7337
:101410008BF82020CBF81C3001E69BF8E03001214E
:10142000B94023EA01030AF5FA718BF8E030B160A4
:10143000FFF75BBA4149059B0A781B6842F004023A
:101440000A7003F00403FEF7D7BC00213C48EFF715
:101450009DFF00287FF45EAA322385F8AB00A5F833
:10146000AC30FFF757BA9846002B0CBF0120022082
:101470009FE7344B022203203349344E0B60327015
:1014800017F0DEFF059B1B6803F00403FEF7B4BCF6
:1014900008231A4602EB820217448AF80030B97812
:1014A000787814F0D5FB069B1E7806F00106FEF74F
:1014B00015BE07231A46EDE795F8A920002A40F04B
:1014C000438395F8AB1081F0010185F8AB1000293A
:1014D00040F099831E4A126812F4003204D01D4A6B
:1014E0001279002A40F0C583114610461A4A565C0C
:1014F0000D2E01F10C0100F0E68201301528F6D125
:10150000FEF77ABCDBF8E400144B90F83A109D78B3
:1015100041446429A8BF642121EAE17180F83A10AE
:10152000002D40F0BC830CF0D9F924E46C2E00208F
:10153000445E0020DB0FC9BFDB0F49C070300020C4
:10154000683000206A350020C834002000360020B2
:1015500098290020D05B0020081F0308414D00207F
:10156000DBF8E4008178B74B4144C829A8BFC82103
:1015700021EAE17181709B78002BD4D014201CF0FB
:1015800053FDDBF8E400CEE7DBF8E400AD4B90F868
:101590003B109D784144FE29A8BFFE2121EAE1715C
:1015A00080F83B10002DBED016201CF03DFDDBF86E
:1015B000E400B8E7089AA34B51784144B1F5967F0F
:1015C000A8BF4FF4967121EAE17151709B78002B0E
:1015D00040F02283DBF8E400A5E7DBF8E400994B58
:1015E00001799B784144C829A8BFC82121EAE1714B
:1015F0000171002B40F04283102D94D04178914B23
:101600004144C829A8BFC82121EAE17141709B78F3
:10161000002B88D013201CF007FDDBF8E40082E7E4
:10162000DBF8E400874BC1789B784144C829A8BF08
:10163000C82121EAE171C170002B40F0F9820F2D21
:101640003FF471AF01787F4B4144C829A8BFC8213E
:1016500021EAE17101709B78002B3FF464AF122006
:101660001CF0E2FCDBF8E4005DE7089A754BD179E9
:101670009878414481F30801D1710028AAD005204F
:101680001CF0D2FCDBF8E4004DE7DBF8E4006D4B26
:10169000017A9D784144C829A8BFC82121EAE17197
:1016A0000172002D3FF43FAF0B201CF0BDFCDBF8B6
:1016B000E40038E7DBF8E400624BC1799D784144EF
:1016C000C829A8BFC82121EAE171C171002D3FF4EA
:1016D0002AAF0A201CF0A8FCDBF8E40023E7DBF8C3
:1016E000E400584B81799D784144C829A8BFC8219E
:1016F00021EAE1718171002D3FF415AF09201CF042
:1017000093FCDBF8E4000EE7DBF8E4004D4B417995
:101710009B784144C829A8BFC82121EAE1714171E1
:10172000002B40F07F82112D7FF41CAFFBE6DBF82D
:10173000E40087E7DBF8E40060E7089A414B917921
:10174000987841446429A8BF642121EAE17191712C
:10175000002840F08A820D2D3FF43CAF089A394BA7
:101760005179987841446429A8BF642121EAE17144
:10177000517100283FF42EAF0E201CF055FCDBF811
:10178000E400D0E6089A15794544642DA8BF642585
:1017900025EAE57515711CF061FC2A4B9B78002B3E
:1017A0003FF418AF032029461CF03EFCDBF8E400B0
:1017B000B9E6089A234B11784144FA29A8BFFA21C7
:1017C00021EAE17111709B78002B3FF403AF0120F7
:1017D0001CF02AFCDBF8E400A5E6089A194B917886
:1017E00041446429A8BF642121EAE17191709B788A
:1017F000002B3FF4EFAE02201CF016FCDBF8E400F7
:1018000091E6139AFFF712BB0F4B1B78002B3EF4A7
:10181000EFAA0E4BDB78002B7EF4EAAA95F8A830ED
:101820000133DBB2032B85F8A8307EF6E1AA084B22
:101830005B7813B9002F7EF4DBAA05F045FDFFF7B6
:1018400049BA00BF414D0020C15B0020DC5B002095
:1018500004790020C04BC1491A684FF47A73B3FB76
:10186000F2F3C3EB431203EB8202059B1B68D20029
:10187000A1F8A82003F00403FEF7BEBA34F9111052
:101880009878B1F5617F4FF4966393FBF0F372DBC8
:1018900040F633008142A8BF01460C2DA1F56171CD
:1018A00091FBF3F100F00D81182D7FF464AAC9B209
:1018B000C8290B46A8BFC823DBF8E400C57D5FFA42
:1018C00083FEAE453FF457AA5B1BA54A80F817E09C
:1018D00048BF0733DB1092785D1CEDB23AB9002D9A
:1018E0003FF449AA284617F0ABFDFFF744BA182089
:1018F0001CF09AFBF3E79B499B4BCA681B688B6003
:101900009B1AC82B7FF629AB012381F82130FFF702
:1019100024BBD8F80010DBF81C200A44CBF81820B0
:10192000FFF7E5BB914B00220120A5E5F0EE477AD9
:10193000FEF7F8BCB0EE677AFEF7DEBC8C4A1268A0
:10194000970304D58B4A1279002A40F0EE808A4A28
:1019500018461946175C0B2F00F10C0023D00131FB
:101960001529F7D1002285F8A720FFF76BB8834B24
:101970000122022080E50C2D7AD100252946804BDA
:1019800009915B78AB423FF4F6A9284606F000F9CE
:10199000734B09999B781BB1C9B20C201CF044FB16
:1019A0000135EDB29BE7774FD7F800C04800BCF196
:1019B000000F09D000EB010E02EB8E0E9CF801C067
:1019C0009EF801E0E645CDD200EB010E6E486F496E
:1019D00002EB8E024FF0000E3A60A0F800E0C1F872
:1019E00000E0BFE7B0EE667AFFF7E7BBF0EE476ACC
:1019F000FFF7F9BBD8F80020BAF80630642101FBE4
:101A00000323CBF81030FFF748BB06231A4641E505
:101A100001231A463EE502231A463BE503231A46F4
:101A200038E504231A4635E505231A4632E505F064
:101A3000CBFA059B1B6803F00403FEF7DDB903F046
:101A400069FEEFF71FF803F04DFEFDF783FA012062
:101A500017F0F6FC95F8A620FFF710B8059B4C4A46
:101A60001B684FF4C871118003F00403FEF7C4B97A
:101A7000182D7FF480A900210B461DE70B464FF679
:101A8000FE71444A908956890144334453819181BF
:101A900003F040FEEEF7F6FF03F024FEFDF75AFADE
:101AA000012017F0CDFC059B1B68002203F0040306
:101AB00085F8A720FEF7A0B90B460221E1E7022333
:101AC000DFE7CDB25BE72F4FD7F800E04100BEF172
:101AD000000F08D00E1802EB86069EF801E076781B
:101AE0007645BEF489A90144274E284802EB8102BD
:101AF00000213A6031800160FEF77EB901210020AB
:101B00000AF097FC95F8A620FEF7DDBF0021FF2024
:101B10000AF08FFC95F8A620FEF7D2BF01200AF04C
:101B200088FC95F8A620FEF7C8BF1B4A1278002A49
:101B30007FF40DAF17F08AFB069B1B7803F00103BF
:101B400010E74FF6FE739CE70021012285F8A910EB
:101B500085F8AA20FEF750B9B86C002094640020E4
:101B6000414D0020DC5B0020009A0020D63400208C
:101B700098290020D05B0020081F03082035002092
:101B80000036002014240020622400206424002059
:101B9000FC9A0020E07800204F410020039A115D5C
:101BA0009847032C1BDC40F2EE2240F6CA0C0028BA
:101BB0003EF4A4AD39F824E0BAF802104FF47A7379
:101BC000A0EB0E0003FB00F0A1EB0E0190FBF1F087
:101BD00018449042B8BF10466045A8BF604600B2A6
:101BE000FEF78CBD002F3EF484A895F8A5E0BEF169
:101BF000000F3EF4B7A817F029FB96F800E085F82F
